:020000040800F2
:10000000F84D0320D54C00083F03000841030008C9
:1000100045030008490300084D03000800000000E4
:10002000000000000000000000000000890200083D
:100030005103000800000000DD020008D54B000855
:10004000EF4C0008EF4C0008EF4C0008EF4C0008A4
:10005000EF4C0008EF4C0008EF4C0008EF4C000894
:10006000EF4C0008EF4C0008EF4C0008EF4C000884
:10007000EF4C0008EF4C0008EF4C0008EF4C000874
:10008000EF4C0008EF4C0008EF4C0008EF4C000864
:10009000EF4C0008EF4C0008EF4C0008EF4C000854
:1000A000EF4C0008892C0008EF4C0008EF4C0008CA
:1000B000EF4C0008EF4C0008B9C50108EF4C0008F0
:1000C000EF4C0008EF4C0008EF4C0008EF4C000824
:1000D000EF4C000801310008EF4C0008EF4C00081D
:1000E000EF4C0008EF4C0008EF4C0008EF4C000804
:1000F000EF4C0008EF4C0008EF4C0008EF4C0008F4
:10010000EF4C0008EF4C0008EF4C0008EF4C0008E3
:10011000EF4C0008EF4C0008EF4C0008EF4C0008D3
:10012000EF4C0008EF4C0008EF4C0008EF4C0008C3
:10013000EF4C0008EF4C0008EF4C0008EF4C0008B3
:10014000EF4C0008EF4C0008EF4C0008EF4C0008A3
:10015000EF4C0008EF4C0008EF4C0008EF4C000893
:10016000EF4C0008EF4C0008EF4C0008EF4C000883
:10017000EF4C0008EF4C0008EF4C0008EF4C000873
:10018000EF4C0008EF4C000800F002F800F06CF8AB
:100190000AA090E8000C82448344AAF10107DA45E2
:1001A00001D100F061F8AFF2090EBAE80F0013F0C8
:1001B000010F18BFFB1A43F001031847B4AE070044
:1001C000D4AE07000A444FF0000C10F8013B13F0C6
:1001D000070408BF10F8014B1D1108BF10F8015BA0
:1001E000641E05D010F8016B641E01F8016BF9D193
:1001F00013F0080F1EBF10F8014BAD1C0C1B09D1EA
:100200006D1E58BF01F801CBFAD505E014F8016B5B
:1002100001F8016B6D1EF9D59142D6D370470000ED
:100220000023002400250026103A28BF78C1FBD8FF
:10023000520728BF30C148BF0B60704764291DF0CA
:10024000238375291DF0208363291DF0F885732908
:100250001DF0FD85002070471FB51EF01EFF1DF02C
:1002600051FD1FBD10B510BD1DF014FE1146FFF766
:10027000F3FF00F0D6FB1DF032FE03B4FFF7F2FFF0
:1002800003BC04F01DFD00002A4B19680868B0E8A3
:10029000F04F80F30988BFF36F8F4FF0000080F3B9
:1002A000118870470000000006480068006880F36D
:1002B000088862B661B6BFF34F8FBFF36F8F00DF60
:1002C00000BF00BF08ED00E0DFF80C00016841F45A
:1002D00070010160704700BF88ED00E0EFF3098016
:1002E000BFF36F8F134B1A681EF0100F08BF20ED7D
:1002F000108A20E9F04F106008B44FF0500080F3EE
:100300001188BFF34F8FBFF36F8F19F0B8FF4FF015
:10031000000080F3118808BC19680868B0E8F04F45
:100320001EF0100F08BFB0EC108A80F30988BFF3ED
:100330006F8F70476C020020EFF3058070477047A5
:1003400000BFFEE700BFFEE700BFFEE700BFFEE71D
:10035000704700005F48006840F080505D490860C9
:100360005D48006840F440405B49086059483838AF
:10037000006858493839086008460068086008462F
:10038000006840F4805008605448091F0860081F46
:10039000006840F08070091F086000BF4D48403879
:1003A000006800F000700028F8D040F202704C495C
:1003B000086048483838006820F00300454938395B
:1003C00008600846006840F00200086000BF41482D
:1003D0003838006800F00C000828F8D1704710B5D4
:1003E00000BF00BF00BF00BF3E48006840F470007F
:1003F0003C49086037484038006840F00100354902
:1004000040390860002033493839086031484038A5
:100410000068354908402F49403908603348091DB4
:100420000860081F006820F48020091F0860002071
:10043000284934390860FFF78DFF10BD70B50020E2
:100440000021022200230224224D383D2D6805F0B0
:100450000C0020B1042806D0082829D107E0244D3B
:10046000244E356028E0244D224E356024E0194D9D
:100470003C3D2D68C5F38053164D3C3D2D6805F07D
:100480003F044BB91A4DB5FBF4F5124E3C3E3668AD
:10049000C6F3881605FB06F10E4D3C3D2D68C5F3ED
:1004A00001456D1C6A00B1FBF2F5124E356003E0A8
:1004B0000F4D104E356000BF00BF064D383D2D6812
:1004C000C5F303150D4E705D0A4D2D68C540094EEC
:1004D000356070BD40380240007000401064010774
:1004E000003C024088ED00E0FFFFF6FE10300024E3
:1004F0000024F4000000002000127A000400002014
:100500001CB50121084604F09BFF4FF48070009059
:1005100000208DF8040003208DF8050001208DF8DF
:1005200007006946FE4804F0EBFCFE4801F0B7F80E
:10053000FD481CF05BF81CBD00B589B00020FB49EC
:100540000870FB490870FB490870FB490870FB49BB
:1005500008600021FA4A11605160FA490860F148C8
:1005600001F09DF8642018F06CF8F74802F08EFF57
:100570000A2018F066F801A9F44803F0C8F9EA481F
:100580001CF02CF8E74800F088FEF148007830B9FC
:100590000120F04908701220EF49087012E0EC4881
:1005A00000785A280ED10420EA490870EB480078F8
:1005B000012807DBE9480078122803DCE7480078C7
:1005C000E5490870E5480078122802DD1120E2496B
:1005D000087009B000BD0BE0642019F027FDD24877
:1005E0001CF07AF8D0481CF0EEF80020DC49486195
:1005F000F2E708B51AF00FF800901EE0D94800683D
:10060000401CD84908600A21684619F0B4FCD64855
:1006100001F055FBD44802F00AFED24800680A21D6
:10062000B0FBF1F201FB120020B9D04802F0CEFE7F
:1006300005F0BFFC0020CA490861DFE79DE000200B
:10064000C749C860BB480078002872D002F0CDFCD2
:10065000C82019F0EBFC02F0E7FCC82019F0E6FC1A
:1006600002F0C3FCC82019F0E1FC02F0DDFCC82058
:1006700019F0DCFC02F0B9FCC82019F0D7FC02F03C
:10068000D3FC4FF4FA7019F0D1FC0020B449C860D3
:1006900002F0ABFC4FF4C87019F0C8FC02F0C4FCC7
:1006A000C82019F0C3FC02F0A0FC4FF4C87019F088
:1006B000BDFC02F0B9FCC82019F0B8FC02F095FCB2
:1006C0004FF4C87019F0B2FC02F0AEFC4FF4FA70AF
:1006D00019F0ACFC0020A249C86002F086FCC820DA
:1006E00019F0A4FC02F0A0FCC82019F09FFC02F055
:1006F0007CFCC82019F09AFC02F096FCC82019F086
:1007000095FC00209649C86002F06FFCC82019F0E3
:100710008DFC02F089FC002407E000209049C860AD
:100720004FF4C87019F082FC641C052C25D2F4E744
:10073000FFE781480078012806D102F056FC4FF40B
:10074000FA7019F073FC18E07948007801280CD190
:1007500002F04BFC4FF4FA7019F068FC02F064FCF4
:100760004FF4FA7019F062FC07E002F05DFC6420BF
:1007700019F05CFC7E4803F047FD60E708B519F00E
:100780004AFF009019E000207549886067480078AA
:1007900003280EDA0A21684619F0EDFB75481BF0B4
:1007A000CAFD6C480078012807D15E4800F077FF49
:1007B00003E04FF47A7019F039FCE4E711E000200F
:1007C0006749486059480078032806DA142019F070
:1007D0002DFC694816F00EFC03E04FF47A7019F016
:1007E00025FCECE708B519F016FF009011E0002099
:1007F0005B4908604D480078032806DA0121684605
:1008000019F0B9FB11F0B5FE03E04FF47A7019F05E
:100810000DFCECE71CB504460121080304F010FEB2
:100820001BF0BDF817F0C4FF544908605448042178
:1008300000230A02CDE9001052A1AFF2570019F0CF
:1008400077F95448052100234FF48062CDE9001068
:1008500051A1AFF2970019F06BF953480221002320
:10086000CA01CDE9001051A1AFF2EF0019F060F913
:100870005248032100238022CDE9001050A1AFF29D
:10088000432019F055F95148062100234FF4807296
:10089000CDE900104EA1AFF2A52019F049F94F485B
:1008A000072100234FF48072CDE900104CA1AFF274
:1008B000D92019F03DF91BF095F81A4800F0FCFA20
:1008C000642019F0B3FB174800F087FC1CF04BFACA
:1008D000642019F0ABFB1CF0D4FA44A1224802F0CA
:1008E00098FC322019F0A2FB0E4800F08BFA32205F
:1008F00019F09CFB45F2555005F052FB032005F022
:1009000052FB40F6FF7005F051FB002005F048FB5C
:1009100005F054FB00203F4908603F4800687DE037
:1009200000000240B000002072430320C8000020F5
:100930003500002036000020340000202C0000206C
:100940001800002028000020F3180020121A0020B0
:1009500057000020370000205500002054000020E0
:100960000C030020AC0000206A040020CE00002010
:10097000182B0020604303200002002040000020CC
:100980009C0000206C6974746C655F76676C5F74A2
:1009900061736B00A0000020646973706C61795F03
:1009A0007461736B00000000940000204B65796255
:1009B0006F6172645F7461736B00000098000020C7
:1009C0006C6564305F7461736B000000A4000020EC
:1009D000556172745F7461736B000000A8000020A1
:1009E00052463433335F7461736B00005379732064
:1009F0007374617274696E672C63726561746520CB
:100A000036207461736B73202E2E2E2E2E2E0D0A1F
:100A100000000000B48240429000002019F0D6F897
:100A20001CBD1CB500BF00BF00BF00BF2A481BF0A3
:100A3000B6F900240BE04FF48061284804F0C2FAB4
:100A400018B9274800F00CFE00E003E0641C2548BC
:100A50008442F0D300BF224800F021FE4FF0006036
:100A60002149086007230222C821102002F0F5F96D
:100A7000642004F0B7F84FF4407004F04BF94FF4E1
:100A8000E1311A4802F060FBFFF73AFDFFF754FD31
:100A90001CF0F7F901F0FDFD0F481BF080F9144838
:100AA00003F057FB4FF4FA61124802F081FC08F0A2
:100AB000E1FA15F0F6FE15F01EFF0F4801210023A4
:100AC0000A02CDE900100DA1AFF2B72019F030F8FD
:100AD00019F057FD00201CBD6043032000040240B4
:100AE000B0000020A086010008ED00E06A040020AC
:100AF000182B0020CE00002090000020737461723B
:100B0000745F7461736B000070477047012080F35D
:100B1000108800BF7047002080F3108800BF704726
:100B200010B5034600200FE0002207E000BF00BF21
:100B300000BF00BF00BF00BF541CA2B241F2A864B6
:100B4000A242F3DB441CE0B28842EDDB10BD7FB56E
:100B5000064600BF00BF0020F8490860F84800685A
:100B6000401CF7490860F7480068401CF5490860D8
:100B7000F34800680A2802D2F3481BF0C9FCF34886
:100B80000068401CF149086008464068401C486005
:100B900008468068401C88600846C068401CC860E1
:100BA00008464069401C486108460069401C0861CD
:100BB000E748007800B17FBD00250020E549886046
:100BC000E2480068052800D93125E048406805283A
:100BD00000D93225DD488068052800D93325DB4857
:100BE000C068052800D93425D8484069052800D9AF
:100BF0003525D6480069052800D9362525B1D648BF
:100C00000078401CD4490870D3480078012801D1ED
:100C1000D2490870D048007805282DDDD048D0F89A
:100C2000AC00401CCE49C1F8AC00CE4968461CF06F
:100C3000A5FE8DF80750002409E01DF80400CA49FC
:100C4000888032213046FFF76BFF601CC4B20A2C4B
:100C5000F3DBFFF75BFF00BFBFF34F8FC3480068B4
:100C600000F4E060C2490843001DC0490860BFF3BA
:100C70004F8F00BF00BFFEE700BF9CE710B5BD4827
:100C8000FFF765FF10BD7047704770B5A0B006460E
:100C90000D46012D27D100228021684617F060F90A
:100CA00000240CE04FF6FF7000EA44116B4620224E
:100CB000B14802F066FD0A2019F0B8F9641C202C36
:100CC000F0D3AE4968461CF059FE6B461022002155
:100CD000A94802F056FD0A2019F0A8F9A8A1AF48CA
:100CE00002F097FA03E0AEA1AC4802F092FAAB48EA
:100CF00002F09DFA012019F099F9012D11D100207F
:100D0000944908704870782048804FF4615088807A
:100D10004FF41670C8800B4608227621964802F0E0
:100D200030FD20B070BD70B590B0064600BF00BF6A
:100D30000020A24908608249086008AB1022002107
:100D40008D4802F0DEFC6B46102211468A4802F004
:100D5000D8FC0A2019F06AF9002500240FE008A841
:100D6000005D8649095D884205D01DF8040094495C
:100D7000095D884201D1681CC5B2601CC4B2102C48
:100D8000EDDB0F2D1CDA01213046FFF77EFF7B4B98
:100D900010220021784802F0F4FC0A2019F046F9EC
:100DA000874B10221146744802F0EBFC0A2019F020
:100DB0003DF984A1794802F02CFA002061490860CD
:100DC00000BF00BF00BF00BF624B082276216A4807
:100DD00002F097FC10B070BD704710B503460020BC
:100DE0000DE0002207E000BF00BF00BF00BF00BF52
:100DF00000BF541CE2B2022AF5DB441CA0B28842B8
:100E0000EFDB10BD10B58AB0044600BF00BF00BFC5
:100E100000BF00221821724817F0A2F800222021FA
:100E200001A817F09DF810226E496D481CF03AFE9B
:100E300000206B49087448746BA1584802F0E9F926
:100E40006749564802F0E5F95BA1544802F0E1F920
:100E500068480168514802F0DCF9674801684F486A
:100E600002F0D7F965A14D4802F0D3F96448016852
:100E70004A4802F0CEF961A1484802F0CAF90022BE
:100E8000202101A817F06CF804225E48016809A827
:100E90001CF07CFE01A9099817F038F901A93F4818
:100EA00002F0B7F944A13D4802F0B3F90AB010BD11
:100EB000704700BF00BF704730B589B0054600BF1E
:100EC00000BF5148046804F07C44A40E082C30D0C4
:100ED00006DC062C2ED2DFE804F0DC1015212627D4
:100EE000112C28D004DC092C26D0102C22D1C4E0EF
:100EF000202C22D0212CF9D1C6E044A101A81CF05D
:100F00003DFDCBE047A101A81CF038FD1448D0F806
:100F1000B000401C1249C1F8B000BFE046A101A8D2
:100F20001CF02CFDBAE000BF49A101A81CF026FD71
:100F3000B4E095E0ADE0A1E093E0A4E02000002063
:100F40002C00002030000020604303200C03002010
:100F5000C800002024030020B40000204800002026
:100F600030030020A4F00108001001400CED00E067
:100F70000000FA05B0000020F4180020C2F00108BB
:100F8000526573746F726520466163746F72792065
:100F9000446565706C790D0A000000006A04002049
:100FA000526573746F726520466163746F72792045
:100FB000536C696768746C790D0A00002400002086
:100FC000B0F0010873797374656D2066697273748B
:100FD0002072756E20666C61670D0A0000000000CB
:100FE000F4020020A020000844657669636520496A
:100FF000443A000084000020780000202000000017
:101000007C00002074000020743802400D0A5265F4
:101010007365742050696E2052657365740D0A0003
:10102000000000000D0A506F776572204F6E20524D
:10103000657365740D0A00000D0A506F7765724F75
:101040006E20526573657450696E0D0A00000000D1
:101050000D0A536F66742052657365740D0A0000A3
:1010600000BFF2A101A81CF089FCF648D0F8B4003A
:10107000401CF449C1F8B40010E000BFF2A101A87F
:101080001CF07CFC0AE000BFF5A101A81CF076FC76
:1010900004E0F9A101A81CF071FC00BF00BFFE48EC
:1010A000006840F08070FC49086001A9FB4802F02C
:1010B000B0F800BF00BF09B030BD704700BF00BF2F
:1010C00070472DE9F04107460C46F54800780028A6
:1010D00039D0F448016820461CF050FCF2A12046AB
:1010E0001CF08FFC20461CF06DFCC5B26119EF4A64
:1010F0001268106816F0A9FDEBA120461CF081FCD7
:1011000020461CF05FFCC5B26119E94A12681068FC
:1011100016F09BFDE4A120461CF073FC20461CF059
:1011200051FCC5B2E3480268E3480168E34803F0B4
:1011300068FC06466119304616F087FDC0A12046BE
:101140001CF05FFC46E0D748016820461CF016FC06
:10115000D5A120461CF055FC20461CF033FCC5B23E
:101160006119D24A1268106816F095FFCEA1204688
:101170001CF047FC20461CF025FCC5B26119CC4A86
:101180001268106816F087FFC7A120461CF039FCD2
:10119000C948016820461CF034FCC3A120461CF05D
:1011A00030FCC448016820461CF02BFCBEA1204640
:1011B0001CF027FC20461CF005FCC5B2BD480268A7
:1011C000BD480168BD4803F01CFC06466119304665
:1011D00016F03BFDBDE8F081704710B58CB00446B9
:1011E000684604F05CF8B6A1AC4802F012F8202181
:1011F00004A81CF032FD04A9009816F087FFAFF296
:10120000482104A81CF0FDFBB3A1A44802F001F89A
:1012100004A9A24801F0FDFF202104A81CF01DFD37
:1012200004A9019816F072FFAFF2742104A81CF013
:10123000E8FBACA1994801F0ECFF04A9974801F044
:10124000E8FF202104A81CF008FD04A9029816F06C
:101250005DFFAFF29C2104A81CF0D3FBA3A18F4833
:1012600001F0D7FF04A98D4801F0D3FF202104A885
:101270001CF0F3FC04A9039816F048FFAFF2C82154
:1012800004A81CF0BEFB9BA1844801F0C2FF04A986
:10129000824801F0BEFF0CB010BD10B5C2B00446CC
:1012A0006A464FF4FF51954802F080FC9DF800001B
:1012B0009DF80110884208D19DF80100FF2804D054
:1012C0009DF800008E49087002E008208C490870E3
:1012D0009DF802009DF80310884208D19DF8020095
:1012E000FF2804D09DF802008649087002E0022021
:1012F000844908709DF804009DF80510884208D1C3
:101300009DF80500FF2804D09DF804007E49087070
:1013100002E000207C4908709DF808009DF8091043
:10132000884208D19DF80900FF2804D09DF80800E4
:101330007649087002E00020744908709DF80C009E
:101340009DF80D10884208D19DF80D00FF2804D0AB
:101350009DF80C006E49087002E000206C4908708E
:101360009DF810009DF81110884208D19DF81000DA
:10137000FF2804D09DF810006649087002E00020A4
:101380006449087064490A98884207D063490B98F9
:10139000884203D000206249086002E06049089852
:1013A000086060A13D4801F034FF6B464FF4807245
:1013B00001213A4801F060FEAFF20441374801F0E4
:1013C00028FF6A4601214D4802F0F0FB5CA133483A
:1013D00001F01FFF6B464FF4807201212F4801F08E
:1013E0004BFEAFF22C412D4801F013FF42B010BD6F
:1013F000F0B5C3B007460025002605224FF4FF7163
:101400003E4802F0DBFC322018F010FE0024534866
:1014100002782146641C01A84254504802782146B3
:10142000641C01A842543748027899E00D0A49200B
:101430005761746368646F672052657365740D0A41
:1014400000000000300300200D0A5720576174632C
:1014500068646F672052657365740D0A00000000B0
:101460000D0A4C6F7720506F776572205265736557
:10147000740D0A00000000000D0A446F6E277420EE
:101480006B6E6F7720726561736F6E205265736546
:10149000740D0A0000000000743802406A04002045
:1014A000C8000020680000202C0000006C00002014
:1014B000700000207C00002078000020582B0020C5
:1014C0000A53797374656D206672657175656E6314
:1014D000793A0D0A00000000535953434C4B3A002F
:1014E0000000000048434C4B3A00000050434C4B76
:1014F000313A000050434C4B323A0000121A00209F
:101500005400002056000020570000205800002002
:10151000590000205A0000205555AAAAFE7F5A5AA9
:10152000300000200A4C6F616420706172656D6547
:10153000746572205465737420446174613A0000CC
:101540000A466C61736820706167652031205465BC
:10155000737420446174613A00000000550000205B
:101560002146641C01A842546E4802782146641C3E
:1015700001A842546C4802782146641C01A84254D8
:10158000694802782146641C01A8425466480278E2
:101590002146641C01A84254634802782146641C19
:1015A00001A84254614802782146641C01A84254B3
:1015B0005E4802782146641C01A842545B480278C8
:1015C0002146641C01A84254584802782146641CF4
:1015D00001A84254564802782146641C01A842548E
:1015E000534802782146641C01A8425450480278AE
:1015F0002146641C01A842544D4802782046611CD3
:101600008CB201A90A544B4802782046611C8CB266
:1016100001A90A54474802782046611C8CB201A9EE
:101620000A54444802782046611C8CB201A90A542D
:10163000404802782046611C8CB201A90A543E48F9
:1016400000680A9009903D480B903D480C90032398
:1016500001AA4FF4FF513B4802F001FC43B0F0BD3A
:101660001CB504460121084603F0EAFE4FF4004190
:10167000354803F0C1FC4FF40140009000208DF884
:10168000040001208DF8060003208DF805000020DD
:101690008DF8070069462C4803F032FC1CBD1CB5D0
:1016A00004460121084603F0CBFE0121022003F08D
:1016B000C7FE4FF40040009001208DF80400002088
:1016C0008DF8060003208DF8050001208DF8070035
:1016D00069461D4803F014FC69461C4803F010FCE1
:1016E0004FF48070009000208DF804008DF8060003
:1016F00003208DF8050001208DF807006946124887
:1017000003F0FEFB4FF400410F4803F077FC4FF469
:1017100000410E4803F072FC1CBD00B50C48FFF7F9
:10172000B2FA00BD560000205700002058000020EB
:10173000590000205A000020300000205555AAAA68
:10174000FE7F5A5A121A0020000002400004024094
:10175000B000002070B505460E4600BF41F26D0096
:10176000284490F80D040028F8D1552484F07A0418
:10177000744000BF5520FA498880012018F056FCBB
:101780007A20F7498880012018F050FCF4488680C0
:10179000012018F04BFC0020F1498880012018F04E
:1017A00045FCEF488480012018F040FC002041F205
:1017B0006D012944A1F80E0470BD70472DE9F8436E
:1017C00080460C460027A089B0F5006F52DCE08906
:1017D000B0F5806F4EDC02E0012018F027FCE148F4
:1017E00080780028F8D102E0012018F01FFCDD48C5
:1017F00000880028F8D10120DA498870668960895C
:1018000000B1761E002510E0102000EB0523D5481E
:10181000C01C1A1805EB8601D34802F0C7F9C8218D
:10182000D14802F099FA681CC5B2042DECDB4FF4E4
:101830008060E08110222146CA48C01C1CF032F9A9
:10184000C8490B314FF4816016F0EAFC0090042285
:101850006946C448C01D1CF025F94FF48260C14997
:10186000088000208870084601F0E1FC142018F080
:10187000DDFB00E001273846BDE8F8832DE9F041A3
:1018800080460D46A889B0F5006F3CDCE889B0F5CC
:10189000806F38DC687A3138022834DAB34800784F
:1018A000022803D0B148007803282CD1687A312867
:1018B00001D1002601E04FF400666C8904B1641E7A
:1018C000A400264406F00F0018B93109A64802F01A
:1018D00092F8002413E04FF4FA71A34802F03CFAA6
:1018E000102000EB042308F603001A1831199E4853
:1018F00002F09DF9C8219C4802F02EFA641C042CC9
:10190000E9D3002700E001273846BDE8F0812DE942
:10191000F041C6B007464FF00008002600224FF401
:10192000887102A816F01CFB07F60304E18901F197
:10193000080007F60B0116F073FC0190606801992E
:1019400088427DD1207A313805287AD2DFE800F04C
:101950000304348B960000BF15F0ADFF8348007878
:1019600030B9207A312803D101208049087016E06F
:101970007E480078012806D102207C4908700020AA
:101980007B4908700BE079480078022805D1774937
:10199000087000207649087001E04FF00108B8F1A6
:1019A000010F08D006A97348FFF78BFB4FF47A703C
:1019B000714908602C2667E021463846FFF75EFF34
:1019C0000546002D4CD16089A18988423FD16B48E2
:1019D000D0F8A400401C6949C1F8A4006548FFF78D
:1019E000FBFB1022214602A81CF05CF8022264A135
:1019F00006A81CF059F91226A6F1080004A916F051
:101A00000FFC0190042201A903A81CF0BFF802AB4F
:101A100032460021384601F02FFB524801F007FC06
:101A20000A2018F003FB00BFBFF34F8F5548006832
:101A300000F4E06054490843001D5249086001E089
:101A400023E01EE0BFF34F8F00BF00BFFEE703207F
:101A5000464908704FF47A7047490860102601E043
:101A60004FF0010810E021463846FFF7A7FE054673
:101A70000DB9002601E04FF0010805E04FF0010824
:101A800002E04FF0010800BF01E04FF00108B8F19B
:101A9000010F06D102223DA106A81CF005F912266D
:101AA00007E0102E05D1022235A106A81CF0FCF893
:101AB0001226AEB11022214602A81BF0F3FFA6F1B8
:101AC000080004A916F0ACFB0190042201A903A8A8
:101AD0001CF05CF802AB32460021384601F0CCFA2B
:101AE000207A31280ED12148007801280AD13846C1
:101AF00001F09DFB0A2018F099FA4FF4E1313846C5
:101B000001F022FB46B0BDE8F0812DE9F043C5B0FD
:101B1000054600BF00BF00BF00BF4FF0000900270F
:101B200040F6050010F80580B8F1280F03D0B8F191
:101B30002A0F6ED148E000BF00BF05F6090440F649
:101B40000900465D532E30D1A078522822D1E28878
:101B5000A1880DF10A030E4801F0D3FDE78830E0BB
:101B6000001001406A040020121A0020C800002062
:101B7000B5000020B0000020C40000203003002089
:101B80004F4B00000CED00E00000FA05455200004C
:101B9000F4180020A078572813D1E288A18805F610
:101BA00011036A4801F0EDFD0BE0492E05D1A07844
:101BB000522801D1E78804E003E0452E01D04FF020
:101BC0000109B81D87B241E005F6090440F6090095
:101BD000465D462E32D1A07852281BD1E0784428A9
:101BE00008D1A1880DF10A02594801F0DFFF4FF436
:101BF000807725E0E078532822D1554801F0B5FEE2
:101C00008DF80A000DF10B01514801F059FE05272E
:101C100016E018E0A078572807D1A18804F108023F
:101C20004B4802F004F800270AE0A078452807D1C5
:101C3000A188474801F02EFF002701E04FF001097D
:101C4000B81D87B202E04FF0010900BF00BFB9F133
:101C5000000F0AD0B8F1800F01DAFA2600E0FB2667
:101C600031462846FFF776FD20E055208DF8040028
:101C70007A208DF805008DF80680B81FC11700EB9B
:101C80001161090A8DF80710C11700EB11610912E3
:101C9000A0EB0121C9B28DF8081000208DF80900D1
:101CA00001AB3A460021284601F0E6F9002128461A
:101CB00001F032FA00BF00BF45B0BDE8F0832DE966
:101CC000F041044604F60300D0F86608401C04F610
:101CD0000301C1F86608032801D0BDE8F08104F6CD
:101CE0000300B0F8640800B9F7E704F603052846D6
:101CF000B0F86468002794F80308AA2808D140F6D1
:101D00000400005D752803D12046FFF7FEFE15E0B4
:101D100094F80308472811D140F60400005D4928D3
:101D20000CD140F60500005D412807D140F60600C1
:101D3000005D502802D12046FFF7E9FD0021204632
:101D400001F0EAF900BFC8E770477047F4180020B7
:101D5000121A00201CB5FE480068AA2800D11CBD3C
:101D60003C20009001208DF8040000208DF8060032
:101D700003208DF8050001208DF807006946F5481D
:101D800003F0BEF84FF48040009001208DF804006D
:101D900000208DF8060003208DF8050001208DF845
:101DA00007006946EC4803F0ABF84FF4C2500090CE
:101DB00001208DF8040000208DF8060003208DF826
:101DC000050001208DF807006946E44803F098F803
:101DD0000120E3490860E349C1F88802E049091F8E
:101DE0000860AA20DA49086000BFB8E71CB5D848E7
:101DF0000068552800D11CBD3C20009000208DF8C3
:101E0000040003208DF8050001208DF807006946C5
:101E1000D04803F075F84FF48040009000208DF812
:101E2000040003208DF8050001208DF807006946A5
:101E3000C94803F065F84FF4C250009000208DF8B7
:101E4000040003208DF8050001208DF80700694685
:101E5000C24803F055F80120C1490860C149C1F8E2
:101E60008802BF49091F08605520B949086000BFB2
:101E7000C1E708B500909DF8001001F00101BA4AD1
:101E800011609DF80010C1F34001B84AC2F89812E1
:101E90009DF80010C1F38001B14A183211609DF81D
:101EA0000010C1F3C001B14AC2F8B0129DF8001091
:101EB000C1F30011AE4AC2F888129DF80010C1F3B8
:101EC0004011C2F88C129DF80010C1F38011C2F8C5
:101ED00090129DF80010C909C2F8941208BD10B5FF
:101EE000002420219B4803F06DF8012801D144F023
:101EF00080041021974803F065F8012801D144F0CF
:101F000040040821934803F05DF8012801D144F012
:101F1000200404218F4803F055F8012801D144F032
:101F200010044FF480518D4803F04CF8012801D182
:101F300044F008044FF40061884803F043F8012896
:101F400001D144F004044021844803F03BF8012807
:101F500001D144F002044FF480417F4803F032F88D
:101F6000012801D144F00104204610BD10B50446FB
:101F7000FFF7F0FE00207A490839086001207B490C
:101F8000C1F8940200207649091F08602046FFF737
:101F900070FF00207349C1F8880200BF0120754915
:101FA00008607249C1F8900210BD10B50446FFF7F1
:101FB000D1FE01206A49083908606C49C1F89402D1
:101FC00000206749091F08602046FFF752FF0020E4
:101FD0006449C1F8880200BF01206649086063496E
:101FE000C1F8900210BD10B5044600205C49091FDD
:101FF00008602012FFF73DFF00205A49C1F888020F
:1020000000BF01205B490860E0B2FFF732FF00200B
:102010005449C1F8880200BF01205649086053495D
:10202000C1F8900210BD10B5FFF7E0FE01204C4949
:10203000083908604B49C1F8880200204849091F47
:10204000086000BF00204949C1F8940200BFFFF7B3
:1020500046FF04460120424908604449C1F8900205
:10206000204610BD2DE9F04104460D4616461F4698
:102070002A20FFF77BFF2012FFF797FFE0B2FFF760
:1020800094FF3012FFF791FFF0B2FFF78EFF2B2085
:10209000FFF76CFF2812FFF788FFE8B2FFF785FF14
:1020A0003812FFF782FFF8B2FFF77FFF2C20FFF70F
:1020B0005DFFBDE8F08170B50646EF2340F23F12A8
:1020C00000210846FFF7CEFFFFF744FE0120244918
:1020D000083908602549C1F8940200240BE0002566
:1020E00004E03046FFF77FFF681C85B2B5F5A07F9E
:1020F000F7DB601C84B2F02CF1DB70BD1CB54FF433
:102100002040009001208DF8040000208DF806008A
:1021100002208DF8050001208DF8070069460E4861
:1021200002F0EEFE4FF48060009001208DF8040074
:1021300000208DF8060002208DF8050001208DF8A2
:1021400007006946054802F0DBFE0120064913E05E
:10215000BC000020000002400004024000080240D1
:102160009402414200804142B88240420000414214
:102170000000404288824142091D0860FE49C1F8C2
:10218000B4021CBD1CB501210F2003F059F93C20FD
:10219000009001208DF8040000208DF80600032037
:1021A0008DF8050001208DF807006946F34802F01C
:1021B000A7FE4FF48040009001208DF8040000201D
:1021C0008DF8060003208DF8050001208DF807002A
:1021D0006946EB4802F094FE41F678000090012039
:1021E0008DF8040000208DF8060003208DF805000E
:1021F00001208DF807006946E24802F081FE0420C4
:10220000009001208DF8040000208DF806000320C6
:102210008DF8050001208DF807006946DA4802F0C4
:102220006FFE1CBD10B5FFF769FF0020D74908609D
:102230004FF4967016F005FA0120D549C1F8A802AE
:10224000322016F0FEF90020D2490860C82016F0AE
:10225000F8F90120CE49C1F8A8024FF4FA7016F03F
:10226000F0F910BD10B5FFF78DFFFFF7DBFFC820B9
:10227000FFF77CFEFF20FFF798FE9320FFF795FE07
:102280004220FFF792FE3620FFF770FEC820FFF7CE
:102290008CFE3A20FFF76AFE5520FFF786FEC0202D
:1022A000FFF764FE1320FFF780FE0E20FFF77DFE90
:1022B000C120FFF75BFE0220FFF777FEC520FFF786
:1022C00055FED320FFF771FEB120FFF74FFE00202F
:1022D000FFF76BFE1B20FFF768FEB420FFF746FEFA
:1022E0000220FFF762FEE020FFF740FE0020FFF72C
:1022F0005CFE0320FFF759FE0820FFF756FE06207C
:10230000FFF753FE1320FFF750FE0920FFF74DFEA5
:102310003920FFF74AFE3920FFF747FE4820FFF734
:1023200044FE0220FFF741FE0A20FFF73EFE082090
:10233000FFF73BFE1720FFF738FE1720FFF735FEAB
:102340000F20FFF732FEE120FFF710FE0020FFF71D
:102350002CFE2820FFF729FE2920FFF726FE01206A
:10236000FFF723FE0D20FFF720FE0320FFF71DFEE1
:102370003F20FFF71AFE3320FFF717FE5220FFF72A
:1023800014FE0420FFF711FE0F20FFF70EFE0E20B3
:10239000FFF70BFE3720FFF708FE3820FFF705FE9A
:1023A0000F20FFF702FE1120FFF7E0FD782016F066
:1023B00048F92920FFF7DAFD10BD01B5BDF800107E
:1023C000C8B2FFF7D3FD08BD01B5BDF80010C8B213
:1023D000FFF7EBFD08BD08B5FFF725FE0090BDF83F
:1023E000000008BD70B505460C46E8B2FFF7BEFD1B
:1023F0002012FFF7DAFDE0B2FFF7D7FD70BD10B590
:1024000004462046FFF7D9FF052002F008FCFFF73D
:10241000E2FF10BD10B52C20FFF7A8FD10BD30B5B0
:10242000014601F01F04C1F34513CA0AE50205EB9A
:1024300043151544A8B230BD00BF011EA0F1010232
:10244000D0B2FAD1704770B504460D46524948895A
:10245000FFF7B3FF2012FFF7B7FFE0B2FFF7B4FFBB
:102460004D498889FFF7A9FF2812FFF7ADFFE8B2B1
:10247000FFF7AAFF70BD2DE9F04104460D46002686
:102480000027B04644480088A04203DD4248408807
:10249000A84202DC0020BDE8F08129462046FFF773
:1024A000D2FF2E20FFF789FFFFF795FF0646022097
:1024B000FFF7C2FFFFF78FFF06460220FFF7BCFFC2
:1024C000FFF789FF8046F7B24FF6FF7000EA072753
:1024D0003046FFF7A4FFDEE710B52920FFF76DFFB8
:1024E00010BD10B52820FFF768FF10BD10B50446D9
:1024F0003620FFF73BFD2046FFF757FD10BD70B5B6
:1025000004460D4629462046FFF79DFFFFF782FF50
:10251000FFF720FC01201F491C3908601C49C1F845
:1025200094021E480088FFF75EFD70BD70B504463A
:102530000D46164618494889FFF73FFF2012FFF75E
:1025400043FFE0B2FFF740FF13498889FFF735FFEB
:102550002812FFF739FFE8B2FFF736FF0E49087A75
:10256000FFF704FDFFF7F6FB01200A491C3908605C
:102570000749C1F8940213E0008040420000024085
:102580000004024000080240000C0240BC824042AD
:1025900000004142A80241425C040020B800002033
:1025A0003046FFF720FD70BD70B52DED048B04465D
:1025B000BE20FFF702FF0520FFF706FF20461CF0B4
:1025C000F3FA41EC190B9FEDF70B53EC102B1CF0B9
:1025D000FFFA41EC180B1CF0A3FA85B22846FFF76E
:1025E000F3FE0120FFF7F0FEFF20FFF7EDFE0020D5
:1025F000FFF7EAFE0020FFF7E7FEBDEC048B70BD9D
:1026000018B90021E94A917102E00121E74A91716C
:102610004FF4A071E54A1180F02151802A215181A7
:102620002B2191812C21118170472DE9F04704461F
:102630000D4616461F46A019401E1FFA80F8E819DD
:10264000401E1FFA80F9D9494889FFF7B6FE2012CB
:10265000FFF7BAFEE0B2FFF7B7FE4FEA2820FFF718
:10266000B3FE08F0FF00FFF7AFFED0498889FFF7FF
:10267000A4FE2812FFF7A8FEE8B2FFF7A5FE4FEA76
:102680002920FFF7A1FE09F0FF00FFF79DFEBDE83E
:10269000F08710B549F24130C4498880FFF7E2FD68
:1026A00049F24130C14988800120FFF7A9FF10BDE0
:1026B00010B504462046FFF7FEFC10BD2DE9F05F83
:1026C00005460E4617469846DDF828A04FF0000B49
:1026D000781B401C1FFA80FB34461BE0214628462D
:1026E000FFF7B1FEFFF796FEFFF734FB0120B0497C
:1026F0000860B049C1F894024FF0000906E0504666
:10270000FFF771FC09F101001FFA80F9D945F6DBEA
:10271000601C84B24445E1DDBDE8F09F2DE9F84F2F
:1027200007460D4690469946DDF828B0A8EB07000D
:10273000401C1FFA80FAA9EB0500401C80B20090F3
:1027400000241CE0281981B23846FFF77CFEFFF711
:1027500061FEFFF7FFFA0120954908609549C1F82D
:102760009402002607E004FB0A613BF81100FFF722
:102770003AFC701C86B25645F5DB601C84B20098AA
:102780008442DFDBBDE8F88F2DE9FF4F85B081463D
:102790008A460020049003900798A0EB090508984A
:1027A000A0EB0A06CDF80890CDF804A0002D01DDBD
:1027B000012705E00DB9002702E04FF0FF376D4219
:1027C000002E02DD4FF0010806E016B94FF00008B8
:1027D00002E04FF0FF387642B54201DD2C4600E0C2
:1027E00034464FF0000B21E0019A91B2029A90B268
:1027F000FFF785FE04982844049003983044039022
:102800000498A04205DD0498001B04900298384407
:1028100002900398A04205DD0398001B03900198E5
:10282000404401900BF101001FFA80FB601C8345BE
:10283000DADD09B0BDE8F08F2DE9F04104460D4620
:1028400016461F462B46324629462046FFF79CFF78
:102850003B46224629462046FFF796FF3B46324636
:1028600039462046FFF790FF3B4632462946304620
:10287000FFF78AFFBDE8F0812DE9F04706460F46D5
:102880009046002445460320A0EB48093CE07A1B13
:1028900091B2321990B2FFF732FE3A1B91B272191F
:1028A00090B2FFF72CFE3A1991B2721990B2FFF76D
:1028B00026FE7A1991B2321990B2FFF720FE7A19EA
:1028C00091B2321B90B2FFF71AFE3A1991B2721B05
:1028D00090B2FFF714FE7A1B91B2321B90B2FFF751
:1028E0000EFE3A1B91B2721B90B2FFF708FE641CF9
:1028F000B9F1000F03DAA000801D814404E0601BE1
:1029000080000A3081446D1EAC42C0DDBDE8F08716
:102910002DE9F84F80460E4617461C46B346204622
:10292000E31704EB5373DB1021464FEAE47C04EB1E
:102930005C7C4FEAEC0CA4EBCC0CBCF1000F02D099
:102940004FF0010C01E04FF0000C6344224604EB11
:10295000D27C4FEA6C0C03FB0CF3DBB20093A7F1C3
:102960002000C7B2002566E00C2C07D107EB47001A
:10297000114901EB800010F8059023E0102C05D1DF
:102980000E4800EB071010F805901BE0182C07D13B
:1029900007EBC7000A4901EB800010F8059011E031
:1029A000BDE8F88F66666666666604405C040020D3
:1029B0008C02414200004142D3F0010847F5010872
:1029C00037FB01084FF0000A2FE009F0800030B11A
:1029D0008F48028831464046FFF7A8FD07E00A9875
:1029E00028B98C48028831464046FFF79FFD4FEAE0
:1029F00049604FEA1069701C86B287484088B0422F
:102A000000DCCDE7A6EB0B00A0420AD15E4608F140
:102A100001001FFA80F880480088404500DCBFE7CD
:102A200006E00AF1010000F0FF0ABAF1080FCCDB62
:102A300000BF681CC5B20098854295DB00BFAFE7B8
:102A400010B50246012000E050430B1EA1F1010425
:102A5000E1B2F9D110BD2DE9FF4F81B00746914693
:102A60001E460E9D4FF0000A002439E0301B401E28
:102A7000C1B20A20FFF7E4FFB9FBF0F00A21B0FB76
:102A8000F1F201FB1208BAF1000F16D1701EA0423C
:102A900013DDB8F1000F0ED10020AB4605EBDB7162
:102AA000491001FB0471009088B22B462022029944
:102AB000FFF72EFF12E04FF0010A0020AB4605EBB6
:102AC000DB71491001FB0471009088B208F13001FC
:102AD000CAB22B460299FFF71BFF00BF601CC4B2AD
:102AE000B442C3DB05B0BDE8F08F2DE9FF4F83B0E2
:102AF000064692461F46DDE9104800200290002558
:102B00004DE0781B401EC1B20A20FFF799FFBAFBC7
:102B1000F0F00A21B0FBF1F201FB1209029850BB60
:102B2000781EA84227DDB9F1000F22D108F08000FD
:102B300078B108F00100A34604EBDB71491001FBFA
:102B40000561009088B2234630220499FFF7E0FE29
:102B50000EE008F00100A34604EBDB71491001FB15
:102B60000561009088B2234620220499FFF7D0FE29
:102B700013E00120029008F00100A34604EBDB7192
:102B8000491001FB0561009088B209F13001CAB219
:102B900023460499FFF7BCFE00BF681CC5B2BD42C6
:102BA000AFDB07B0BDE8F08F2DE9F84F04460D46C6
:102BB00090469946DDE90A6704F0FF0A08EB040035
:102BC0001FFA80F809EB05001FFA80F916E044456A
:102BD00002DB5446A81985B24D4500DB14E0002005
:102BE00000903A78334629462046FFF791FE30465A
:102BF00006EBD07104EB61018CB27F1C38787E2823
:102C000002DC38782028E2DA00BFBDE8F88F000047
:102C1000B8000020BA0000205C0400207FB5054603
:102C20000C460121480402F065FC0295ADF8044011
:102C30000020ADF80600ADF80C0001A9264803F00D
:102C400054FB01221146244803F0F0FF01212248E1
:102C500003F0D4FB19208DF8000002208DF801004C
:102C600001208DF802008DF80300684602F057F845
:102C70007FBD10B50021194A11605160632140F2F7
:102C8000E730FFF7CBFF10BD10B50121124803F06C
:102C9000E4FF01281AD1114802684068521C40F133
:102CA00000000E490A60486001200EF069FB0C48E4
:102CB0000068401C0A49086008460068B0F57A7F41
:102CC00004D3FDF7DBFF002005490860012102481D
:102CD00003F0D4FF10BD00000044014018000020A4
:102CE000C00000201CB500200190009002F0CCF93B
:102CF0009948006840F480309749086000BF9648C2
:102D0000006800F4003000900198401C0190009889
:102D100018B90198B0F5A04FF1D18F48006800F4C0
:102D2000003010B10120009001E0002000900098D8
:102D3000012846D188484030006840F080508649DC
:102D4000403108608548006840F44040834908608D
:102D500081480830006880490831086008460068EA
:102D600040F4004008600846006840F4A050086045
:102D70007B48091F0860081F006840F08070091F29
:102D8000086000BF7448006800F000700028F9D0A7
:102D900040F20570734908606F480830006820F001
:102DA00003006D49083108600846006840F00200E1
:102DB000086000BF68480830006800F00C00082870
:102DC000F8D11CBD2DE9F84304460D4616461F46B2
:102DD0004FF0000802F058F9012002F07EF902F0ED
:102DE000A1F98046B8F1010F35D15B484030006849
:102DF00040F080505849403108605848006840F41D
:102E0000404056490860002002F02AFA4FF4A050D2
:102E100002F030FA4FF4805002F036FA33462A4678
:102E200021464FF48000009702F0BFF9012002F024
:102E3000CCF900BF392002F057F90028FAD040F24F
:102E4000057048490860022002F0FAF900BF02F05C
:102E500001FA0828FBD1BDE8F8832DE9FC410446BE
:102E60000D4616461F460020019002F00DF9012084
:102E700002F07EF93848006800F0020001900198E5
:102E8000022834D134484030006840F08050324944
:102E9000403108603148006840F440402F490860E4
:102EA000002002F0DDF94FF4A05002F0E3F94FF4F6
:102EB000805002F0E9F933462A4621460020009767
:102EC00002F073F9012002F080F900BF392002F00E
:102ED0000BF90028FAD040F2057022490860022060
:102EE00002F0AEF900BF02F0B5F90828FBD1BDE849
:102EF000FC811CB50121084602F0A2FA4FF4807053
:102F0000009002208DF8040000208DF806000120BA
:102F10008DF8070003208DF805006946124801F07E
:102F2000EFFF1CBD1CB50121042002F089FA4FF40B
:102F30000070009002208DF8040000208DF806003B
:102F400001208DF8070003208DF805006946074829
:102F500001F0D6FF1CBD00000038024000700040A8
:102F600019544007003C02400000024000080240A3
:102F700070471CB50121022002F062FA4FF4805024
:102F8000009001208DF8040000208DF80600032039
:102F90008DF8050001208DF807006946324801F0E0
:102FA000AFFF4FF48051304802F028F81CBD1CB52B
:102FB0000121022002F044FA4FF480512A4802F025
:102FC0001BF84FF48050009000208DF80400012081
:102FD0008DF8060003208DF8050000208DF807000D
:102FE0006946214801F08CFF1CBD1CB5012102205F
:102FF00002F026FA4FF4C070009001208DF8040012
:1030000000208DF8060003208DF8050001208DF8C2
:1030100007006946154801F073FF00201449086055
:103020001449C1F8A0021CBD1CB50121022002F008
:1030300007FA01200E4908600E49C1F8A0024FF4BA
:10304000C070009000208DF8040001208DF806006B
:1030500003208DF8050000208DF80700694603481D
:1030600001F04EFF1CBD00000004024000080240B9
:103070009C024142000041422DE9F04104460F46C6
:1030800015461E4600BF00BF00BF02E0012016F03B
:10309000CDFFA0780028F9D10120A0702088C0F5CC
:1030A0000060A8420DDB2288E11C50182A463146F8
:1030B0001AF0F8FC2088284420800020A070BDE889
:1030C000F0810020A0700120F9E701B56B460122D4
:1030D00011468B48FFF7D0FF08BD00BF00BF00219D
:1030E00041F26D02024482F80D1441F26D02024475
:1030F00082F80C1441F26D020244A2F80E147047DB
:1031000010B57F481AF080FF10BD704700BF00BFA8
:10311000002181700180704700BF00BF642300F66A
:103120000302C2F866380023A2F8643859B10021BE
:1031300005E0002300F6030253544A1C91B240F606
:1031400064029142F5DB704730B587B005460C4606
:103150000121084602F074F90121102002F0CAF999
:1031600007220921674801F056FF07220A21654816
:1031700001F051FF4FF4C060059002208DF8180057
:103180008DF8190000208DF81A0001208DF81B0021
:1031900005A95C4801F0B4FE01940020ADF80800D8
:1031A000ADF80A00ADF80C00ADF810000C20ADF839
:1031B0000E0001A9544802F0FEFA0121524802F023
:1031C00082FB012240F225514F4802F032FC0122DD
:1031D00040F226614C4802F02CFC25208DF80000BE
:1031E00003208DF801008DF8020001208DF8030006
:1031F000684601F094FD00BF00BF20212846FFF77C
:103200008BFF2846FFF769FF2846FFF77FFF07B0CF
:1032100030BD70B505460C4620461AF0D3FB86B289
:103220002346324601212846FFF726FF70BD70B5C0
:10323000044600BF00BF208808B9002070BD02E02E
:10324000012016F0F3FEA0780028F9D10120A0702B
:1032500002E0012016F0EAFE41F26D00204490F8F1
:103260000D040028F5D12088B0F5806F01DC258899
:1032700001E04FF480652A46E11C41F26D002044D4
:103280001AF010FC2088421BE01C41191AF00AFCBD
:103290002088401B208041F26D002044A0F80E548D
:1032A00041F26D00211804F58050C0F87D1441F200
:1032B0006D002044B0F80E04401E41F26D0121441F
:1032C000A1F80E0404F58050D0F87D24D0F87D04D8
:1032D000401C04F58051C1F87D0410780A498880AB
:1032E0000020A070012041F26D01214481F80D04FD
:1032F0000020A3E700B50248FFF707FF00BD00006C
:103300006A0400200000024000100140002101700A
:10331000704770B58AB006460C461546012102205A
:1033200002F0D7F80121042002F08AF84FF400706F
:10333000089002208DF8240003208DF8250000203D
:103340008DF8260001208DF8270008A9344801F0E7
:10335000D7FD02220921324801F05DFEA8B2ADF886
:1033600014000020ADF816000694ADF81C0005A965
:103370002C4802F0BAFF6020ADF800000120ADF843
:1033800002000020ADF80C00600802906946254854
:1033900003F02CF90821234803F0E8F90121214822
:1033A00003F00EF801211F4803F028F80AB070BDA1
:1033B00070B504460D46002020701B48B0FBF5F6A2
:1033C000711E63222046FFF7A4FF70BD10B50446AE
:1033D000207801280DD113482030008840F4805017
:1033E000104920310880142016F020FE00202070A3
:1033F0000AE02078022807D00A482030008820F40C
:10340000805008492031088010BD012101707047AB
:1034100002210170704700B50448FFF777FF00BD37
:10342000000802400004004040420F00CE0000208F
:10343000704770B505460C4600BF02216E4803F088
:1034400009FF0028F9D021466B4803F0BAFE00BFFF
:103450000121694803F0FEFE0028F9D0664803F018
:10346000ADFEC0B270BD70B505460C46624800881E
:103470004FF6C7710840604908800846008820431D
:10348000088001215C4803F01BFE70BD10B588B0B8
:1034900004460121022001F0D3FF0121080302F0BC
:1034A00029F8C020069001208DF81C0000208DF81E
:1034B0001E0003208DF81D0001208DF81F0006A9B5
:1034C0004E4801F01DFD40214C4801F095FD802142
:1034D0004A4801F091FD3820069002208DF81C002A
:1034E00000208DF81E0003208DF81D0001208DF8AE
:1034F0001F0006A9414801F003FD052203213F48B2
:1035000001F089FD052204213C4801F084FD0522DB
:1035100011463A4801F07FFD0121080302F03FF80F
:1035200000214FF4805002F03AF80020ADF804007A
:103530004FF48270ADF806000020ADF808000220BC
:10354000ADF80A000120ADF80C004002ADF80E0005
:103550003820ADF810000020ADF812000720ADF8BB
:10356000140001A9244803F0B1FC10212448FFF7FE
:103570007AFF0121204803F0A3FDFF212046FFF739
:1035800058FF08B010BD70B505460C4600BF0221BB
:10359000194803F05FFE0028F9D02146164803F0D1
:1035A00010FE00BF0121144803F054FE0028F9D09A
:1035B000114803F003FEC0B270BD10B5044600BF51
:1035C00002210D4803F046FE0028F9D0FF210A48E9
:1035D00003F0F7FD00BF0121074803F03BFE002880
:1035E000F9D0054803F0EAFDC0B210BD00B50448AB
:1035F000FFF71EFF00BD0000003001400004024044
:10360000F318002000210DE0002207E000BF00BFFA
:1036100000BF00BF00BF00BF531CDAB2022AF5DBB7
:103620004B1C99B28142EFDB704770471CB50446D2
:103630000121022001F004FF44F208000090012063
:103640008DF8040000208DF8060001208DF8070099
:1036500002208DF805006946944801F051FC1020C5
:10366000009000208DF804008DF8070069468F480F
:1036700001F046FC1CBD70B5054602E0012016F0C5
:10368000D5FC8B4800780128F8D0012088490870C3
:103690004021864801F0B2FC8021844801F0ACFC56
:1036A00000BF00BF05218348FFF76DFF8148FFF78A
:1036B00084FF044640217D4801F09EFC00BF00BF0E
:1036C00000207B490870204670BD70B505460C4649
:1036D0004021764801F092FC8021744801F08CFC76
:1036E00000BF00BF01217348FFF74DFF214671481D
:1036F000FFF749FF40216D4801F07EFC00BF00BF8D
:1037000070BD2DE9F84380460E4617461C4602E080
:10371000012016F08BFC664800780128F8D00120C3
:103720006349087000964021604801F067FC8021E1
:103730005E4801F061FC00BF00BF03215D48FFF758
:1037400022FF9DF801105B48FFF71DFF9DF8001058
:103750005848FFF718FF002506E05648FFF72DFFF1
:103760002070641C681C85B2BD42F6DB40214F48C6
:1037700001F042FC00BF00BF00204D490870BDE8C9
:10378000F8832DE9F84380460E4617461C4602E0B2
:10379000012016F04BFC464800780128F8D00120A3
:1037A0004349087000964021404801F027FC8021E1
:1037B0003E4801F021FC00BF00BF06213D48FFF755
:1037C000E2FE4021394801F017FC00BF00BF012094
:1037D000FFF718FF4021354801F010FC80213348E5
:1037E00001F00AFC00BF00BF02213248FFF7CBFE08
:1037F0009DF801102F48FFF7C6FE9DF800102D48D8
:10380000FFF7C1FE002506E021782A48FFF7BBFE3E
:10381000641C681C85B2BD42F6DB4021234801F0E0
:10382000EBFB00BF00BF0120FFF7ECFE40211F486B
:1038300001F0E4FB80211D4801F0DEFB00BF00BF6A
:1038400004211C48FFF79FFE4021184801F0D4FBDB
:1038500000BF00BF022016F0E9FB002014490870E9
:10386000BDE8F88338B505460C4600BF00BF6B467F
:10387000022221461048FFF744FF00BF00BFBDF8F9
:10388000000038BDF8B506460D46144600946B4658
:10389000022229460848FFF774FF00BF00BFF8BDA9
:1038A00000B50548FFF7C1FE00BD0000000402405E
:1038B000CF000020F3180020F41800207047704754
:1038C00070B505460C468021FC4801F097FB40216D
:1038D000FA4801F091FB00BF00BF9F21F848FFF7B5
:1038E00052FEF748FFF769FE2070641CF448FFF7AA
:1038F00064FE2070641CF248FFF75FFE2070641CB9
:103900008021EE4801F078FB00BF00BF70BD30B5EC
:1039100089B004460D4601A92046FFF7D1FF9DF866
:1039200006008DF808009DF805008DF809009DF847
:1039300004008DF80A0000208DF80B00E149029880
:103940000861E1A1E548FFF764FCDE4800690590E5
:1039500005AB04220121E148FFF78EFBE0A1DF481F
:10396000FFF757FC002009B030BD70B5054602E0F6
:10397000012016F05BFBDB4800780128F8D001201D
:10398000D84908708021CD4801F038FB4021CB4850
:1039900001F032FB00BF00BF0521C948FFF7F3FD6E
:1039A000C748FFF70AFE04468021C44801F024FB03
:1039B00000BF00BF0020CB490870204670BD70B525
:1039C00005460C468021BD4801F018FB4021BB484C
:1039D00001F012FB00BF00BF0121B948FFF7D3FD82
:1039E0002146B748FFF7CFFD8021B44801F004FB22
:1039F00000BF00BF70BD38B505460C4602E001208F
:103A000016F014FBB74800780128F8D00120B5491A
:103A100008708021A94801F0F1FA4021A74801F07F
:103A2000EBFA00BF00BF0621A548FFF7ACFD8021DF
:103A3000A24801F0E1FA00BF00BF0121AA48FDF74A
:103A40006FF880219D4801F0D9FA40219B4801F090
:103A5000D3FA00BF00BF2003009020219848FFF751
:103A600092FD9DF802109648FFF78DFD9DF801101C
:103A70009348FFF788FD9DF800109148FFF783FDFC
:103A800080218E4801F0B8FA00BF00BF00209549A0
:103A9000087038BD38B505460C4602E0012016F026
:103AA000C5FA904800780128F8D001208D490870A7
:103AB0008021824801F0A2FA4021804801F09CFA5E
:103AC00000BF00BF06217E48FFF75DFD80217B48D7
:103AD00001F092FA00BF00BF01218348FDF720F8F2
:103AE0008021764801F08AFA4021744801F084FA76
:103AF00000BF00BF20040090D8217148FFF743FDAC
:103B00009DF802106E48FFF73EFD9DF801106C48CD
:103B1000FFF739FD9DF800106948FFF734FD80215B
:103B2000664801F069FA00BF00BF00206D490870C7
:103B300038BD10B5044602E0012016F077FA694856
:103B400000780128F8D001206649087080215B4880
:103B500001F054FA4021594801F04EFA00BF00BF6D
:103B600006215748FFF70FFD8021544801F044FA21
:103B700000BF00BF01215C48FCF7D2FF80214F4805
:103B800001F03CFA40214D4801F036FA00BF00BF79
:103B9000C7214B48FFF7F7FC8021484801F02CFA79
:103BA00000BF00BF00204F49087010BDF8B50746A0
:103BB0000E46144602E0012016F038FA4948007813
:103BC0000128F8D0012047490870009680213B4821
:103BD00001F014FA4021394801F00EFA00BF00BF8D
:103BE00003213748FFF7CFFC9DF801103448FFF759
:103BF000CAFC9DF800103248FFF7C5FC0021304890
:103C0000FFF7C1FC002506E02D48FFF7D6FC04F8BD
:103C1000010B681C85B2FF2DF6D98021274801F0E1
:103C2000EBF900BF00BF00202E490870F8BDF8B5C1
:103C300007460E46144602E0012016F0F7F929481F
:103C400000780128F8D001202649087080211B48FF
:103C500001F0D4F94021194801F0CEF900BF00BFAE
:103C600006211748FFF78FFC8021144801F0C4F9A2
:103C700000BF00BF01211C48FCF752FF00968021C5
:103C80000E4801F0BBF940210C4801F0B5F900BF26
:103C900000BF02210A48FFF776FC9DF80110084892
:103CA000FFF771FC9DF800100548FFF76CFC002140
:103CB0000348FFF768FC002524E0000000040240F0
:103CC000F3180020F8180020466C617368205465D2
:103CD000737420446174613A000000006A0400209B
:103CE0000D0A0000CF000020B00000202178C1485C
:103CF000FFF749FC641C2178BE48FFF744FC641CB4
:103D0000681C85B2802DF1D38021BB4801F074F985
:103D100000BF00BF0020B9490870F8BD10B50446C7
:103D2000B921B448FFF72FFC10BD10B5044680211F
:103D3000B14801F063F94021AF4801F05DF900BFDF
:103D400000BFAB21AB48FFF71EFC8021AA4801F061
:103D500053F900BF00BF10BD70B506460C460025E4
:103D60000DE0A748FFF701FE00F0010018B10120A7
:103D700016F05CF901E0002070BD681C85B2A54218
:103D8000EFDB0120F8E72DE9F04107460D46164626
:103D900000240EE04FF4FA713846FFF7DDFF2919D1
:103DA0003846FFF777FEC8213846FFF7D5FF601C7D
:103DB00084B2B442EEDB0020BDE8F0812DE9F05F73
:103DC00004468946154602E0012016F02FF92078B6
:103DD0000028F9D1012020700DB10A2D00DD032546
:103DE0004FF0000835E064212046FFF7B5FF494653
:103DF0002046FFF700FE64212046FFF7ADFF4FF09D
:103E0000000A4FEA091B002617E00BEB0601621CB3
:103E10002046FFF7CBFE002707E0601CC05DFF28AF
:103E200002D04FF0010A02E07F1CFF2FF5D900BF3E
:103E3000BAF1010F00D102E0761C102EE5D300BFCD
:103E4000BAF1000F03D100202070BDE8F09F08F107
:103E50000108A845C7D3002020700120F5E72DE90F
:103E6000FF5F04460E461F4602E0012016F0DEF812
:103E700020780028F9D1012020700FB10A2F00DD31
:103E8000032731462046029AFFF7D1FE0A21204639
:103E9000FFF762FF621C31462046FFF787FE4FF4B2
:103EA0008072611C029819F03DFD00287ED055A15A
:103EB0005948FFF7AEF94FEA1618A6EB081000F1C3
:103EC000010B4FEA081955A15348FFF7A2F9002248
:103ED0004FF48051584814F043F8002508E0564844
:103EE00000EB052209EB05012046FFF75FFE6D1C84
:103EF0005D45F4D34FF0000A64E050A14648FFF757
:103F000088F90020207031090A223D48FFF756FF4A
:103F1000002853D1012020704CA13F48FFF779F9C8
:103F2000002520E0444800EB052209EB050120466E
:103F3000FFF77DFE0A212046FFF70EFF09EB050182
:103F4000621C2046FFF732FE3B4901EB05204FF48F
:103F50008072611C19F0E6FC20B146A12E48FFF7E3
:103F600058F902E06D1C5D45DCD300BF4AA12A4828
:103F7000FFF74FF931462046029AFFF758FE0A2113
:103F80002046FFF7E9FE621C31462046FFF70EFE91
:103F90004FF48072611C029819F0C4FC50B944A11E
:103FA0001D48FFF736F90020207000E00DE004B056
:103FB000BDE8F09F44A11848FFF72BF901202070BD
:103FC0000AF1010ABA4598D307E00020207039A110
:103FD0001148FFF71EF90020E7E70020207040A1FC
:103FE0000D48FFF716F90120DFE700B50448FFF799
:103FF00065FC00BDF318002000040240CF00002043
:10400000121A0020666C61736820C3BBB1A3B4E6CA
:10401000D5FDC8B70D0A00006A040020B0D1B5B1C3
:10402000C7B0C9C8C7F8CAFDBEDDD4DDB4E6D4DA6E
:10403000C4DAB4E60D0A0000171B0020B2C1B3FDBC
:10404000B5B1C7B0C9C8C7F80D0A0000CAB9D3C313
:10405000D2D1B1A3B4E6B5C4C4DAB4E6CAFDBEDDBC
:10406000D6D8D0C2D0B4B5B1C7B0C9C8C7F80D0A48
:1040700000000000BBD8D0B4D4F8BEADB1A3B4E604
:10408000D4DAB5B1C7B0C9C8C7F8CAFDBEDDD3D050
:10409000CEF30D0A00000000D0B4B5B1C7B0D2B362
:1040A000D2AAB1A3B4E6B5C4CAFDBEDD0D0A0000B4
:1040B000D6D8D0C2B1A3B4E6464C415348CAFDBEDF
:1040C000DDD5FDC8B70D0A00D6D8D0C2B1A3B4E67D
:1040D000464C415348CAFDBEDDB4EDCEF30D0A0097
:1040E000666C617368207772697465206572726F9F
:1040F000720D0A0070472DE9F04180460D46A04838
:1041000001F045FE074602219D4801F02EFF002DDB
:1041100002DD681E84B200E003244FF6FF7000EA5F
:10412000043404F47044C7F30B0727439548465DF5
:10413000122E02D1012001F070FD07230122314629
:104140008F4801F08CFD8E4801F0E5FD3846BDE852
:10415000F08110B58CB004460121042001F070F903
:104160000121080201F0C6F907200A9003208DF80A
:104170002C0000208DF82F000AA9834800F0C0FE13
:104180000121080201F00BFA00214FF4807001F0C8
:1041900006FA00200690099008904FF480300790AE
:1041A00006A801F005FD002000908DF804008DF8B0
:1041B00005000290049001208DF8140069467048B3
:1041C00001F0C7FC6E48806820F410606C4988607C
:1041D000012001F022FD0121694801F000FD0120CC
:1041E00014F02FFA00212046FFF785FF012014F07C
:1041F00028FA00212046FFF77EFF012084F83E00C8
:10420000002020870CB010BD2DE9F047044600BF08
:1042100000BF54F83A0F401C206021793A3C2046F8
:10422000FFF769FF804647463F13C8F30B0807EBCB
:10423000870004EB4000218F20F811804FF0000A26
:1042400000260AE007EB870004EB400030F81A0074
:1042500006440AF1010000F0FF0ABAF1050FF1DB94
:104260000520B6FBF0F081B204F1280020F8171009
:1042700030F8176041F67970464342F21070B6FB91
:10428000F0F604F1300020F81760B5B237B1012F15
:104290002ED0022F2DD0032F45D135E040F2FA4623
:1042A0006E434FF47A70B6FBF0F085B2B5F57A6FD5
:1042B00003DB04203549088019E040F6D8608542C8
:1042C00003DB03203149088011E0B5F5616F03DBA2
:1042D00002202E4908800AE040F64850854203DB60
:1042E00001202A49088002E00020284908801BE0BC
:1042F0001AE0A08D14F0BCF9254908800846008812
:10430000C01F00B208800FE0A94609EB89004FEA00
:104310004009A9F58059A9F55B69192099FBF0F9C5
:1043200009F1190900E000BF00BF00BF00BF00BFD6
:1043300000BF94F83E00401CC0B284F83E00032841
:104340000ADB002084F83E00208F401C2087208F4D
:10435000052801DB00202087BDE8F0870246002009
:1043600006E002F1300333F8103021F81030401C21
:104370000428F6D3704700B50648FFF7BBFE00BD22
:1043800000200140D0000020000802403C00002036
:104390003A000020182B002000BF00BF7047704774
:1043A0007047F0B50546002092F903400A2694FBB9
:1043B000F6F430341C54401C92F9034094FBF6F799
:1043C00006FB174430341C54401C19B13A241C54C9
:1043D000441CE0B292F904400A2694FBF6F430340F
:1043E0001C54441CE0B292F9044094FBF6F706FB1F
:1043F000174430341C54441CE0B219B13A241C5404
:10440000441CE0B292F905400A2694FBF6F43034DD
:104410001C54441CE0B292F9054094FBF6F706FBED
:10442000174430341C54441CE0B2F0BD70B5034650
:10443000002093F907400A2594FBF5F43034145416
:10444000401C93F9074094FBF5F605FB1644303405
:104450001454401C19B13A241454441CE0B293F98A
:1044600008400A2594FBF5F430341454441CE0B29F
:1044700093F9084094FBF5F605FB164430341454C8
:10448000441CE0B219B13A241454441CE0B293F92C
:1044900009400A2594FBF5F430341454441CE0B26E
:1044A00093F9094094FBF5F605FB16443034145497
:1044B000441CE0B270BD10B50246002091F90030F6
:1044C000002B03DB91F90030632B00DD012091F913
:1044D0000130012B03DB91F901300C2B00DD0220B0
:1044E00091F90230012B03DB91F902301F2B00DD23
:1044F000032091F90330002B03DB91F90330172BD4
:1045000000DD042091F90430002B03DB91F9043025
:104510003B2B00DD052091F90530002B03DB91F9E1
:1045200005303B2B00DD0620B1F90630B3F5FA6FFC
:1045300005DBB1F9063040F63404A34200DD072064
:1045400010BD70472DE9F04F8046FE48814202D9E8
:104550000120BDE8F08F002500230DE0FA4EFB4856
:10456000405D08B1FA480644B14200D206E0581C4A
:1045700003B2891B681CC5B2642DEFDB00BF58B2C3
:10458000107003F5FA6000B2D080F04810F803C054
:104590000025012411E0EF484657ED484643BCF1A1
:1045A000000F02D0022C00D10644B14200D206E036
:1045B000601CC4B2891B681CC5B20C2DEBDB00BFAC
:1045C00060B25070E248B1FBF0F040B29070907869
:1045D000401C40B29070DE48B1FBF0F900FB1911AD
:1045E0004FF46160B1FBF0F040B2D0704FF4616005
:1045F000B1FBF0F900FB19113C20B1FBF0F040B227
:1046000010713C20B1FBF0F900FB191040B2507161
:10461000B2F9063054789778012C01D0022C04D1DD
:1046200004F10C00C4B2581E03B204F1010909EBF5
:1046300049094FF0050A99FBFAF94FF0020A0AFB03
:10464000047AD144994418464FEAE37A03EB9A7A04
:1046500009EBAA094FF0640A93FBFAFAA9EB0A09DD
:104660004FF4C87A93FBFAFAD14409F101094FF0EB
:10467000070A99FBFAFB0AFB1B994FFA89F982F8A2
:104680000A90002065E770B504460E4600BF00BFE3
:10469000251D2A4631462046FFF754FF294620466D
:1046A000FFF74FFF00BF00BF70BD02790A7042796B
:1046B0004A7082798A70C279CA70027A0A71427A23
:1046C0004A714289CA8082890A81827B8A727047D4
:1046D000704770B504460D46207913F068F940B272
:1046E0002870607913F063F940B26870A07913F014
:1046F0005EF940B2A870E07913F059F940B2E87061
:10470000207A13F054F940B22871607A13F04FF90F
:1047100040B26871A07B13F04AF940B2A87270BD34
:104720002DE9F04F83460C4600BF00BFB4F90600E8
:10473000B0F5FA6F07DA94F90000E080E08800F540
:10474000FA6000B2E08021465846FFF7B4FE054605
:1047500015B10020BDE8F08FB4F90680A8F5FA6025
:104760000FFA80F80025002708E0774807447748CB
:10477000405D08B176480744681CC5B24545F4DB86
:10478000724810F808A094F90100401E724931F9EE
:10479000106094F902000644761EBAF1000F04D0AE
:1047A00094F90100022800DD761C94F903004FF40F
:1047B000616110FB01F094F90410C1EB011100EBF1
:1047C000810094F9051000EB0109B94440F2A320DF
:1047D000704309EBC0194846BCE730B50446251DB7
:1047E00029462046FFF79CFF30BD2DE9F0470446DF
:1047F0000E4691463146022013F019FB8046B8F16F
:10480000000F01D1182000E040464FF4616100FB29
:1048100001F5B11C022013F00AFB8046C8EB08101A
:1048200005EB8005311D022013F001FB8046454455
:10483000E07908B9182001E094F907004FF46161AC
:10484000484394F90810C1EB011100EB810194F980
:1048500009000F18E81B002802DC781B484502D22B
:104860000120BDE8F0870020FBE7C2790A70027AD8
:104870004A70427A8A7070472DE9F04180460F46AF
:1048800016461D460424F18888B2294613F06CFAB6
:104890001FB12D202855601CC4B296F901000A21D1
:1048A00090FBF1F030302855601CC4B296F901003D
:1048B00090FBF1F201FB120030302855601CC4B2AD
:1048C0001FB12D202855601CC4B296F902000A21A0
:1048D00090FBF1F030302855601CC4B296F902000C
:1048E00090FBF1F201FB120030302855601CC4B27D
:1048F0001FB120202855601CC4B22B1932463946FE
:104900004046FFF74EFDBDE8F08114490968491C97
:10491000124A1160704770B506460C464FF4FA65AE
:10492000207813F05BF80544E580207813F056F802
:1049300040B22070607813F051F840B26070E078B7
:104940000EE00000801319BC8033E101A0080208CA
:104950008051010094080208040902084C0000205C
:1049600013F03CF840B2E070A07813F037F840B292
:10497000A070207913F032F840B22071607913F002
:104980002DF840B2607121463046FFF7C9FE70BD78
:104990007FB505460E46144610222146684619F09A
:1049A0003CF86A4631462846FFF7CCFD9DF80000EA
:1049B00012F0FDFF40B220709DF8010012F0F7FFE9
:1049C00040B260709DF8020012F0F1FF40B2A0709A
:1049D0009DF8030012F0EBFF40B2E0709DF8040078
:1049E00012F0E5FF40B220719DF8050012F0DFFFE4
:1049F00040B260719DF80A0012F0D9FF40B2A07277
:104A00007FBD2DE9FF4780460C461546E01D13F09B
:104A100061FB00B2ADF80600BDF90600642190FB11
:104A2000F1F201FB120040B28DF800005CA12046BB
:104A300019F056FB18B101208DF801006EE058A165
:104A4000204619F04DFB18B101208DF8010065E0FA
:104A500054A1204619F044FB18B102208DF8010042
:104A60005CE051A1204619F03BFB18B103208DF802
:104A7000010053E04DA1204619F032FB18B104208B
:104A80008DF801004AE04AA1204619F029FB18B12F
:104A900005208DF8010041E046A1204619F020FBD9
:104AA00018B106208DF8010038E043A1204619F026
:104AB00017FB18B107208DF801002FE03FA1204619
:104AC00019F00EFB18B108208DF8010026E03CA17A
:104AD000204619F005FB18B109208DF801001DE0F2
:104AE00038A1204619F0FCFA18B10A208DF801000F
:104AF00014E035A1204619F0F3FA18B10C208DF816
:104B000001000BE031A1204619F0EAFA18B10C209F
:104B10008DF8010002E00C208DF8010026796779FC
:104B2000A7F1300040B28DF80200312E06D19DF879
:104B300002000A3040B28DF8020010E0322E06D199
:104B40009DF80200143040B28DF8020007E0332EC9
:104B500005D19DF802001E3040B28DF802002846B3
:104B600013F0B8FA40B28DF80300E81C13F0B2FA63
:104B700040B28DF80400A81D13F0ACFA40B28DF8D5
:104B8000050069464046FFF7CBFD8146484604B024
:104B9000BDE8F08700B50E48FFF701FC00BD00003E
:104BA0004A616E00466562004D617200417072009C
:104BB0004D6179004A756E004A756C004175670059
:104BC000536570004F6374004E6F76004465630058
:104BD000582B002010B515F088FF012801D016F0E1
:104BE00019FF10BD70B50446042000F0E5F8324806
:104BF000047025464FF47A70454301202F49088000
:104C00004FF0E020006940F002004FF0E021086121
:104C100008464561006940F00100086170BD70B54B
:104C2000034600224FF0E0267569234E367803FBD9
:104C300006F44FF0E026B16910E04FF0E026B069CD
:104C400088420BD0884202D20E1A324402E02E1A59
:104C50000E4432440146A24200D300E0EDE700BF1B
:104C600070BD70B5044615F040FF012810D0134800
:104C70000088844206D311480088B4FBF0F528462A
:104C800015F0D4F90D480088B4FBF0F100FB114495
:104C90004FF47A7104FB01F0FFF7C1FF70BD30B52E
:104CA0000446002504E04FF47A70FFF7B8FF6D1C4E
:104CB000A542F8D330BD0000D4000020D60000206B
:104CC00000BF704770B504460D46E0B2FEF7FDF92F
:104CD000204670BD0948804709480047FEE7FEE7C7
:104CE000FEE7FEE7FEE7FEE7FEE7FEE7FEE7FEE79C
:104CF00004480549054A064B70470000DF030008D9
:104D000089010008F8430320F84D0320F8450320EB
:104D1000F845032032490143324A1160704770B5AB
:104D2000002100230F22C4781CB32E4C246804F405
:104D3000E064C4F5E064C4F30721C1F10404E3B204
:104D40000A4144789C40E1B28478144021430C0726
:104D5000210E254C05786155047804F01F050124C7
:104D6000AC4005786D11AD0005F1E025C5F80041B6
:104D700009E0047804F01F050124AC401B4D0678BF
:104D8000761145F8264070BD194A0A400243154B7A
:104D90001B1F1A60704739B1124A121D1268024374
:104DA000104B1B1D1A6006E00E4A121D126882434A
:104DB0000C4B1B1D1A607047042808D14FF0E021EE
:104DC000096941F004014FF0E022116107E04FF062
:104DD000E021096921F004014FF0E02211617047E0
:104DE0000000FA050CED00E000E400E080E100E0E6
:104DF00080FFFF1F10B504469848844208D1012166
:104E0000084600F088FB0021012000F084FB76E0DA
:104E10009348844208D10121022000F07CFB00214C
:104E2000022000F078FB6AE08E48844208D101211C
:104E3000042000F070FB0021042000F06CFB5EE019
:104E40008948844208D10121082000F064FB002138
:104E5000082000F060FB52E08448844208D1012120
:104E6000102000F058FB0021102000F054FB46E019
:104E70007F48844208D10121202000F04CFB002112
:104E8000202000F048FB3AE07A48844208D1012112
:104E9000402000F040FB0021402000F03CFB2EE0D1
:104EA0007548844208D10121802000F034FB0021A4
:104EB000802000F030FB22E07048844208D10121BC
:104EC000801500F028FB0021A01500F024FB16E05F
:104ED0006B48844208D10121401500F01CFB0021E1
:104EE000601500F018FB0AE06648844207D10121F2
:104EF000001500F010FB0021201500F00CFB10BD88
:104F0000F0B50A4600210023002400BF3DE0012542
:104F100005FA01F3156805EA03049C4234D10568DB
:104F20004F000326BE40B543056015794E00B540DD
:104F30000668354305601579012D02D01579022DDB
:104F400016D185684F000326BE40B543856055796C
:104F50004E00B540866835438560456801268E4021
:104F6000B5434560456896798E40B6B23543456095
:104F7000C5684F000326BE40B543C560D5794E00D5
:104F8000B540C6683543C560491C1029BFD3F0BD84
:104F90004FF6FF7101600021017141718171C17192
:104FA000704708B54FF480320092009A0A4300928D
:104FB000009AC261C161009AC261C2690092C2696D
:104FC000009208BD0246002013690B400BB101207E
:104FD00000E0002070470146086980B27047024631
:104FE000002053690B400BB1012000E00020704706
:104FF0000146486980B2704701837047418370471A
:105000000AB1018300E04183704741617047426902
:105010004A4042617047F0B5002300244D07ED0E71
:1050200002FA05F3CE1000F1200555F826504E0780
:10503000F70E0F26BE40B543CF1000F1200646F80C
:105040002750CE1000F1200555F8265045EA0304FC
:10505000CE1000F1200545F82640F0BD00000240CA
:105060000004024000080240000C02400010024010
:105070000014024000180240001C024000200240C0
:105080000024024000280240FA48006840F0010075
:10509000F84908600020F74908310860F5480068C1
:1050A000F5490840F3490860F448091D0860F448D0
:1050B000F04984310860F1481038091D0860ED4856
:1050C000006820F48020EB4908600020E9490C3199
:1050D0000860E8498C31086070470021E54A921C5D
:1050E000117011460870704710B501460022002368
:1050F00000204A11012A02D1DE4C236808E0022A6E
:1051000003D1DC4C7034236802E0DA4C7434236839
:1051100001F01F02012494401C400CB1012000E06A
:10512000002010BD38B5002000900024002500BFED
:105130003120FFF7D9FF05460098401C00900098E9
:10514000B0F5A04F01D0002DF2D03120FFF7CCFFF9
:1051500008B1012400E00024204638BD01460020AB
:10516000C44A106820F0F80040EAC100106070479F
:10517000C449086070470021BE4A70321170117036
:10518000012802D004280AD104E00121B94A703272
:10519000117005E00521B74A7032117000E000BFC0
:1051A00000BF7047B8490860704770B5049C41EA79
:1051B00082150126C6EB530645EA0645054345EA36
:1051C0000465AC4E361D356070BDAE49086670474B
:1051D00010B5830143EA01731343A64C8434236062
:1051E00010BDA8498866704710B5830143EA016382
:1051F00043EA02739F4C8834236010BDA1490867BD
:105200007047A049C864704702460020994B083394
:10521000186820F0EC6042EA01031843954B08330C
:105220001860704702460020924B0833186820F03F
:10523000784042EA010318438E4B083318607047E8
:10524000014600208B4A0832106820F00300084312
:105250001060704787480830006800F00C00704705
:1052600001460020834A0832106820F0F00008430D
:1052700010607047014600207E4A0832106820F412
:10528000E05008431060704701460020794A083218
:10529000106820F4604040EAC10010607047F0B52B
:1052A000002100220024022500260223714F083726
:1052B0003F6807F00C0121B1042905D0082937D136
:1052C00005E0724F076036E0714F076033E0694FC9
:1052D0003F1D3F68C7F38056664F3F1D3F6807F08C
:1052E0003F036EB16A4FB7FBF3F7DFF888C10CF1EB
:1052F000040CDCF800C0CCF3881C07FB0CF40CE0B9
:10530000624FB7FBF3F7DFF86CC10CF1040CDCF86B
:1053100000C0CCF3881C07FB0CF4564F3F1D3F68C0
:10532000C7F301477F1C7D00B4FBF5F7076002E07F
:10533000564F076000BF00BF4E4F08373F6807F069
:10534000F0010909534F7A5C0768D7404760494F1D
:1053500008373F6807F4E051890A4E4F7A5C476886
:10536000D7408760434F08373F6807F46041490BD7
:10537000484F7A5C4768D740C760F0BD002100F411
:105380004072B2F5407F0AD13A4A0832116821F4DE
:10539000F811414A02401143364A08321160354A39
:1053A00070321268C0F30B031A43324B70331A6029
:1053B00070473549443908607047334940390860BF
:1053C000704736490860704701460020294A8C32F0
:1053D000106820F01F004A1E1043264A8C321060CD
:1053E000704701460020234A8C32106820F4F850A0
:1053F0004A1E40EA02201F4A8C3210607047014664
:1054000000201C4A8C32106820F4401008431060C1
:10541000704701460020174A8C32106820F4400083
:1054200008431060704701460020124A8C32106811
:1054300020F44030084310607047194908607047F5
:1054400039B10C4A3032126802430A4B30331A60C9
:1054500006E0084A303212688243064B30331A6045
:105460007047F9B1034A343212680243014B3433B6
:105470001A601CE000380240FFFFF6EA10300024FA
:105480000030002000004742800E47420024F40014
:1054900000127A00DC000020FFFCFF0F5C01474295
:1054A000E01147428F4A126882438E4B1A60704760
:1054B00039B18C4A121D126802438A4B1B1D1A60B7
:1054C00006E0884A121D12688243864B1B1D1A6033
:1054D000704739B1834A0C3212680243814B0C3356
:1054E0001A6006E07F4A0C32126882437D4B0C330F
:1054F0001A60704739B17B4A103212680243794B07
:1055000010331A6006E0774A103212688243754BF6
:1055100010331A60704739B1724A243A1268024354
:10552000704B243B1A6006E06E4A243A12688243AC
:105530006C4B243B1A60704739B16A4A203A1268B2
:105540000243684B203B1A6006E0664A203A126824
:105550008243644B203B1A60704739B1614A1C3A60
:10556000126802435F4B1C3B1A6006E05D4A1C3A1E
:10557000126882435B4B1C3B1A60704739B1594A31
:10558000143A12680243574B143B1A6006E0554A1E
:10559000143A12688243534B143B1A60704739B176
:1055A000504A103A126802434E4B103B1A6006E014
:1055B0004C4A103A126882434A4B103B1A607047BB
:1055C00039B1484A1C3212680243464B1C331A60F8
:1055D00006E0444A1C3212688243424B1C331A6074
:1055E000704739B13F4A2032126802433D4B2033A5
:1055F0001A6006E03B4A203212688243394B20335E
:105600001A60704739B1374A243212680243354B69
:1056100024331A6006E0334A243212688243314B45
:1056200024331A60704739B12E4A2C321268024373
:105630002C4B2C331A6006E02A4A2C321268824323
:10564000284B2C331A60704739B1264A3032126821
:105650000243244B30331A6006E0224A303212688B
:105660008243204B30331A607047012808D11D490E
:105670003C31096841F008011A4A3C32116007E0E8
:1056800018493C31096821F00801164A3C32116082
:10569000704739B1134A273A12780243114B273B1E
:1056A0001A7006E00F4A273A127882430D4B273BC7
:1056B0001A7070470B484030006840F0807009490C
:1056C00040310860704701460020064A283A1268B7
:1056D0000A400AB1012000E0002070470149263944
:1056E000087070473438024010B50446FA488442C6
:1056F00008D101211020FFF752FF00211020FFF7F1
:105700004EFF57E0F548844209D101214804FFF7D4
:1057100035FF00214FF40030FFF730FF4AE0F0483A
:10572000844209D101218804FFF728FF00214FF4AA
:105730008020FFF723FF3DE0EA48844209D10121A0
:10574000C804FFF71BFF00214FF40020FFF716FFEE
:1057500030E0E548844209D101210805FFF70EFF3A
:1057600000214FF48010FFF709FF23E0DF48844257
:1057700008D101212020FFF712FF00212020FFF790
:105780000EFF17E0DA48844209D101218807FFF7AC
:10579000F5FE00214FF08040FFF7F0FE0AE0D5480B
:1057A000844207D101214005FFF7E8FE0021600592
:1057B000FFF7E4FE10BD2DE9FF4705460E46002425
:1057C000A14600BFA046B08900B100BF2C8A24F4D6
:1057D0004054F08804432C82AC8941F20C6084432D
:1057E000B08831890843718908430443AC81AC8A8D
:1057F00024F44074B0890443AC826846FFF74FFD3F
:10580000B548854202D0B948854202D1DDF80C90F6
:1058100001E0DDF80890A88900F4004040B109EBF0
:10582000C90000EB091031684900B0FBF1F707E04F
:1058300009EBC90000EB091031688900B0FBF1F7F2
:105840006420B7FBF0F004012009642101FB10780B
:10585000A88900F4004040B1322000EBC800B0FB42
:10586000F1F000F00700044308E0322000EB0810DC
:105870006421B0FBF1F000F00F0004432C81BDE87F
:10588000FF874FF41651016000218180C1800181A2
:105890000C21418100218181704710B50246002012
:1058A000108A20F470600B884C8823438C88234333
:1058B000CC8823431843108210BD00210180418011
:1058C0008180C180704721B1828942F40052828177
:1058D00004E082894DF6FF731A4082817047028B83
:1058E00002F47F420283028B0A430283704721B194
:1058F000828942F40042828103E08289C2F30E026F
:105900008281704721B1828A42F40062828204E07F
:10591000828A4FF2FF731A4082827047C1F30802F5
:105920008280704701468888C0F308007047028A69
:105930004FF6F0731A400282028A0A4302827047CD
:1059400021B1828942F00202828104E082894FF60D
:10595000FD731A408281704782894FF2FF731A40AB
:10596000828182890A4382817047028A4FF6DF73FF
:105970001A400282028A0A430282704721B1028AD7
:1059800042F48042028204E0028A4BF6FF731A401E
:1059900002827047818941F001018181704721B104
:1059A000828A42F00802828204E0828A4FF6F7730C
:1059B0001A4082827047028BD2B20283028B42EA83
:1059C00001220283704721B1828A42F02002828242
:1059D00004E0828A4FF6DF731A408282704721B159
:1059E000828A42F01002828204E0828A4FF6EF73CC
:1059F0001A4082827047828A4FF6FB731A40828275
:105A0000828A0A438282704721B1828A42F002026E
:105A1000828204E0828A4FF6FD731A4082827047C8
:105A20001AB1838A0B43838202E0838A8B43838289
:105A30007047F0B50346002400260025002040F6FC
:105A40006A17B94200D100BF1846C1F3421401F0F1
:105A50001F06012707FA06F5012C01D10C3004E0DE
:105A6000022C01D1103000E014301AB107682F4326
:105A7000076002E00768AF430760F0BD0246002000
:105A8000B1F5007F00D100BF13880B400BB101209E
:105A900000E00020704701F40072B2F5007F00D1F1
:105AA00000BFCA430280704770B50246002400233D
:105AB0000025002040F66A16B14200D100BFC1F3B4
:105AC000421501F01F03012606FA03F3012D13D13D
:105AD0009689334017E00000001001400044004068
:105AE00000480040004C00400050004000140140BD
:105AF00000780040007C0040022D02D1168A33401D
:105B000001E0968A33400C12012606FA04F4168846
:105B1000344013B10CB1012000E0002070BD10B57D
:105B20000022002340F66A14A14200D100BF0A12ED
:105B300001249440A3B2DC43048010BD10B50121C0
:105B40000802FFF72CFD00214FF48070FFF727FDBE
:105B500010BD30B50246002000235068F84C2040AC
:105B60000D790C6844EA0524204350609068F54C98
:105B70002040D1E903542C438D682C434D7944EAED
:105B8000450420439060D06A20F470000C7D641EB0
:105B9000E4B2234340EA0350D06230BD00210160EB
:105BA000017141718160C16001610121017570471E
:105BB0000021E54A1168E54A1140D0E900231A4363
:105BC00083681A43C3681A431143E14AC2F80413B5
:105BD00070470021016041608160C160704721B160
:105BE000826842F00102826003E0826822F00102D2
:105BF000826070470A4600214168D64B1940114324
:105C0000416070474162826270470A4600214168E4
:105C100021F01F0111434160704738B1CA4909683A
:105C200041F40001CA4AC2F8041306E0C6490968F3
:105C300021F40001C64AC2F80413704738B1C249C2
:105C4000096841F48001C24AC2F8041306E0BE4963
:105C5000096821F48001BE4AC2F804137047F0B508
:105C600004460D4600200021092D11DDE068A5F154
:105C70000A0606EB4607072606FA07F18843A5F150
:105C80000A0606EB460603FA06F10843E0600CE05C
:105C9000206905EB4507072606FA07F1884305EB5F
:105CA000450603FA06F108432061072A0FDA606B04
:105CB000561E06EB86071F2606FA07F18843561E76
:105CC00006EB860605FA06F10843606322E00D2A1A
:105CD0000FDA206BD61F06EB86071F2606FA07F1A0
:105CE0008843D61F06EB860605FA06F108432063B3
:105CF00010E0E06AA2F10D0606EB86071F2606FA01
:105D000007F18843A2F10D0606EB860605FA06F1B7
:105D10000843E062F0BD816841F0804181607047D6
:105D2000014600208A6802F080420AB1012000E0AA
:105D30000020704721B1826842F48062826003E0F3
:105D4000826822F480628260704721B1826842F0EA
:105D50000202826003E0826822F0020282607047E1
:105D600010B50A4600210023416821F46041531E0A
:105D700041EA4331416010BD21B1426842F4006202
:105D8000426003E0426822F40062426070470146CC
:105D9000C86C80B270476C48001D0068704721B124
:105DA000826842F48072826003E0826822F480722A
:105DB0008260704721B1826842F40072826003E021
:105DC000826822F400728260704738B15E490968C7
:105DD00041F400515E4AC2F8041306E05A490968CA
:105DE00021F400515A4AC2F804137047F0B5044632
:105DF0001546002000220026092911DDE068A1F1E6
:105E00000A0707EB470C072707FA0CF29043A1F1AA
:105E10000A0707EB470703FA07F21043E0600CE0BC
:105E2000206901EB410C072707FA0CF2904301EBC4
:105E3000410703FA07F210432061A06BC0F301563B
:105E4000EF1C06F1010CA7EB0C0707EB870C1F27D3
:105E500007FA0CF29043EF1C06F1010CA7EB0C07BC
:105E600007EB870701FA07F21043A063F0BD10B5F6
:105E70000A4600210023816B21F44011531E41EAA0
:105E80000351816310BD08B5002300930090009B6F
:105E90000B440093009B1A6008BD0A4600218168EC
:105EA00021F470211143816070470A460021816806
:105EB00021F44011114381607047816841F48001F1
:105EC00081607047014600208A6802F480020AB1AE
:105ED000012000E00020704721B1426842F4806256
:105EE000426003E0426822F480624260704721B160
:105EF000426842F48052426003E0426822F48052D9
:105F00004260704708B5024600200090009201F1FF
:105F10002800009B184400900098006880B208BDDB
:105F200010B50B460021D9B2012404FA01F11AB1CF
:105F300044680C43446002E044688C43446010BDF4
:105F4000FFFEFFFCFDF7FFC004230140E030FCFF33
:105F500000200140FFFD3FFF0246002013680B4078
:105F60000BB1012000E000207047CA430260704777
:105F700070B502460020002300240B12556801264C
:105F80008E4005EA060415681D4015B10CB10120CC
:105F900000E0002070BD00220A12D3430360704766
:105FA0000E49086070470D49486070470B4988608A
:105FB00070474AF6AA200949086070474CF6CC4061
:105FC00006490860704701460020044AD2680A402A
:105FD0000AB1012000E000207047000000300040BE
:105FE000704700000FB4044910B503AA029817F0D7
:105FF00033FF10BC5DF814FBD80000207047000090
:106000000000000000000000000000000000000090
:106010000000000000000000000000000000000080
:1060200057313800000000000000000000000000B0
:106030000001000000020000640000004D617920B2
:10604000323920323032350032303A32353A343358
:106050000000000053544D33324634313252450073
:106060004E4F4E4500000000000000000000000000
:106070004E4F4E45000000000000000000000000F0
:106080003132302E32342E3234322E36333A3830EA
:10609000313500000000000000000000000000009A
:1060A0007777772E67756F7965652E636F6D000062
:1060B00000000000000000000000000000000000E0
:1060C0003133393232323830353836000000000092
:1060D0003133393232323832353836000000000080
:1060E0004E4F4E4500000000000000000000000080
:1060F00000000000000000000000000000000000A0
:10610000000000000000000000000000000000008F
:10611000000000000000000000000000000000007F
:10612000000000000000000000000000000000006F
:10613000000000000000000000000000000000005F
:106140004D6F64656C3A2057313820202C4D4355F3
:106150003A2053544D33324634313252452C486143
:1061600072645665723A312E302C536F66745665E0
:10617000723A312E302E300D0A000000E007000088
:10618000485F302E312E3020535F312E302E3000BC
:1061900010B50446FE48844208D101210846FFF7A5
:1061A000FEF900210120FFF7FAF99DE0B4F1804FDC
:1061B00008D101210846FFF7E1F900210120FFF78E
:1061C000DDF991E0F348844208D101210220FFF774
:1061D000D5F900210220FFF7D1F985E0EE4884428D
:1061E00008D101210420FFF7C9F900210420FFF79D
:1061F000C5F979E0E948844208D101210820FFF778
:10620000BDF900210820FFF7B9F96DE0E4488442A8
:1062100008D101211020FFF7B1F900211020FFF76C
:10622000ADF961E0DF48844208D101212020FFF769
:10623000A5F900212020FFF7A1F955E0DA488442B2
:1062400008D101210220FFF7AAF900210220FFF75F
:10625000A6F949E0D548844209D101210804FFF795
:106260009EF900214FF48030FFF799F93CE0D048C7
:10627000844209D101214804FFF791F900214FF42C
:106280000030FFF78CF92FE0CA48844209D1012180
:106290008804FFF784F900214FF48020FFF77FF98D
:1062A00022E0C548844208D101214020FFF766F969
:1062B00000214020FFF762F916E0C048844208D16F
:1062C00001218020FFF75AF900218020FFF756F9BD
:1062D0000AE0BB48844207D101218015FFF74EF93F
:1062E0000021A015FFF74AF910BD00220288A84B33
:1062F00098420ED0AC4B98420BD0B0F1804F08D0F2
:10630000A44B984205D0A44B984202D0A34B98428C
:1063100004D14FF68F731A404B881A43A04B984212
:1063200007D0A04B984204D04FF6FF431A400B8988
:106330001A4302804B68C3620B880385944B9842D2
:1063400002D0994B984201D18B7A03860123838234
:1063500070474FF0FF314160002101800181418091
:10636000817270470185828270470A460021018848
:106370004FF68F7319401143018070474162704797
:10638000C16270470146486A70470146088D7047F0
:1063900021B1028842F00202028004E002884FF636
:1063A000FD731A400280704721B1028842F0040256
:1063B000028004E002884FF6FB731A4002807047A7
:1063C00021B1028842F08002028004E002884FF688
:1063D0007F731A400280704702884FF6F7731A40A5
:1063E000028002880A430280704702884FF6FF430A
:1063F0001A40028002880A430280704721B1028855
:1064000042F00102028004E002884FF6FE731A4057
:106410000280704770B5002400220023058C4FF6DF
:10642000FE7635400584028C8388048B4FF68F7589
:106430002C40B51E2C400D882C43751E2A408D899A
:106440002A434D882A43524DA84202D0564DA842B5
:1064500013D14FF6F7752A40CD892A434FF6FB75C5
:106460002A408D882A434FF6FF652B404FF6FF5593
:106470002B400D8A2B434D8A2B43838004838D68E8
:106480004563028470BD70B5002400220023058C92
:106490004FF6EF7635400584028C8388048B48F6EE
:1064A000FF752C404FF6FF452C400D884FF6FF76C8
:1064B00006EA05252C434FF6DF752A408D8906EA4A
:1064C00005152A434D8806EA05152A43304DA84292
:1064D00002D0354DA8421DD14FF67F752A40CD8997
:1064E0004FF6FF7606EA05152A434FF6BF752A4098
:1064F0008D8806EA05152A434FF6FF352B404FF2EB
:10650000FF752B400D8A06EA85052B434D8A06EA66
:1065100085052B43838004838D688563028470BD69
:1065200070B5002400220023058C4FF6FF6635402D
:106530000584028C8388848B4FF68F752C404FF630
:10654000FC752C400D882C434FF6FF552A408D8951
:106550004FF6FF7606EA05252A434D8806EA05250B
:106560002A430B4DA84202D00F4DA84238D14FF21A
:10657000FF752A40CD894FF6FF7606EA05252A43A6
:106580004FF6FF352A408D8806EA05252A4319E093
:10659000000001400004004000080040000C0040E2
:1065A0000010004000140040000401400040014081
:1065B000004401400048014000180040001C004019
:1065C000002000404EF6FF752B404DF6FF752B4026
:1065D0000D8A06EA05152B434D8A06EA05152B435D
:1065E000838084838D68C563028470BD70B500228A
:1065F00000230024058C4EF6FF7635400584038C7D
:106600008488828B48F6FF752A404FF6FF452A4062
:106610000D884FF6FF7606EA05252A434DF6FF75ED
:106620002B408D8906EA05352B434D8806EA053552
:106630002B43FE4DA84202D0FD4DA84208D14BF697
:10664000FF752C400D8A4FF6FF7606EA85152C4320
:10665000848082838D680564038470BD002101807D
:106660004180818081608181C18101824182704746
:1066700070B50346002000241846183001258D40CF
:10668000ACB21D8CA5431D8409B108290AD100EBC9
:10669000610005684FF68F76354005600568154343
:1066A00005600FE00D1FC5F34E052844056848F648
:1066B000FF763540056005684FF6FF7606EA02264C
:1066C0003543056070BD4163704781637047C163A6
:1066D0007047016470470A460021018B4FF68F73A3
:1066E00019401143018370470A460021018B48F687
:1066F000FF7319404FF6FF7303EA02231943018326
:1067000070470A460021818B4FF68F731940114361
:10671000818370470A460021818B48F6FF73194038
:106720004FF6FF7303EA02231943818370470A4639
:106730000021018B4FF6F773194011430183704715
:106740000A460021018B4FF2FF7319404FF6FF7389
:1067500003EA02231943018370470A460021818B13
:106760004FF6F77319401143818370470A460021A1
:10677000818B4FF2FF7319404FF6FF7303EA022338
:106780001943818370470A460021018B4FF6FB7342
:1067900019401143018370470A460021018B4FF6CF
:1067A000FF3319404FF6FF7303EA022319430183B5
:1067B00070470A460021818B4FF6FB731940114345
:1067C000818370470A460021818B4FF6FF331940C1
:1067D0004FF6FF7303EA02231943818370470A4689
:1067E0000021018B4FF67F731940114301837047DD
:1067F0000A460021018BC1F30E014FF6FF7303EA35
:1068000002231943018370470A460021818B4FF60A
:106810007F7319401143818370470A460021818BA1
:10682000C1F30E014FF6FF7303EA0223194381837C
:1068300070470A460021018C4FF6FD731940114341
:10684000018470470A460021018C4FF6F773194006
:106850001143018470470A460021018C4FF6DF7313
:1068600019404FF6FF7303EA02131943018470477E
:106870000A460021018C4FF67F7319404FF6FF73D3
:1068800003EA02131943018470470A460021018C70
:106890004FF6FF5319404FF6FF7303EA02231943E3
:1068A000018470470A460021018C4FF2FF731940A2
:1068B0004FF6FF7303EA02231943018470470A4627
:1068C0000021018C4DF6FF7319404FF6FF7303EA68
:1068D000023319430184704730B5002301248C40F2
:1068E000A3B2048C9C430484048C02FA01F5ADB27B
:1068F0002C43048430BD30B5002304248C40A3B263
:10690000048C9C430484048C02FA01F5ADB22C4340
:10691000048430BD828B4FF2FF331A408283828B16
:106920004FF6FF7303EA01231A4382837047F0B5E1
:106930000C461546002100220026078C4EF6FF7CEF
:1069400007EA0C070784818B028C4FF6FF7707EA72
:10695000043640F6FF4739404FF6FF7707EA052730
:1069600039434FF6FF7707EA0337394345F6FF7798
:106970003A4046F480573A4381830284F0BD828BCB
:106980004FF6F3731A408283828B0A4382837047E7
:10699000F0B50C461546002100220026078C4FF664
:1069A000FF6C07EA0C070784818B028C4FF6FF7798
:1069B00007EA04264FF60C7739404FF6FF7707EACF
:1069C00003172F4339434FF2FF573A4046F480777D
:1069D0003A4381830284F0BD028B4FF2FF331A40A9
:1069E0000283028B4FF6FF7303EA01231A430283EB
:1069F0007047F0B50C461546002100220026078C92
:106A00004FF6EF7C07EA0C070784018B028C4FF6E8
:106A1000FF7707EA041640F6FF4739404FF6FF7745
:106A200007EA033739434FF6FF7703E000000140E0
:106A30000004014007EA052739434FF65F773A40E3
:106A400046F010073A4301830284F0BD028B4FF6F3
:106A5000F3731A400283028B0A4302837047F0B536
:106A60000C46154600210022068C4FF6FE773E406C
:106A70000684018B028C4FF60C7631407E1C06EAB0
:106A800003162E4331434FF6F576324044F00106AB
:106A9000324301830284F0BD70B505460C46208860
:106AA00050B92389A28861882846FFF7D8FFE1887A
:106AB0002846FFF7CBFF25E0208804280AD1238948
:106AC000A28861882846FFF794FFE1882846FFF7EF
:106AD00083FF17E0208808280AD12389A2886188CB
:106AE0002846FFF755FFE1882846FFF748FF09E0F1
:106AF0002389A28861882846FFF719FFE188284684
:106B0000FFF708FF70BD00210180418001218180D5
:106B10000021C180018170472DE9F04105460C46F6
:106B200000260127608808B9022600E00026A08818
:106B3000012801D1022700E001272088A0B923897C
:106B4000A28861882846FFF78AFFE1882846FFF778
:106B50007DFF23893A4631462846FFF74AFFE18800
:106B60002846FFF739FF13E02389A2886188284669
:106B7000FFF73FFFE1882846FFF72EFF23893A46BB
:106B800031462846FFF76BFFE1882846FFF75EFF96
:106B9000BDE8F0810146486B70470146886B70473D
:106BA0000146C86B70470146086C70470A884B88DD
:106BB0001A438B881A43CB881A430B891A434B8993
:106BC0001A438B891A43A0F84420704700210180A2
:106BD00041808180C180018141818181704731B1D3
:106BE000B0F8442042F40042A0F8442005E0B0F898
:106BF0004420C2F30E02A0F84420704721B18288DD
:106C000042F00402828004E082884FF6FB731A404F
:106C10008280704721B1828842F00102828004E0C4
:106C200082884FF6FE731A40828070471AB18389BA
:106C30000B43838102E083898B4383817047818288
:106C4000704702460020138A0B400BB1012000E080
:106C500000207047CA430282704730B502460020C8
:106C600000230024158A05EA0103958905EA010439
:106C700013B10CB1012000E0002030BDCA430282F4
:106C8000704741EA0203A0F8483070471AB183897F
:106C90000B43838102E083898B438381704721B159
:106CA000828842F00802828004E082884FF6F773FF
:106CB0001A408280704701894FF6F87211400181B5
:106CC00070470A46002101894FF68F73194011431E
:106CD0000181704730B504460D4629462046FFF72E
:106CE000F0FF208940F00700208130BD2DE9F04100
:106CF00004460D4616461F46602D06D13B4601222E
:106D000031462046FFF775FE05E03B46012231463D
:106D10002046FFF7A4FE29462046FFF7D2FF208930
:106D200040F007002081BDE8F08130B50C4600211D
:106D30000189C9B24FF6FF7505EA032515432543BE
:106D40002943018130BD2DE9F04105460E46174625
:106D50009846002443463A4631462846FFF7E5FF69
:106D60002C894FF6F870044044F007044FF68F70FA
:106D7000044044F070042C81BDE8F081F0B5044675
:106D80000D4616461F463B46324629462046FFF72B
:106D9000CCFF208940F480402081F0BD82884FF6EE
:106DA0008F731A40828082880A43828070470289EA
:106DB0004FF6F8731A40028102890A430281704734
:106DC00002894FF67F731A40028102890A430281C9
:106DD0007047F0B50C4615461E46002100220023E0
:106DE0000189028B038C4FF6F877394021434FF627
:106DF000FC473A4040F201173A434FF6DD773B40FB
:106E00004FF6FF7707EA06172F433B4301810283C2
:106E10000384F0BD21B1828842F08002828004E0C8
:106E200082884FF67F731A4082807047A0F8501016
:106E30007047000010B50446FB48844208D1012188
:106E40008014FEF7ACFB0021A014FEF7A8FB3CE089
:106E5000F648844208D101210014FEF78FFB00217F
:106E60002014FEF78BFB30E0F148844208D1012169
:106E7000C013FEF783FB0021E013FEF77FFB24E045
:106E8000EC48844208D101214014FEF788FB002120
:106E90006014FEF784FB18E0E748844209D1012121
:106EA0000805FEF77CFB00214FF48010FEF777FB0E
:106EB0000BE0E248844208D101214805FEF76FFB50
:106EC00000214FF40010FEF76AFB10BD10B5002240
:106ED000028802F441520B884C8823438C88234358
:106EE000CC8823430C8923434C8923438C89234337
:106EF000CC8923431A430280838B4FF2FF742340D3
:106F000083830B8A038210BD2DE9F04F00250223F5
:106F100000244FF0010900220026002794469046E5
:106F2000B0F81CA04FF2400B0AEA0B0AA0F81CA014
:106F30004FF0020AA0F820A0858BD1F808A0BAF182
:106F4000020F01D100BF82E0B1F804A0BAF1000F36
:106F500002D14FF0010901E04FF00209DFF8E0A291
:106F6000DAF800A00AF4000ABAF1000F09D0DFF83D
:106F7000D0A2DAF800A02AF4000ADFF8C4B2CBF8F5
:106F800000A0DFF8BCA20AF17C0ADAF800A0CAF37C
:106F9000881CDFF8ACA20AF17C0ADAF800A0CAF378
:106FA0000278DFF89CA2AAF1040ADAF800A00AF03D
:106FB0003F07DFF88CA2AAF1040ADAF800A00AF46D
:106FC000800ABAF5800F08D1DFF878A2BAFBF7FA89
:106FD0000AFB0CFABAFBF8F607E0DFF86CA2BAFB82
:106FE000F7FA0AFB0CFABAFBF8F6B1F806A0BAF504
:106FF000007F0ED14FEA162A0AEB8A0A4FEA4A0AA4
:10700000D1F808B0BAFBFBFA0AF1050A1FFA8AF2B6
:107010000FE04FEA491AB6FBFAFA0AEB8A0A4FEA7E
:107020004A0AD1F808B0BAFBFBFA0AF1050A1FFABE
:107030008AF24FF00A0AB2FBFAF202F00104A2EB64
:10704000040ACAF34F034FF6FF7A0AEA0424022B1C
:1070500001DBFF2B01DD02230024B1F806A04AEA80
:10706000040A4AEA030AA0F820A0B1F804A0B1F883
:107070000CB04AEA0B0AB1F802B04AEA0B0AB1F8BE
:1070800000B04AEA0B0A4AF4006A4AEA0505858319
:10709000BDE8F08F0021018041808180C1800181A5
:1070A00041818181C18107210182704700210180D6
:1070B00041808180C18002218160002181817047EF
:1070C00021B1028842F04002028004E002884FF6BB
:1070D000BF731A400280704721B1828B42F48062F4
:1070E000828304E0828B4FF6FF331A40828370471D
:1070F00002884FF2FF731A40028002880A4302801E
:107100007047B1F5804F04D1028842F4804202807A
:1071100004E002884BF6FF731A40028070474FF676
:10712000FF62914204D0028842F48072028004E03F
:1071300002884FF6FF631A400280704721B18288AF
:1071400042F00402828004E082884FF6FB731A400A
:107150008280704721B1828842F01002828004E070
:1071600082884FF6EF731A408280704730B5002254
:107170000023848B4FF240052C4084830224048436
:10718000828B0C88B4F5007F01D00C8814B94FF4C1
:10719000807308E00C88B4F5407F03D00C88B4F508
:1071A000807F00D100238C888D892C434D882C430F
:1071B0001C4344F400642243828330BD0146888925
:1071C00070478181704721B1028842F400520280E9
:1071D00004E002884DF6FF731A4002807047018870
:1071E00041F480510180704702460020012901D0FE
:1071F000108B00E0908A70470146088A70471AB1E8
:1072000083880B43838002E083888B4383807047AD
:1072100030B5002400230C110125A540ABB2AAB162
:1072200085881D43858014E000300140003800400F
:10723000003C004000340140005001400054014037
:107240000838024000127A000024F40085889D432B
:10725000858030BD0246002013890B400BB1012010
:1072600000E000207047CA4302817047F0B5024633
:10727000002000240023002501F00F070126BE4056
:10728000B4B20B1101269E40B3B2968806EA0305FC
:107290001689264016B10DB1012000E00020F0BD96
:1072A00010B5002201F00F040123A3409AB2D3438A
:1072B000038110BD10B5044614B909F007FF044658
:1072C0000CB9002010BD206BFCE770B504462046C9
:1072D00001F00CFF05462C63204601F033FF70BD22
:1072E00010B5044614B909F0F1FE04460CB90020AB
:1072F00010BD606BFCE710B5044614B909F0E6FE5A
:1073000004460CB9002010BDA06BFCE770B5054623
:107310000E46304601F0D4FE00B170BD304601F09B
:10732000E5FE0446AC4200D1F7E70123324605F101
:10733000240104F124000AF069FE00BFEDE710B556
:10734000044614B909F0C2FE04460CB9002010BD71
:10735000206AFCE770B5044614B909F0B7FE04468C
:107360000CB9002070BD24B1D4F860010AF01CF8FB
:10737000F8E74FF0FF36002009F038FF054610E02F
:10738000D5F860010AF010F8B04201D9304603E0A8
:10739000D5F860010AF008F80646284609F026FFED
:1073A0000546002DECD13046DCE710B5044614B993
:1073B00009F08CFE044604B910BD09F0EAFFC4F8D8
:1073C000600100BFF8E7000007B581B0BDF8080014
:1073D000C00AC2F1FF014843BDF80410C90A01FB0D
:1073E0000200010ABDF8000061F3CF200090BDF853
:1073F0000800C0F34510C2F1FF014843BDF8041076
:10740000C1F3451101FB0200010ABDF8000061F360
:107410004A100090BDF8080000F01F00C2F1FF0103
:107420004843BDF8041001F01F0101FB0200010AEE
:10743000BDF8000061F304000090BDF8001008469C
:1074400004B000BD10B55C21FA480AF0AEFC10BDD6
:1074500030B587B005460C46FF21E173F648006859
:107460000690A01CBDF818106181207A08B9A08987
:1074700008B10321A181F048001D006805906088D3
:10748000B22200900599FFF79FFF0190BDF804001C
:107490006080E948083000680490A088B22200901B
:1074A0000499FFF791FF0190A01CBDF80410A18082
:1074B000E1480C3000680390208A992200900399DB
:1074C000FFF782FF0190A01CBDF804102182DA486A
:1074D000103000680290B2220299206AFFF774FF10
:1074E0000190BDF8040020843220005D10280ADAE3
:1074F000D148143000680190BDF804002086662150
:107500003220015500BF07B030BD30B587B0054609
:107510000C46FF21E173C848183800680690A01C8B
:10752000BDF818106181207A08B9A08908B103213B
:10753000A181C1481438006805906088B22200908B
:107540000599FFF741FF0190BDF804006080BA483B
:10755000103800680490A088B22200900499FFF7C8
:1075600033FF0190A01CBDF80410A180B2480C3874
:1075700000680390208A992200900399FFF724FF66
:107580000190A01CBDF804102182AB4808380068A7
:107590000290B2220299206AFFF716FF0190BDF80F
:1075A000040020843220005D10280ADAA248001F5F
:1075B00000680190BDF80400208666213220015544
:1075C00000BF07B030BD9D4A02619D4A426169B16A
:1075D000D1F8A82112B1D1F8A82102614FF4D672D6
:1075E00052581AB14FF4D67252584261704770B572
:1075F00090480AF013FC04460CB900BFFEE70CB932
:10760000002070BD042120460AF0CFFB0020393451
:1076100044F82D0CE07F20F00100E077002044F8D2
:10762000210CE07F20F00400001DE077E07F20F0D7
:107630000200E077E07F20F008000830E077E07F8C
:1076400020F010001030E077393C0DF09DFF05462A
:1076500029462046FFF7B7FF2046D2E770B504461B
:10766000E06848B1E168086800221021C3699847C2
:10767000E168086801F066FD20460AF0F9FB05465E
:1076800007E000202968C862294620460AF051FC1C
:107690000546002DF5D120460AF0A0FC214665489C
:1076A0000AF057FC20460AF036FE70BD70B505465C
:1076B0002C46002609E094F83000C0F3401000B1D9
:1076C0002646204601F0FCFC0446002CF3D116B1FE
:1076D000304602F067FA70BD2DE9F84F044688463F
:1076E000914694F8580000F0010008B1BDE8F88F09
:1076F000E56800264FF0010A4FF0010B00BF8DB97D
:1077000094F85800C0F3001000B956B9BBF1000F4F
:1077100000D1EBE72046C04705464FF0000AD346AC
:1077200000E0E3E716B92E4606B9DFE7BAF1000F2D
:1077300006D029462046C8470546B54200D1D5E7C0
:107740004FF0010A05B9DAE7286801F0BCFC00B97E
:1077500000E0D4E700BFE068A84200D1C6E7E068D7
:10776000A8B1E168086800221021C3699847E16860
:10777000002208680D2102F0B1F80090009801285D
:1077800000D0B3E7E168086801F0DCFC00BFE56009
:10779000E168086800220F21C3699847E168002268
:1077A00008680C2102F09AF80746012F00D09DE7E7
:1077B000E1680868FFF77AFFE168086801F0C2FC39
:1077C000A06910B12046A169884700BF8EE710B5B7
:1077D00004461C4A1C492046FFF77EFF10BD10B529
:1077E00004461A4A1A492046FFF776FF10BD70B5C5
:1077F000044614F8580FC0F30015207820F010004C
:107800001030207014F85809C0F3C00018B9204691
:10781000FFF7E5FF07E094F85800C0F3C00010B18F
:107820002046FFF7D4FF94F8580065F3041084F85D
:10783000580070BDC42E0020380902080B750008DE
:10784000517400085D1E0108491F0108331F01081B
:10785000711E01082DE9F04107460C460FB9BDE83D
:10786000F08138460AF004FB064608E03068A04282
:1078700000D1F4E7314638460AF05BFB0646002E9D
:10788000F4D1E06A30B1204603F011F810B1E06A9B
:10789000FFF7ADFFE76238460AF028FB05460DB951
:1078A00000BFFEE705B9DAE72C6038460AF0E0FAD7
:1078B000A84202D13846FFF79AFF00BFCFE770B564
:1078C0000546EC6A04B970BDE06800B9FBE7E06802
:1078D0000068A84215D120460AF0CAFAE168884239
:1078E0000CD120460AF030FBE168884206D1E168FD
:1078F000086800221021C369984702E02046FFF77C
:1079000076FFE0680068A84201D10020E0602046D0
:107910000AF0AEFA064611E03068A84209D13146B5
:1079200020460AF016FB30460AF0F5FC0020E8621B
:1079300006E0314620460AF0FCFA0646002EEBD15E
:1079400000BF00BFBFE770B50446E06858B1E1680A
:10795000086800221021C3699847E168086801F0AF
:10796000F1FB0020E06020460AF082FA054607E0BD
:1079700000202968C862294620460AF0DAFA05463E
:10798000002DF5D120460AF029FB70BD014609B94A
:1079900000207047C86808B90020FAE7C868006886
:1079A000F7E72DE9F04104460E46374694F85800B3
:1079B000C0F34000B84201D1BDE8F08194F858000E
:1079C00067F3410084F858002046FFF7DFFF0546C3
:1079D00085B100220F212846EB699847E168002213
:1079E00008680C2101F07AFF8046B8F1010F00D041
:1079F000E2E700BF284601F0A5FB00BFDCE72DE968
:107A0000F04106460EB9BDE8F081F46A04B9FAE720
:107A100094F8580000F0010000B1F4E7002120467E
:107A2000FFF7BFFF20460AF023FA054640E028682A
:107A3000B04238D1E068A0B1E168086800221021A6
:107A4000C3699847E168002208680D2101F046FFEC
:107A50000746012F00D0D6E7E168086801F072FB05
:107A600000BFE560E068E8B1E168086800220F2126
:107A7000C3699847A06910B12046A1698847E168A9
:107A8000002208680C2101F029FF0746012F00D0D1
:107A9000B9E7E168086801F055FBE1680868FFF79D
:107AA00005FE00BF06E0294620460AF042FA0546D8
:107AB000002DBCD100BF00BFA5E731B990F8582018
:107AC00022F0010280F8582006E090F8582022F0B9
:107AD0000102521C80F85820704773B506463046A4
:107AE000FFF754FF05460DB901207CBD01AA112105
:107AF0002846EB6998470446012C01D02046F4E75C
:107B000001AA0B21284601F0E9FE0446012C01D010
:107B10002046EAE72046E8E770B504460D462561B1
:107B2000E06818B1E168086801F00CFB70BD70B541
:107B300004460D466561E06818B1E168086801F027
:107B400001FB70BD8161704790F8582061F382029B
:107B500080F85820704790F8582061F3C30280F8ED
:107B60005820704790F8582061F3041280F858208C
:107B7000704770B504460D46294604F11C0003F019
:107B8000F9FA94F85800C0F3400038B1606960B168
:107B900004F11C0120466269904706E0206920B18B
:107BA00004F11C0120462269904704F11C0070BDBD
:107BB000014609B9002070470869FCE7014609B988
:107BC000002070474869FCE7014609B9002070476A
:107BD0008869FCE7014609B90020704791F8580010
:107BE000C0F34000F9E7014609B90020704791F859
:107BF0005800C0F38000F9E7014609B9002070473A
:107C000091F85800C0F30010F9E770B505460DF083
:107C1000BBFC064625B131462846FFF7D4FC70BDB3
:107C200008480AF025F9044608E031462046FFF7E7
:107C3000CAFC214603480AF07CF90446002CF4D122
:107C400000BFECE7C42E002070B504463CB194F8A8
:107C50004C0020F00200801C84F84C0012E0002050
:107C600009F05FFB05460AE095F84C0020F00200A1
:107C7000801C85F84C00284609F053FB0546002D72
:107C8000F2D100BF70BD10B50020FFF7DDFF10BDC1
:107C900090F84C10C1F3400129B300224263826383
:107CA000C26390F8401021F0010280F8402090F863
:107CB000401021F0020280F8402090F84C1021F092
:107CC000010280F84C200022426482648285C285D1
:107CD0000286428690F84C1021F0020280F84C2077
:107CE0000021FE4A11607047014691F83000C0F350
:107CF000400010B10020F94A106091F83000C0F344
:107D0000400070472DE9FF41044694F82400C0F379
:107D1000400008B9BDE8FF81E56903E0284601F0AD
:107D2000CFF90546284602F075FD08B1002DF5D1C2
:107D300005B9EFE7284602F067FDD8B994F82400AA
:107D400020F0020184F82410E548EB690E21026856
:107D50002846984700220921284601F0BFFD204609
:107D6000FFF7C2FF00B1D5E700220921284601F044
:107D7000B5FDCFE7284602F041FD0646A08AD84966
:107D80000968497DC1F1640110FB01F0642190FB99
:107D9000F1F001B2A182E08AD1490968497DC1F1BF
:107DA000640110FB01F0642190FBF1F001B2E1826B
:107DB000A08A10B9E08A00285DD002A9284601F007
:107DC00050FA284601F0B3FAA18A08440FFA80F865
:107DD000284601F0A0FA0146E08A084407B2032EC3
:107DE00005D13A464146284601F044FA0EE006F035
:107DF000010020B14146284601F012FF06E006F0DE
:107E0000020018B13946284601F017FF6946284696
:107E100001F027FABDF90800BDF90010884201D031
:107E2000A08A38BBBDF90A00BDF90210884201D012
:107E3000E08AF8B994F8240020F0020184F82410B4
:107E40000021A181E181A182E182A548EB690E2197
:107E50000268284698472046FFF746FF00B159E7D9
:107E600000220921284601F039FD2046FFF73CFF9A
:107E700000B14FE71AE094F8240020F0020184F8E2
:107E800024109748EB690E2102682846984720463F
:107E9000FFF72AFF00B13DE700220921284601F043
:107EA0001DFD2046FFF720FF00B133E700BF31E79B
:107EB0002DE9F041044694F83000C0F3C00058B1F9
:107EC0000021A161E1610020A062E06294F830002D
:107ED00020F0080084F830008049A0690860084656
:107EE0000068002874D010217C48006801F0F4FA82
:107EF00000283AD079480068C36979480A210268A5
:107F00007648006898472046FFF7EEFE08B1BDE8C6
:107F1000F08194F82400C0F34000D0B994F8300008
:107F200000F0010050B9002203216C48006801F004
:107F3000D5FC2046FFF7D8FE00B1E8E70022062175
:107F40006648006801F0CAFC2046FFF7CDFE00B18C
:107F5000DDE7002207216148006801F0BFFC2046F0
:107F6000FFF7C2FE00283FD0D1E75C480068C36934
:107F70005B480A2102685948006898472046FFF785
:107F8000B3FE00B1C3E794F8300000F0010078B907
:107F900094F82400C0F3400050B9002203214F4858
:107FA000006801F09BFC2046FFF79EFE00B1AEE7A3
:107FB00094F82400C0F3400058B900220621474835
:107FC000006801F08BFC2046FFF78EFE08B19EE7AB
:107FD0008EE0002207214148006801F07FFC204626
:107FE000FFF782FE00B192E72046FFF77DFE00B169
:107FF0008DE74FF000083948006801F0B8F90546F0
:1080000020213648006801F067FA10BB3348076842
:1080100010E0384601F054F8074607B90CE020217B
:10802000384601F059FA08B1002705E0384601F05A
:108030009EF90546002DECD000BF4DB147B1284652
:10804000FFF7D1FD20B14FF001083846FFF7D7FC0C
:1080500000BF2249206A0968884219D0B8F1000F90
:1080600016D100220D21206A01F038FC2046FFF7CE
:108070003BFE00B14BE700220C21A06901F02EFC71
:108080002046FFF731FE00B141E714480168216244
:108090002046FFF729FE00B139E71048066803E0E3
:1080A000304601F00DF80646304602F0B3FB08B149
:1080B000002EF5D1B6B1304602F0A6FB90B194F88F
:1080C0002400C0F3400068B100220A21304601F0CC
:1080D00005FC2046FFF708FE20B118E7F00000205D
:1080E000EC0000200021A1610020A062E06200BF3E
:1080F000E06960B194F83000C0F3400038B9204620
:10810000FFF700FE2046FFF7EFFD00B1FFE600BFDE
:10811000FDE62DE9F04F87B00446A569002703E08E
:10812000284600F0CDFF0546284602F073FB08B153
:10813000002DF5D115B907B0BDE8F08F284602F043
:1081400057FB00B9F7E7284602F058FB0646218A9C
:10815000A089084401B22182618AE089084401B201
:10816000618294F8240000F0010058BB06F0010081
:1081700070B1B4F91000002802DDB4F9100002E07B
:10818000B4F910004042F8490968097D884211DAC3
:1081900006F00200B0B1B4F91200002802DDB4F913
:1081A000120002E0B4F912004042EF490968097D6B
:1081B000884207DB94F8240020F00100401C84F87A
:1081C0002400012794F8240000F0010000287DD04D
:1081D000A08910B9E0890028F9D0E3490968C86886
:1081E00009F013F88246B5F910B0B5F912000690FF
:1081F000284600F065FF039001F034FD0590284605
:1082000000F05EFF039001F025FD0490284601F088
:108210008EF88046284601F07EF88146032E12D162
:108220003FB1208A40440FFA80F8608A48440FFA30
:1082300080F9E089484402B2A089404401B228464E
:1082400001F018F81CE006F0010058B11FB1208AB7
:1082500040440FFA80F8A089404401B2284601F05A
:10826000DFFC0DE006F0020050B11FB1608A484407
:108270000FFA80F9E089484401B2284601F0DDFC9C
:10828000B5F9100058452DD1B5F912100698814264
:1082900028D1284600F014FF019001F0E3FC039080
:1082A000284600F00DFF019001F0D4FC02900599E2
:1082B0000398884215D104990298884211D1AA499D
:1082C0000968C86808F0A1FF019000E028E0019A61
:1082D000A2EB0A0291B2A44A1268D06808F09BFF90
:1082E00000BF1CE094F8240020F00200801C84F8F9
:1082F0002400A7B19C48EB690D21026828469847E5
:108300002046FFF7F1FC00B115E7002208212846BE
:1083100001F0E4FA2046FFF7E7FC00B10BE700BFED
:1083200000BF08E72DE9F04107460C460025391D3E
:1083300004F1100009F08BFB00282BD0201D09F060
:1083400097FD80460BE041463846FFF7EBFF0546B8
:1083500005B107E04146201D09F0EBFD8046B8F16C
:10836000000FF0D100BFA5B9204602F035FA80B168
:10837000264608E0304600F0A6FE00B105E0304693
:1083800000F09EFE0646002EF4D100BF06B9254639
:1083900000BF00BF2846BDE8F0812DE9F04104464A
:1083A0007249A069086094F83000C0F3C00008B1B9
:1083B000BDE8F0816C480068C66800276B4800681B
:1083C00028BB3046FEF797FF054629462046FFF7B3
:1083D000A9FF664908600846006848B93046FEF7BC
:1083E0007FFF054629462046FFF79CFF5F4908604E
:1083F0005E48006848B93046FEF75CFF05462946EE
:108400002046FFF78FFF5949086001272FE094F8B5
:108410002400C0F3400050BB10215448006801F014
:108420005BF820BB3046FEF766FF0546294620462E
:10843000FFF778FF4D4908600846006848B93046A4
:10844000FEF74EFF054629462046FFF76BFF4749DA
:1084500008604648006848B93046FEF72BFF0546DD
:1084600029462046FFF75EFF4049086001273FB1DB
:10847000E06928B10021A182E1822046FFF742FC99
:108480003A49A0690968884273D0A1882181E188AE
:108490006181A069B0B1A5693348EB69092102681F
:1084A000284698472046FFF71FFC00B180E70022CE
:1084B0000221284601F012FA2046FFF715FC00B110
:1084C00076E700BF29480168A1610168E1610068A1
:1084D00000284ED008F05DFFA06294F8300020F034
:1084E000010084F8300094F8240020F0010184F8A1
:1084F000241094F8240020F0020184F824100021B4
:1085000021826182A181E18118480568884609E0DD
:1085100095F83000C0F3401000B1A846284600F09E
:10852000CFFD0546002DF3D1B8F1000F02D0404633
:1085300001F038FB0D480068C3690B480721026849
:108540000A48006898472046FFF7CEFB00B12FE7A6
:10855000002211460548006801F0C0F92046FFF7E7
:10856000C3FB28B124E704E0EC000020F000002069
:1085700000BFA1882089081A01B2A181E188608921
:10858000081A01B2E181B4F9140000EB8000C010B8
:10859000A082B4F9160000EB8000C110E182B4F9AA
:1085A0001400002804DAA08A401C01B2A18207E06E
:1085B000B4F91400002803DDA08A401E01B2A18294
:1085C000B4F91600002804DAE08A401C01B2E18206
:1085D00007E0B4F91600002803DDE08A401E01B26E
:1085E000E182A18AB4F90C00800001EBE00001B245
:1085F000A182E18AB4F90E00800001EBE00001B233
:10860000E182F9480068002875D0F7480068C3691E
:10861000F64808210268F448006898472046FFF7AA
:1086200063FB00B1C4E600220121EF48006801F0BD
:1086300055F92046FFF758FB00B1B9E62046FFF791
:1086400068FD2046FFF750FB00B1B1E694F8240026
:10865000C0F3400078BB94F8300000F0010050BB3C
:10866000A06A08F0A1FEE1490968C98A884222D9B6
:10867000DD480068C369DD480B210268DA480068FC
:1086800098472046FFF730FB00B191E60022042115
:10869000D548006801F022F92046FFF725FB00B11C
:1086A00086E694F8300020F00100401C84F8300089
:1086B00008F06FFEE06294F82400C0F34000D0B9E7
:1086C00094F8300000F00100A8B1E06A08F06CFEF8
:1086D000C6490968098B88421CD9C3480068C36928
:1086E000C2480C210268C048006898472046FFF73E
:1086F000FBFA08B15CE60DE000220521BA480068EB
:1087000001F0ECF82046FFF7EFFA00B150E608F070
:1087100040FEE06200BF4BE670B504460D46A06D1A
:10872000A96830F821102184A06DA96800EB8100B0
:1087300041886184B4F92410B4F9200081420DD13C
:10874000B4F92610B4F92200814207D1A87B012890
:1087500004D104F11C00FFF720FE03E004F11C002B
:10876000FFF7A6FB218CA184618CE18470BD2DE90B
:10877000F84304460D46A87B012806D194F84C0026
:10878000C0F3C00008B1BDE8F88394F84C00C0F312
:10879000C00080B194F84C0020F0080184F84C101F
:1087A0000021616494F84C0020F0010184F84C1021
:1087B00000212020015594F82080A97B202001551C
:1087C00069686162676D07B9DDE73846FFF7DEF873
:1087D000854908600846006800B9D4E7A87B0028EE
:1087E00043D13846FFF7F6F900B3B5F90C0000287D
:1087F0000CDA002604E014213846FFF76EF9761CE7
:10880000B5F90C004042B042F5DC0EE0B5F90C00C1
:1088100000280ADD002604E013213846FFF75DF941
:10882000761CB5F90C00B042F6DC1EE0B5F90C0080
:1088300000280BDA002603E03846FEF7C8FF761C56
:10884000B5F90C004042B042F6DC0DE0B5F90C0081
:10885000002809DD002603E03846FEF7C0FF761C3D
:10886000B5F90C00B042F7DC00BF3846FFF78EF8D0
:108870005D4908600846006800B984E7A87B0128C4
:1088800031D1B8F1000F2ED1002000905648006879
:108890006A461221C36954480068984708F079FD78
:1088A00060643846FFF796F910B99DF80000C8B922
:1088B0004D48006800220721C3694B48006898476B
:1088C00004F11C00FFF710FA00B15CE7002211462A
:1088D0004548006801F002F804F11C00FFF704FAB3
:1088E00000B150E7FDE0A87B01284BD1B8F1010FA2
:1088F00048D194F84C0000F001000028F2D1606CDF
:1089000008F052FDE18A8842ECD9002000903648F8
:1089100000686A461221C3693348006898479DF889
:10892000000068B1384609F0F1FB18BB3846FFF784
:1089300051F980F0010631463846FFF732F819E068
:108940002948006800220B21C3692748006898471E
:1089500004F11C00FFF7C8F900B114E7002204215C
:108960002148006800F0BAFF04F11C00FFF7BCF9D1
:1089700000B108E794F84C0020F00100401C84F896
:108980004C00AEE0A87B0028ACD1B8F1010FA9D112
:108990000090154800686A461221C36912480068B1
:1089A00098479DF80000F0B90F48006800220A219E
:1089B000C3690D480068984704F11C00FFF794F95B
:1089C00000B1E0E694F84C0000F0010028B9002264
:1089D00003210548006800F081FF04F11C00FFF747
:1089E00083F928B1CFE61BE0F0000020EC00002066
:1089F00000220621FB48006800F070FF04F11C0013
:108A0000FFF772F900B1BEE600220721F5480068C1
:108A100000F064FF04F11C00FFF766F9A0B3B2E6B2
:108A200097F85800C0F3400078B394F84C0000F079
:108A3000010018B1384609F069FB28B3E94800681D
:108A400000220A21C369E7480068984704F11C0026
:108A5000FFF74AF900B196E600220321E1480068D9
:108A600000F03CFF04F11C00FFF73EF900B18AE67C
:108A700000220621DB48006800F030FF04F11C00F2
:108A8000FFF732F910B17EE622E010E00022072164
:108A9000D448006800F022FF04F11C00FFF724F91D
:108AA00000B170E60A213846FFF717F810E09DF88C
:108AB000000068B197F85800C0F3400040B994F83E
:108AC0004C0000F0010018B901213846FEF769FF9B
:108AD0000021616494F84C0020F0010184F84C10EE
:108AE00000BF0020BF49086000BF4CE62DE9F041FF
:108AF00004460D46A87B012806D194F84C00C0F32B
:108B0000C00008B1BDE8F08194F84C00C0F3C0008B
:108B100080B194F84C0020F0080184F84C1000213A
:108B2000616494F84C0020F0010184F84C1000219D
:108B300020200155676D07B9E4E73846FEF726FFA8
:108B4000A84908600846006800B9DBE7D4F824802B
:108B5000696861622020065DA97B0155A87B012818
:108B600061D1002E5FD108F014FC606468680A28A7
:108B70001ED10A213846FEF7B0FF9A48006800224D
:108B80000721C36997480068984704F11C00FFF764
:108B9000ABF800B1B6E7002211469248006800F039
:108BA0009DFE04F11C00FFF79FF800283AD0A9E7CA
:108BB00068681B2810D11B213846FEF78EFF002263
:108BC00012218848006800F089FE04F11C00FFF7BC
:108BD0008BF80028EAD095E7686809280DD10021B4
:108BE0003846FEF7DEFE3846FEF7F9FD04F11C00BC
:108BF000FFF77AF80028D9D084E768680B280DD1F0
:108C000000213846FEF7CDFE3846FEF7E0FD04F1C0
:108C10001C00FFF769F80028C8D073E73846696878
:108C2000FEF75BFFD9E0A87B012872D1012EFCD1B1
:108C300094F84C0000F0010068BB606C08F0B4FBD5
:108C4000E18A884227D994F84C0020F00100401CAA
:108C500084F84C0068680A28E4D108F09AFBA06404
:108C60006048006800220B21C3695E48006898478D
:108C700004F11C00FFF738F800B143E7002204219B
:108C80005848006800F02AFE04F11C00FFF72CF899
:108C90000028C7D036E794F84C0000F00100002807
:108CA000C0D0A06C08F080FB218B8842BAD908F0B4
:108CB00070FBA06468680A281AD14A48006800223C
:108CC0000C21C36947480068984704F11C00FFF76E
:108CD0000BF800B116E7002205214248006800F0B9
:108CE000FDFD04F11C00FEF7FFFF002875D009E729
:108CF000686809280ED100213846FEF752FE384632
:108D0000FEF76DFD04F11C00FEF7EEFF002864D0B5
:108D1000F8E619E068680B280CD100213846FEF708
:108D200040FE3846FEF753FD04F11C00FEF7DCFF61
:108D300090B3E7E638466968FEF7CFFE04F11C0001
:108D4000FEF7D2FF40B3DDE6A87B28BB012E44D15D
:108D5000C5F8048068680A2837D1224800680022D4
:108D60000A21C3691F480068984704F11C00FEF7F8
:108D7000BBFF00B1C6E694F84C0000F0010060B9FA
:108D8000002203211748006800F0A8FD04F11C0030
:108D9000FEF7AAFF08B1B5E61FE000220621114840
:108DA000006800F09BFD04F11C00FEF79DFF00B180
:108DB000A8E6002207210B48006800F08FFD04F1AF
:108DC0001C00FEF791FF00B19CE60021616494F85D
:108DD0004C0020F0010184F84C100020014908608B
:108DE00000BF8FE6F000002070B504460D46206DF0
:108DF00090B1B4F92400B5F90010884205D1B4F956
:108E00002600B5F90210884206D0B5F90220B5F95E
:108E10000010206D00F02EFA298821846988618471
:108E2000207F012804D104F11C00FFF7B6FA03E00B
:108E300004F11C00FFF73CF8218CA184618CE184D3
:108E400070BD7FB504468949E0680860084600683F
:108E5000C06800B97FBD85480068FEF719FF8348E8
:108E6000006890F84C00C0F3800000B1F2E700BF4A
:108E700069467E48006808F060FA05467B4800684D
:108E8000FEF706FF00207A4908609DF80E0077493A
:108E90000968087775480068007F012807D108F045
:108EA00078FA72490968C968C1F860010EE06F4834
:108EB00000680078042809D1BDF80C0030B108F032
:108EC00068FA6A490968C968C1F8600167480068BA
:108ED0000078012805D1694664480068FFF784FFDF
:108EE0001FE0624800680078022805D169465F48A3
:108EF0000068FFF7FBFD14E05C4800680078042878
:108F000005D1694659480068FFF731FC09E0574828
:108F100000680078032804D1694654480068FFF7C8
:108F2000FBFB52480068FEF7B3FE002DA0D10020E5
:108F30004E4908604E49086000BF8BE74B48006807
:108F40007047014609B9002070470878FCE710B562
:108F5000044694F84C0020F0010184F84C1008F00D
:108F600018FAA06408F015FA606410BD00B97047E3
:108F7000CA4390F84C3062F3820380F84C3000BF53
:108F8000F5E770B504460D462078012800D070BD85
:108F90002565E068FEF7AFF906463146206D00F022
:108FA000CDFDB4F92220B4F92010206D00F062F953
:108FB00000BFECE70278022A02D00278042A00D12E
:108FC000416570470278032A00D1816570470278B5
:108FD000012A07D00278032A04D04FF0FF320A801A
:108FE0004A8003E0028C0A80428C4A807047014626
:108FF0000878022801D000207047486AFCE7014643
:1090000009B9002070470878012804D0087803289F
:1090100001D00020F6E791F84000C0F34000F1E7EE
:1090200018B900220A804A8070470278012A06D0C7
:109030000278032A03D000220A804A8003E0028DCE
:109040000A80428D4A8000BFEEE790F84C1021F074
:109050000801083180F84C107047014609B900201A
:109060007047086AFCE7024800687047EC0000207F
:10907000F000002010B5FE48007800B110BD09F0E6
:10908000B7F809F038FA08F058FAFEF7DBF902F001
:109090007AF801F021FC4FF4B271F64808F085FE31
:1090A0005C21F54808F081FEFEF7EDFD07F0E2FCDB
:1090B000012007F0A5F90120ED49087000BFDDE7A8
:1090C000014608687047014691F83000C0F300106F
:1090D000704710B50246134600BF1C462046FFF7F6
:1090E000EFFF0346002BF8D1204610BD2DE9F041DB
:1090F0000646306808B9354603E03046FFF7E9FF19
:109100000546DC4808F0B4FE044617E004F12400EC
:1091100008F0AEFE07460AE0AF4202D12046BDE8A5
:10912000F081394604F1240008F003FF0746002FC0
:10913000F2D12146CF4808F0FCFE0446002CE5D1D0
:109140000020ECE72DE9FC4706463046FFF7BBFF61
:1091500008B1BDE8FC873046FFF7BBFF0446204658
:10916000FFF7C4FF81464846FEF7A4F8A04209D0A5
:109170004846FEF7B5F8A04204D04846FEF7BBF8D3
:10918000A04244D13046FFF79BFF07464FF001084D
:10919000B6F9345006F11001684601F095FBBDF8B0
:1091A0000000401B00B2ADF80000BDF80200401BFB
:1091B00000B2ADF80200BDF80400284400B2ADF8DA
:1091C0000400BDF80600284400B2ADF8060013E024
:1091D00007F110026946684608F0C6FB8046B8F100
:1091E000000F00D10AE03846FFF76DFF00B1B0E78D
:1091F0003846FFF765FF0746002FE9D100BFB8F1F9
:10920000000F03D06946484601F0D5FE00BF00BFFD
:109210009FE72DE9F04107460D461646381D08F038
:1092200027FE044619E0208A284400B22082608A82
:10923000304401B26182A08A284401B2A182E08A4E
:10924000304401B2E182324629462046FFF7E1FF71
:109250002146381D08F06DFE0446002CE3D1BDE820
:10926000F08170B505460C4605F11001204601F06D
:109270002BFB70BDFEB504460E4617462568288AAE
:10928000304406B2688A384407B2208A301A00B2E5
:10929000ADF80800608A381A00B2ADF80A00BDF8CF
:1092A000080018B9BDF80A0000B9FEBD2046FFF756
:1092B00049FF69462046FFF7D4FF208ABDF8081011
:1092C000084400B22082608ABDF80A10084401B246
:1092D0006182A08ABDF80810084401B2A182E08A28
:1092E000BDF80A10084401B2E182BDF90A20BDF9B7
:1092F00008102046FFF78DFF6A4602212046E369E9
:109300009847224601212846EB6998472046FFF7F7
:1093100019FF00BFC9E710B502461046FFF7D0FE9F
:109320000446518A608A081A03B2184610BD10B567
:1093300002461046FFF7C4FE0446108A218A401AEE
:1093400003B2184610BD00B503461A460BE092F86A
:109350003000C0F3801010B192F8330000BD104609
:10936000FFF7AEFE0246002AF1D1FF20F6E70146E4
:10937000C86A70472DE9F0410546AE6AFEB92C680F
:1093800019E0A06AB0B1A06A007800F0010080B9CD
:109390002046FFF7ECFF07463846FEF7F7FAA042F3
:1093A00005D13846A16AFEF7E4FB064600E0A66A4E
:1093B00003E000BF2468002CE3D100BF00BFE86ACF
:1093C00048B1E86AFEF7E2FAA84204D13146E86AF9
:1093D000FEF7CFFB064606B9284E3046BDE8F081C1
:1093E0002DE9FC41064688461746022F52D106F168
:1093F0001001404608F065FB10B90020BDE8FC8173
:109400003046FFF7B7FF0546287AFB2801DA00202F
:10941000F4E7B5F9064047F61840844201D1002030
:10942000ECE769463046FFF71CFFBDF8000020441A
:1094300000B2ADF80000BDF80400001B00B2ADF8AA
:1094400004006946404608F03CFB08B90020D5E717
:1094500069463046FFF705FFBDF80200204400B220
:10946000ADF80200BDF80600001B00B208E00000E5
:10947000F4000020882E0020942E0020602C002074
:10948000ADF806006946404608F01BFB08B900200D
:10949000B4E710E07FB93046FFF76CFF0446304672
:1094A000FFF751FF05462B462246414606F11000C4
:1094B00006F08AFE00BF0120A0E70162704710B5E8
:1094C00004460020A086002205212046E369984733
:1094D0002046FFF737FE10BD024692F832000840E2
:1094E00008B1012070470020FCE72DE9F041054656
:1094F0000C4616464FF001082846FFF73BFF07468B
:10950000012C07D101212846FFF7E6FFC8B14FF033
:10951000000816E0052C08D1B7F91200B5F934108F
:1095200088420EDD788AA8860BE0042C03D12846F9
:10953000FFF7C5FF05E0062C03D13046F9A1016015
:1095400000BF4046BDE8F081C16170472DE9F041A0
:1095500006460D460024002E79D107F0B7FD80465F
:10956000B8F1000F02D10020BDE8F08108F124001D
:1095700008F054FC04460CB900BFFEE70CB900200B
:10958000F2E7002020604421201D08F00EFC00209E
:1095900020820021618207F0B0FD401E01B2A1824D
:1095A000002007F096FD401E01B2E1820020A08657
:1095B000002140200155A187E1870020A0634120C0
:1095C000005D20F00101412001550BF0DDFF074651
:1095D00017B13868A06201E0D448A062D44920469F
:1095E000FFF7B2FFD3492046FFF767FF002044F89A
:1095F000180F6061207E20F001002076207E20F090
:1096000002002076207E20F004002076207E20F0CC
:1096100008002076207E20F010002076207E20F0AA
:10962000200020760020A076207E20F040002076CA
:10963000FF20E076207E20F080002076607E20F003
:10964000FC0060760020E060183C6DE0FFE7301D14
:1096500008F0E4FB04460CB900BFFEE70CB900209B
:1096600082E726604421201D08F09FFB308A20827B
:10967000718A6182308A3C3001B2A182708A2830BE
:1096800001B2E1820020A086002140200155A1877F
:10969000E1870020A0634120005D20F0010141200E
:1096A00001550BF071FF074617B1B868A06201E0E1
:1096B000A148A0629E492046FFF746FF9D492046EB
:1096C000FFF7FBFE002044F8180F6061207E20F0B9
:1096D0000100401C2076207E20F002002076607E73
:1096E00020F00300C01C6076207E20F0040020766D
:1096F000207E20F008002076207E20F010002076CA
:10970000207E20F0200020760020A076FF20E0764A
:10971000207E20F040002076207E20F08000207601
:109720000020E060183C00BF002D76D005F110014C
:1097300004F1100001F0C8F8A88EA0864020415D19
:109740000155A98FA187E98FE187A86BA06341200C
:10975000405D4121095D60F300014120015555F84C
:10976000180F44F8180F287E217E60F3000121763F
:10977000287E4108207E61F341002076687E617E6C
:1097800060F301016176287E8108207E61F382000A
:109790002076287EC108207E61F3C3002076287ED3
:1097A0000109207E61F304102076287E4109207E85
:1097B00061F345102076287EC109207E61F3C71031
:1097C0002076287E8109207E61F386102076A87E8F
:1097D000A076E87EE07628692061183C6869183D2B
:1097E00018B12146E86AFEF735F82846FFF768FC0D
:1097F00070B16EB12846FFF78EFD07462846FFF789
:1098000096FD80463A4641462046FFF733FD04E088
:10981000002211462046FFF72DFD3EB122460121D0
:109820003046F36998472046FFF78CFC20469BE6BC
:109830000146424A106805E002688A4201D10122CD
:10984000027180680028F7D170472DE9FE4F064667
:109850000C4690461F46009400208DF804000290AC
:109860003648006810B13548006802903349C1F8A5
:1098700000D03348D0F800900760FFF75FFB054643
:109880002DB1A86818B141462846AA68904716B17C
:1098900041462046B0472A48C0F800902748006853
:1098A0008068264908609DF8040010B10020BDE8DA
:1098B000FE8F8CB194F83000C00968B1206858B1AF
:1098C0003A464146206800F009F88246BAF1010F95
:1098D00001D00020EBE700BF0120E8E72DE9F041CF
:1098E00004460D46164614B90120BDE8F081334602
:1098F0002A462146A069FFF7A8FF07463846F4E745
:109900002DE9F0470446201D08F0B2FA064620462D
:10991000FFF72DFD8046B8F1000F02D02046FDF77D
:10992000CEFF18E06C765F6F626A0000702B00203B
:10993000EB940008E19300089C2C0020F800002024
:10994000FC0000203146201D08F0F3FA074630469F
:10995000FFF7D6FF3E46002EF4D100221321204609
:10996000FFF7BCFF2046FFF763FF0021204607F00A
:109970001FFE002007F0D5FC05461BE0686BA042E7
:1099800002D0A86BA04202D12846FEF75DF9E86B31
:10999000A04201D10021E963686D404506D1FFF77F
:1099A00062FBA04202D12846FEF74EF9284607F096
:1099B000B8FC0546002DE1D12046FFF781FB81462A
:1099C000214609F1040008F0C4FA0022114620469D
:1099D000E3699847606A10B1606A08F09CFC204611
:1099E00008F099FCBDE8F0872DE9F04704462046D1
:1099F000FFF7A8FB2046FFF7BAFC8046B8F1000F3E
:109A000002D02046FDF75BFF0021204607F0D0FD85
:109A1000201D08F02DFA074608E03946201D08F001
:109A200088FA81463846FFF76BFF4F46002FF4D186
:109A3000002213212046FFF751FF2046FFF7F8FED2
:109A40002046FFF73DFB06464EB92046FFF74EFB8A
:109A5000824621460AF1240008F07BFA03E0214601
:109A6000301D08F076FA002007F05BFC05461BE08D
:109A7000686BA04202D0A86BA04202D12846FEF734
:109A8000E3F8E86BA04201D10021E963686D40452D
:109A900006D1FFF7E8FAA04202D12846FEF7D4F833
:109AA000284607F03EFC0546002DE1D10022114674
:109AB0002046E3699847606A10B1606A08F02BFCA1
:109AC000204608F028FC26B1002201213046F36927
:109AD00098470020BDE8F08710B504462046FFF700
:109AE00083FF10BD10B504462146FC4808F010F86D
:109AF00010BD70B504460D46002625B9201D08F09E
:109B0000B7F9064604E02946201D08F012FA064679
:109B1000304670BD70B5064600213046FFF7E9FFBC
:109B2000044608E021463046FFF7E3FF054620469D
:109B3000FFF75AFF2C46002CF4D170BDF8B504464F
:109B40000D46206800B9F8BD05B9FCE72046FFF7CF
:109B5000F9FA2046FFF7EBFBADF800002046FFF7CF
:109B6000DAFBADF8020026682168081D01232246B1
:109B7000291D08F04BFA2560BDF90220BDF900103F
:109B80002046FFF777FB002201213046F369984712
:109B9000224601212846EB6998472046FFF7D2FA72
:109BA00000BFD0E770B505462846FFF789FA04469E
:109BB000201D08F05DF9A84200D170BD2046FFF7D6
:109BC000C1FA01232A46211D201D08F01FFA2A464A
:109BD00001212046E36998472046FFF7B3FA00BF0A
:109BE000EBE770B505462846FFF76AFA0446201DE4
:109BF00008F0AAF9A84200D170BD2046FFF7A2FAEA
:109C000000232A46211D201D08F000FA2A460121C2
:109C10002046E36998472046FFF794FA00BFEBE738
:109C200070B504460D462046FFF775FB06463246E2
:109C300029462046FFF71EFB70BD70B505460C4651
:109C40002846FFF774FB0646224631462846FFF7B2
:109C500011FB70BD014600BFC88A4A8A801A401CA9
:109C600000B27047014600BF888A0A8A801A401CE9
:109C700000B270472DE9F04F87B004460D461646F6
:109C80001F46DDF840B02046FFF751FB80462046D6
:109C9000FFF741FB81461DB92046FFF711FA054643
:109CA000152E2ED2DFE806F00B2E324653607C9143
:109CB000A5C1CAE2FCFAF9F8F7F6F5F4F300284674
:109CC000FFF7D0FF019000EBD07043102046FFF764
:109CD000C9FF029000EBD070A3EB60000FFA80F890
:109CE0002846FFF7B7FF019000EBD07043102046E5
:109CF000FFF7B0FF029000EBD070A3EB60000FFA0B
:109D000080F95AE14FF00008C14656E12846FFF7B6
:109D1000A9FF019000EBD07043102046FFF7A2FF8F
:109D2000029000EBD070A3EB60000FFA80F84FF0C8
:109D3000000942E12846FFF795FF03462046FFF75A
:109D400091FF181A0FFA80F84FF0000935E14FF033
:109D500000082846FFF77EFF03462046FFF77AFFFC
:109D6000181A0FFA80F928E12846FFF77BFF0190C7
:109D700000EBD07043102046FFF774FF029000EB19
:109D8000D070A3EB60000FFA80F82846FFF762FF5F
:109D900003462046FFF75EFF181A0FFA80F90CE120
:109DA0002846FFF75FFF03462046FFF75BFF181AC0
:109DB0000FFA80F82846FFF74DFF03462046FFF7CD
:109DC00049FF181A0FFA80F9F7E04FF0000828460B
:109DD000FFF740FF019000EBD07043102046FFF7E3
:109DE00039FF029000EBD070A3EB60000FFA80F90E
:109DF000E3E02846FFF736FF03462046FFF732FF31
:109E0000181A0FFA80F82846FFF724FF019000EB9C
:109E1000D07043102046FFF71DFF029000EBD0707A
:109E2000A3EB60000FFA80F9C7E04FF0000820466E
:109E3000FFF710FF40420FFA80F9BEE02846FFF717
:109E400011FF019000EBD07043102046FFF70AFF8E
:109E5000029000EBD070A3EB60000FFA80F8204670
:109E6000FFF7F8FE40420FFA80F9A6E02846FFF718
:109E7000F9FE03462046FFF7F5FE181A0FFA80F8A0
:109E80002046FFF7E7FE40420FFA80F995E085E0B3
:109E90006EE066E054E03BE031E021E007E0FFE700
:109EA0004FF000082846FFF7D5FE814685E028469A
:109EB000FFF7D8FE019000EBD07043102046FFF76B
:109EC000D1FE029000EBD070A3EB60000FFA80F897
:109ED0002846FFF7BFFE81466FE00000D99A0008D0
:109EE0002846FFF7BFFE03462046FFF7BBFE181AC1
:109EF0000FFA80F82846FFF7ADFE81465DE0204668
:109F0000FFF7B0FE40420FFA80F84FF0000954E02E
:109F10002046FFF7A7FE40420FFA80F82846FFF7D9
:109F200099FE019000EBD07043102046FFF792FE9F
:109F3000029000EBD070A3EB60000FFA80F93CE0D8
:109F40002046FFF78FFE40420FFA80F82846FFF7C1
:109F500081FE03462046FFF77DFE181A0FFA80F9AE
:109F60002BE02846FFF77EFE80464FF0000924E0F4
:109F70002846FFF777FE80462846FFF76BFE0190E4
:109F800000EBD07043102046FFF764FE029000EB18
:109F9000D070A3EB60000FFA80F90EE02846FFF7BF
:109FA00061FE80462846FFF755FE03462046FFF730
:109FB00051FE181A0FFA80F900BF00BF2046FFF7C4
:109FC0007FF88246B5F910000690B5F912000590A9
:109FD000BAF910000490BAF91200039006983844B8
:109FE00040440FFA80F80598584448440FFA80F925
:109FF0000498A8EB00000FFA80F80398A9EB000082
:10A000000FFA80F94A4641462046FFF733F94020CF
:10A010000655A787A4F83EB0A5634120005D20F057
:10A0200002014120015507B0BDE8F08F2DE9F04F46
:10A0300085B006460F46904699463046FFF777F9B9
:10A0400082463046FFF767F983463046FFF70AFE3F
:10A05000034600EBD37044103046FFF7FBFD034688
:10A0600000EBD37045101FB93046FFF729F80746BB
:10A07000B8F1150F20D2DFE808F00B2027353F4953
:10A080005A6775868D9BA5AFC0CDD4E2EFF9EC0081
:10A090003846FFF7E7FD034600EBD370C4EB6000E2
:10A0A0000FFA80FA3846FFF7D5FD034600EBD37070
:10A0B000C5EB60000FFA80FBF6E060420FFA80FA11
:10A0C00068420FFA80FBEFE03846FFF7CBFD03460E
:10A0D00000EBD370C4EB60000FFA80FA68420FFA0D
:10A0E00080FBE1E03846FFF7BDFD001B0FFA80FA68
:10A0F00068420FFA80FBD7E060420FFA80FA3846D8
:10A10000FFF7A8FD401B0FFA80FBCDE03846FFF7B4
:10A11000A9FD034600EBD370C4EB60000FFA80FA90
:10A120003846FFF797FD401B0FFA80FBBCE038462E
:10A13000FFF798FD001B0FFA80FA3846FFF78AFDFB
:10A14000401B0FFA80FBAFE060420FFA80FA3846FE
:10A15000FFF780FD034600EBD370C5EB60000FFAFC
:10A1600080FBA1E03846FFF77DFD001B0FFA80FA67
:10A170003846FFF76FFD034600EBD370C5EB600078
:10A180000FFA80FB90E060420FFA80FA68420FFA03
:10A1900080FB89E03846FFF765FD034600EBD3708E
:10A1A000C4EB60000FFA80FA68420FFA80FB7BE094
:10A1B0003846FFF757FD001B0FFA80FA68420FFA86
:10A1C00080FB71E060420FFA80FA3846FFF742FDEB
:10A1D000401B0FFA80FB67E03846FFF743FD03465C
:10A1E00000EBD370C4EB60000FFA80FA3846FFF73B
:10A1F00031FD401B0FFA80FB56E03846FFF732FD79
:10A20000001B0FFA80FA3846FFF724FD401B0FFAB7
:10A2100080FB49E060420FFA80FA68420FFA80FB47
:10A2200042E060420FFA80FA3846FFF713FD03461A
:10A2300000EBD370C5EB60000FFA80FB34E06042A6
:10A240000FFA80FA3846FFF705FD401B0FFA80FB36
:10A250002AE01CE00AE0FFE73846FFF703FD001B99
:10A260000FFA80FA68420FFA80FB1DE03846FFF7CC
:10A27000F9FC001B0FFA80FA3846FFF7EBFC0346A7
:10A2800000EBD370C5EB60000FFA80FB0CE03846A2
:10A29000FFF7E8FC001B0FFA80FA3846FFF7DAFCFC
:10A2A000401B0FFA80FB00BF00BF3046FEF708FFDF
:10A2B0000490B7F910000390B7F9120002900498C7
:10A2C000B0F9100001900498B0F9120000900398C2
:10A2D000484450440FFA80FA0E99029808445844B2
:10A2E0000FFA80FB0198AAEB00000FFA80FA0098A1
:10A2F000ABEB00000FFA80FB5A4651463046FEF7A2
:10A30000B9FF86F84080A6F83C900E98F087B763B6
:10A310004120805D20F00200801C4121885505B05D
:10A32000BDE8F08F38B504464120005DC0F3400021
:10A3300058B1B4F93E000090B4F93C304020025DC1
:10A340002046A16BFFF772FE0AE0B4F93E000090D0
:10A35000B4F93C304020025D2046A16BFFF78AFC37
:10A3600038BD2DE9FC4104460F4690462046FFF7D4
:10A3700079FCB84206D12046FFF76CFC404501D17C
:10A38000BDE8FC812046FEF7DDFE69462046FEF76B
:10A3900068FF208A3844401E01B2A182608A40448E
:10A3A000401E01B2E1826A4602212046E3699847D5
:10A3B0002046FEF785FE064626B12246012130469C
:10A3C000F3699847201D07F053FD054609E0002278
:10A3D00003212846EB6998472946201D07F0A9FD6F
:10A3E0000546002DF3D12046FEF7ACFE4120005D6E
:10A3F00000F0010010B12046FFF794FF00BFBFE757
:10A4000070B504460D462046FFF724FC064632464A
:10A4100029462046FFF7A5FF70BD70B505460C46DE
:10A420002846FFF71FFC0646224631462846FFF71E
:10A4300098FF70BD4122125C61F3000241231A545F
:10A44000704710B5029C10BD10B504462046FEF7BB
:10A4500079FE002204212046E36998472046FEF752
:10A4600071FE10BD70B5054600212846FFF741FB7F
:10A47000044615E0A06A30B92046FFF7F3FF2046F6
:10A48000FFF7E2FF07E0A06A007800F0010010B1DA
:10A490002046FFF7E7FF21462846FFF72AFB044640
:10A4A000002CE7D170BD70B504460D46A56220466C
:10A4B000FFF7D8FF2046FFF7C7FF70BD70B5054610
:10A4C0000E46301D07F0D4FC044612E0A06AA842F4
:10A4D00000D02DB92046FFF7C5FF2046FFF7B4FF97
:10A4E00021462846FFF7EAFF2146301D07F021FDEF
:10A4F0000446002CEAD170BD70B50646002006F077
:10A5000075FE04461DE004F1240007F0B1FC054689
:10A5100010E0A86AB04200D016B92846FFF794FFB1
:10A5200029463046FFF7CAFF294604F1240007F008
:10A5300000FD0546002DECD1204606F057FE0446EE
:10A5400000BF002CDFD170BD70B504460D4694F8F5
:10A550003000C0F3001010B92046FEF7F3FD14F8E8
:10A56000300F65F30410207014F83009C0F30010A8
:10A5700010B92046FEF7E6FD2046FEF7A1FD06468F
:10A58000224601213046F369984770BDCA43D24341
:10A5900090F8303062F3000380F830307047CA43DF
:10A5A000D24390F8303062F3451380F83030704772
:10A5B00030B504460D46012D02D12046FFF7E6FFD7
:10A5C000E843C04394F8301060F3410184F8301040
:10A5D00030BD30B504460D4614F8310F65F3010067
:10A5E000207014F8310900F0030018B10121204651
:10A5F000FFF7DEFF30BDCA43D24390F8303062F33C
:10A60000820380F830307047CA43D24390F830302C
:10A6100062F3C30380F830307047CA43D24390F8E6
:10A62000303062F3C71380F83030704790F8302034
:10A6300061F3861280F83020704770B504460D46ED
:10A6400084F833502046FEF77DFD70BD90F832202F
:10A650000A4380F832207047CA43D1B290F83220C2
:10A660000A4080F83220704781617047994800683D
:10A67000704770B504460D461646E06920B1324673
:10A6800029462046E369984770BD70B504460D46DB
:10A690002946606A07F076FE6062606A70BD70B538
:10A6A00004460D46002625B9201D07F04DFC064640
:10A6B00004E02946201D07F0D1FB0646304670BD58
:10A6C00070B504460026201D07F0D2FB054606E0C3
:10A6D000701C86B22946201D07F02BFC0546002D74
:10A6E000F6D1304670BD70B506460025301D07F026
:10A6F000BFFB04460BE0681C85B22046FFF7F3FF62
:10A70000284485B22146301D07F013FC0446002C76
:10A71000F1D1284670BD70B506460C463046FEF7AE
:10A7200029FE0546A87B00F0040020B12188A889F5
:10A73000084400B22080A87B00F0080020B1A18866
:10A74000A889081A00B2A080A87B00F0020020B1FE
:10A750006188A889084400B26080A87B00F00100ED
:10A7600020B1E188A889081A00B2E08070BD70B5F8
:10A7700005462846FEF7FEFD04462846FFF772FA16
:10A780000146608B091AA08B081A00B270BD70B523
:10A7900005462846FEF7EEFD04462846FFF75AFA1E
:10A7A000E18A411A208B081A00B270BD014641208F
:10A7B000405C00F0010070470146002070470146F0
:10A7C0000020704701460020704701460020704776
:10A7D0000146B1F934007047014691F8300000F0AD
:10A7E00001007047014691F83000C0F340107047F7
:10A7F000014691F83000C0F340007047014691F8DF
:10A80000310000F003007047014691F83000C0F3BA
:10A8100080007047014691F83000C0F3C0007047D7
:10A82000014691F83000C0097047014691F83000A8
:10A83000C0F380107047014691F83200704701461E
:10A84000C86970470146086A7047014688697047C1
:10A850000146486A7047F0B589B007460E46202188
:10A86000304613F0FAF9202101A813F0F6F901AAF5
:10A8700006213846FB699847002406E001A850F8F5
:10A88000240000B903E0601CC4B2082CF6DB00BF52
:10A89000002508E0601E401B01A951F8200046F881
:10A8A0002500681CC5B2A542F4DB09B0F0BD10B5A7
:10A8B0000446E06A30B1E06AFDF768F8A04201D1D1
:10A8C000012010BD0020FCE70A6802604A6842606F
:10A8D00070470000FC0000207047FE480068704789
:10A8E00070B5FC48006806F08DFC0446F948006825
:10A8F00006F0A3FC28B100BFA06900F00100002809
:10A90000FAD1A06920F00100401CA061FFF7E5FF2B
:10A910000546E86828B1A26804F110012846EB68F2
:10A920009847206850B1606840B12168A0688842AB
:10A9300002D16068A06001E02068A06070BD2DE9D0
:10A94000F0418AB00546884695F83000C0F3001003
:10A9500010B10AB0BDE8F081B5F9344004A9284629
:10A96000FEF77FFCBDF81000001B00B2ADF8100030
:10A97000BDF81200001B00B2ADF81200BDF81400C3
:10A98000204400B2ADF81400BDF81600204400B217
:10A99000ADF8160004AA414606A806F0E5FF0646F3
:10A9A000002E4AD0002206A928462B6A984704A9FF
:10A9B0002846FEF756FC04AA414608A806F0D4FF34
:10A9C0000646AEB3281D07F0BFFA07462DE06946DC
:10A9D0003846FEF746FCB7F93440BDF80000001BCE
:10A9E00000B2ADF80000BDF80200001B00B2ADF8E7
:10A9F0000200BDF80400204400B2ADF80400BDF828
:10AA00000600204400B2ADF806006A4608A902A874
:10AA100006F0AAFF06461EB102A93846FFF78FFFCF
:10AA20003946281D07F01AFA0746002FCFD100BF7C
:10AA3000012206A928462B6A984700BF89E72DE91D
:10AA4000F0410546884625B9A2480068FCF732FC6B
:10AA5000054641462846FFF772FF2F462846FEF777
:10AA60002FFB04461BE03946201D07F0F7F9064688
:10AA700008E041463046FFF762FF3146201D07F0EF
:10AA8000EDF90646002EF4D1012241462046236A04
:10AA9000984727462046FEF713FB044600BF002CCC
:10AAA000E1D1BDE8F0812DE9F04106460C460025D4
:10AAB00004F11001304607F004F800282FD094F874
:10AAC0003000C0F3001050BB201D07F0D1F907463D
:10AAD0000BE039463046FFF7E6FF054605B106E0D4
:10AAE0003946201D07F025FA0746002FF1D100BF97
:10AAF000A5B92046FEF73EFC804698F80800FF28DE
:10AB00000BD1022231462046236A984728B12046BD
:10AB1000FEF719FCFF2800D1254600BF00BF2846DC
:10AB2000BDE8F0812DE9FC4104466A48006806F062
:10AB300069FB05466748006806F07FFB28B900BF3F
:10AB4000A86900F001000028FAD105F110022146A1
:10AB5000684606F009FF5F480068FCF7ABFB074654
:10AB600039466846FFF79FFF064669463046FFF7BD
:10AB700066FF58480068FCF7B3FB07466946FFF7D5
:10AB80005EFF54480068FCF7B6FB07466946FFF7CE
:10AB900056FF5048006806F05BFB08B9FFF7A0FEBF
:10ABA000BDE8FC812DE9FE4F05464A48006806F0E5
:10ABB0004FFBD0B14748006806F024FB0446002054
:10ABC00020824448006806F098FA401E01B2A18233
:10ABD000002161823F48006806F07BFA401E01B206
:10ABE000E1822846FFF79EFF88E03A48006806F0B9
:10ABF00009FB0446284600F055FA0290284600F06A
:10AC000058FA82463348006806F063FAB5F9061030
:10AC1000884206DC2F48006806F05BFA401E00B24E
:10AC200001E0B5F906000746E1680298B1FBF0F6CD
:10AC3000564500DD564627480068006950B300209D
:10AC4000ADF80000ADF80400ADF80200701E0FFA78
:10AC500080F900BFADF806901E4800686946026999
:10AC60001C4800689047684600F023FAB04200DCB8
:10AC700006E0A9F101000FFA80F9B9F1000FE9D15E
:10AC800000BFB9F1000F01D1BDE8FE8FBDF906008C
:10AC9000461C00BF4FF0000BB5F9028018E0288871
:10ACA0002082A988A182A4F8128008EB0600401E29
:10ACB00001B2E182B4F91600B84200DDE782B4F9CE
:10ACC00016B02846FFF72EFF08EB06000FFA80F8B3
:10ACD00002E000000401002008EB0600401EB8421C
:10ACE000DDDD5F4509D028882082A988A182A4F8EB
:10ACF0001280E7822846FFF715FF00BF00BFC3E7B9
:10AD000010B50020EE49086000241DE0ED48006801
:10AD100000F59E70005DB0B9EA4909683C3101EB6D
:10AD2000C400FFF73FFFE7480068806958B1E54974
:10AD300009683C3101EBC40006F005FEE0490968F2
:10AD40000844DF490860641CDE480068B0F85C0114
:10AD5000C0F30900A042D9D810BD2DE9FC4100255F
:10AD60005CE0D848006800F59E70405D00B154E09A
:10AD7000002449E0D348006800F59E70005D08B9E2
:10AD8000A54200D13FE0CF4A12683C3202EBC40139
:10AD9000CC4A12683C3202EBC50006F075FE00B9E1
:10ADA00031E0C84800683C3000EBC402C548006888
:10ADB0003C3000EBC501684606F017FE684606F019
:10ADC000C2FD0646BF4909683C3101EBC50006F0EB
:10ADD000BAFD0746BB4909683C3101EBC40006F0E7
:10ADE000B2FD384486420DD2B64909683C3101EBC8
:10ADF000C500694600F051F90121B248006800F52C
:10AE00009E70015500BF641CAE480068B0F85C013C
:10AE1000C0F30900A042ADD800BF6D1CA94800686E
:10AE2000B0F85C01C0F30900A8429AD8BDE8FC81E3
:10AE30002DE9FC5F804606F0ACFA0190A149D8F8F4
:10AE40000C000860FFF789FFFFF75AFF9D48006874
:10AE5000B0F85C01C0F3090000287DD09948006873
:10AE600006F0F6F9002865D09648006806F0CAF9A1
:10AE70000546FFF735FD00BFA86900F00100002876
:10AE8000FAD1D5F808902968A868884201D1686885
:10AE900000E0286800908B48006806F02EF906460E
:10AEA00000243EE08748006800F59E70005DB0BB5E
:10AEB000844800683C3030F93410824800683C30E7
:10AEC00000EBC400B0F9020006FB001047007D490A
:10AED00009683C3101EBC40000F0E4F84FEA400B94
:10AEE000784800683C3000EBC400B0F902A00CE0E8
:10AEF000009AD11909EB07005A4612F08EFD07EBB4
:10AF000046070AF101000FFA80FA6E4800683C30EB
:10AF100000EBC400B0F906005045E9DA00BF601C40
:10AF200084B268480068B0F85C01C0F30900A04230
:10AF3000B8DC00BF4FF48071624800683C3012F00A
:10AF40006AFE20215F48006800F59E7012F085FEC1
:10AF500000205C49096800E012E0C1F85C01594832
:10AF60000068806960B1019806F01EFA04465548F1
:10AF70000068836952482146026852480068984731
:10AF800000F012FEBDE8FC9F70B504461CB1206ABB
:10AF9000FFF74EFF0EE0002006F028F9054606E018
:10AFA000286AFFF745FF284606F020F90546002DE0
:10AFB000F6D100BF70BD2DE9FF4104460F4614B91C
:10AFC00006F084F804460CB9BDE8FF811FB90020E3
:10AFD000C4F85C01F8E70020ADF80800ADF80A00FD
:10AFE000204606F08AF8401E00B2ADF80C0020465C
:10AFF00006F06FF8401E00B2ADF80E0002AA394606
:10B00000684606F0B1FC0646F6B3206918B16946F9
:10B0100020462269904700250AE004F13C0000EB3D
:10B02000C501684606F04DFD00B1CDE7681C85B24C
:10B03000B4F85C01C0F30900A842EEDCB4F85C018E
:10B04000C0F3090020280BDAB4F85C11C1F309023F
:10B0500004F13C0101EBC200694600F01EF80DE06E
:10B060000020C4F85C01B4F85C11C1F3090204F1DA
:10B070003C0101EBC20002A900F00FF8B4F85C013A
:10B08000C0F30900401C00E002E0C4F85C0100BF0E
:10B0900000BF99E70B49086070470A6802604A6878
:10B0A00042607047014688880A88801A401C00B2B6
:10B0B00070470146C8884A88801A401C00B2704711
:10B0C000000100200401002007B581B0BDF8080090
:10B0D000C00AC2F1FF014843BDF80410C90A01FBD0
:10B0E0000200010ABDF8000061F3CF200090BDF816
:10B0F0000800C0F34510C2F1FF014843BDF8041039
:10B10000C1F3451101FB0200010ABDF8000061F323
:10B110004A100090BDF8080000F01F00C2F1FF01C6
:10B120004843BDF8041001F01F0101FB0200010AB1
:10B13000BDF8000061F304000090BDF8001008465F
:10B1400004B000BD18B50346D408BDF8000064F390
:10B15000040000908C08BDF8000064F34A100090D1
:10B16000DC08BDF8000064F3CF200090BDF800407B
:10B17000204618BD70B504460D463C22294620469F
:10B1800012F0D2FC70BD00B589B00020FE490870F5
:10B19000FF21FD48017200200890FB48BDF82010F7
:10B1A000418000200790F848BDF81C1081800021E4
:10B1B000C18041838183C18201830321C183002037
:10B1C0000690F148BDF818104181FF21C17300219C
:10B1D00081810F218173ED4800680590EA48BDF830
:10B1E000141001820121017500214182FF2180F8A4
:10B1F0002C10302211461046FFF7A4FF0190E248C0
:10B20000BDF804100184D82296215520FFF79AFF3B
:10B210000190DD48BDF804104184DD494162002100
:10B22000018502214185FF2180F83310202211463B
:10B230001046FFF787FF0190D348BDF80410018640
:10B24000002180F83210FF2180F8381020221146AA
:10B250001046FFF777FF0190CB48BDF804108186B8
:10B260000221C186002180F839100146C948FFF744
:10B2700081FF0321C74841838183C1820183014645
:10B28000C548FFF777FFF02211461046FFF75AFF37
:10B290000190C148BDF804100184F0221146104607
:10B2A000FFF750FF0190BC48BDF804100186F02262
:10B2B00011461046FFF746FF0190B748BDF804104D
:10B2C0008186D82296215520FFF73CFF0190B24895
:10B2D000BDF804104180014649888180AD49AF48DE
:10B2E000FFF748FF202211461046FFF72BFF019081
:10B2F000AA48BDF804100184202211461046FFF729
:10B3000021FF0190A548BDF80410018620221146B6
:10B310001046FFF717FF0190A048BDF80410818682
:10B320009A48001D006804909C48BDF810104180A8
:10B3300096480830006803909848BDF80C1081804A
:10B340000421C180402211461046FFF7FBFE019008
:10B350009248BDF804104181012181814C21C173C3
:10B3600001468F48FFF706FFE02211461046FFF71F
:10B37000E9FE01908A48BDF804100184E0221146DC
:10B380001046FFF7DFFE01908548BDF804100186E6
:10B39000C02211461046FFF7D5FE01908048BDF847
:10B3A00004108186C7229A216B20FFF7CBFE019003
:10B3B0007B48BDF8041041808B2259212B20FFF7D8
:10B3C000C1FE01907648BDF80410818042222C21F4
:10B3D0001520FFF7B7FE01907148BDF804104181B8
:10B3E0006C497048FFF7C6FE01206E4908700021C5
:10B3F0006C488181017201466B48FFF7BBFE00215A
:10B40000694841838183C182018301466748FFF710
:10B41000B1FE00216548C1835E496548FFF7AAFE79
:10B42000D022A2217620FFF78DFE01906048BDF862
:10B43000041041805D223A211920FFF783FE01901C
:10B440005B48BDF8041081800421C1800F21418335
:10B4500081830A21C18201830621C1832822192107
:10B460000B20FFF76FFE01905148BDF80410418199
:10B4700001218181B221C17344480C3000680290DF
:10B480004B48BDF80810018200214182FF2211467D
:10B490001046FFF757FE01904548BDF8041001849F
:10B4A000FF2211461046FFF74DFE01904048BDF8BF
:10B4B0000410018601463F48FFF75CFE942262219A
:10B4C0003320FFF73FFE01903A48BDF80410418059
:10B4D0003C2226211020FFF735FE01903548BDF8AB
:10B4E00004108180C622B521A420FFF72BFE019015
:10B4F0003048BDF804100184C622B521A420FFF70E
:10B5000021FE01902B48BDF804100186C622B5210A
:10B51000A420FFF717FE01902648BDF8041081868D
:10B5200023492548FFF726FE222211210A20FFF792
:10B5300009FE01902048BDF804104180902262214C
:10B540003720FFF7FFFD01901B48BDF804108180F4
:10B550000D2207210120FFF7F5FD01901648BDF8E7
:10B5600004104181F422DD21C820FFF7EBFD01909A
:10B570001148BDF804100184F422DD21C820FFF732
:10B58000E1FD01900C4819E0702B002050090208E1
:10B590004C010020602C00209C2C0020D82C002086
:10B5A000142D0020AC2B0020E82B0020242C0020A0
:10B5B000502D00208C2D0020C82D0020BDF8041037
:10B5C0000186F422DD21C820FFF7BCFD0190FE4872
:10B5D000BDF8041081860146FC48FFF7CBFD272209
:10B5E00014210220FFF7AEFD0190F848BDF80410C9
:10B5F000418070224C212B20FFF7A4FD0190F348DD
:10B60000BDF804108180C622B521A420FFF79AFD61
:10B610000190EE48BDF804100184C622B521A42093
:10B62000FFF790FD0190E948BDF804100186C6229D
:10B63000B521A420FFF786FD0190E448BDF8041071
:10B640008186E349E348FFF795FDD822114610466D
:10B65000FFF778FD0190DF48BDF804104180D82243
:10B6600011461046FFF76EFD0190DA48BDF8041050
:10B670008180902211461046FFF764FD0190D54865
:10B68000BDF804104181702211461046FFF75AFDA3
:10B690000190D048BDF80410018470221146104674
:10B6A000FFF750FD0190CB48BDF8041001867022D1
:10B6B00011461046FFF746FD0190C648BDF804103C
:10B6C000818609B000BD2DE9FE4304460E461546AD
:10B6D0001F46217A307A814208D0317A207A081ABE
:10B6E0007843217A01EB2020287201E0217A297227
:10B6F000B4F90610B6F9060081420BD0B6F906106F
:10B70000B4F90600081A7843E18801EB202001B261
:10B71000E98001E0E188E980B4F90C10B6F90C0089
:10B7200081420BD0B6F90C10B4F90C00091A794318
:10B7300080B200EB212001B2A98101E0A189A98199
:10B74000E17BF07B814207D0F17BE07B091A7943F2
:10B7500000EB2120E87301E0E17BE973B4F91210FA
:10B76000B6F9120081420BD0B6F91210B4F91200EA
:10B77000091A794380B200EB212001B2698201E00D
:10B78000618A6982B4F91A10B6F91A0081420BD0A5
:10B79000B6F91A10B4F91A00091A794380B200EB0D
:10B7A000212001B2698301E0618B6983B4F91C1027
:10B7B000B6F91C0081420BD0B6F91C10B4F91C007C
:10B7C000091A794380B200EB212001B2A98301E07C
:10B7D000A18BA983B4F91610B6F9160081420BD0DB
:10B7E000B6F91610B4F91600081A7843E18A01EB8D
:10B7F000202001B2E98201E0E18AE982B4F918105F
:10B80000B6F9180081420BD0B6F91810B4F9180037
:10B81000091A794380B200EB212001B2298301E0AB
:10B82000218B2983B4F91E10B6F91E0081420BD07A
:10B83000B6F91E10B4F91E00091A794380B200EB64
:10B84000212001B2E98301E0E18BE983B4F92A10F8
:10B85000B6F92A0081420BD0B6F92A10B4F92A00B1
:10B86000081A7843618D01EB202001B2698501E05F
:10B87000618D6985B4F92810B6F9280081420BD092
:10B88000B6F92810B4F92800081A7843218D01EB85
:10B89000202001B2298501E0218D29852C20015D20
:10B8A000805D81420CD02C20815D005D081A7843B8
:10B8B0002C21095D01EB2020C1B22C20415502E072
:10B8C0002C20015D4155B4F93610B6F9360081429D
:10B8D0000BD0B6F93610B4F93600081A7843E18E69
:10B8E00001EB202001B2E98601E0E18EE9863820F3
:10B8F000015D805D81420CD03820815D005D081AB9
:10B9000078433821095D01EB2020C1B23820415530
:10B9100002E03820015D41553220015D805D8142A9
:10B920000CD03220815D005D081A78433221095D18
:10B9300001EB2020C1B23220415502E03220015DEE
:10B9400041553320015D805D81420CD03320815D03
:10B95000005D081A78433321095D01EB2020C1B254
:10B960003320415502E03320015D4155B7F5807F1A
:10B9700001D1FF2000E0384600F0FF086088019008
:10B980007088424600900199FFF79EFB0290BDF837
:10B9900008006880A0880190B08842460090019914
:10B9A000FFF792FB0290A81CBDF80810A9806089DF
:10B9B00001907089424600900199FFF785FB029043
:10B9C000A81CBDF8081007E0C82D0020042E002098
:10B9D000502D0020402E00206981208A0190308A5D
:10B9E000424600900199FFF76FFB0290A81CBDF83A
:10B9F000081029824246216A306AFFF765FB0290EF
:10BA0000BDF808002884208E0190308E42460090B8
:10BA10000199FFF759FB0290BDF808002886A08E17
:10BA20000190B08E424600900199FFF74DFB0290C5
:10BA3000BDF80800A886802F10DAA17BA9732078B2
:10BA400000F001002870616A6962217D2975392042
:10BA5000005D00F00100392148550FE0B17BA9736A
:10BA6000307800F001002870716A6962317D2975B3
:10BA70003920805D00F0010039214855BDE8FE8382
:10BA800070B505462C68E06F10B12846E16F884715
:10BA9000204606F040FC70BD2DE9F04104460E46FC
:10BAA000254604F13C07D4F87880B3B242463946C3
:10BAB0002846FFF708FEA06FFEF71EFDBDE8F081E7
:10BAC00070B50446204605F062FD002020614FF469
:10BAD000807060611B4860601B48A0601B48E0608C
:10BAE000802006F0E8FB05460DB900BFFEE705B96A
:10BAF00070BD0020E867A86715492846FFF73AFBA4
:10BB0000134905F13C00FFF735FB256000BFEFE767
:10BB10002DE9F04105460E46174698462C68A66763
:10BB20003C223946204611F0FFFF3C22414604F1F9
:10BB30003C0011F0F9FF3C223946A06F11F0F4FFF0
:10BB4000BDE8F08199BA00085B15010881BA0008C8
:10BB5000602C002010B5044654480068844202D886
:10BB60005348006810BD514804605148006860B9EE
:10BB7000204606F0A0FB4E4908600846006808B958
:10BB800000BFFEE74A480068ECE7214648480068E5
:10BB900006F0F8FB464908600846006808B900BF8F
:10BBA000FEE743480068DDE710B54148006840B152
:10BBB0003F48006806F0AFFB00203D4908603B4964
:10BBC000086010BD10B503460BB9002010BD082B4E
:10BBD00007DA581E374C54F82000405C5043000AE6
:10BBE000F4E7012000EB410050435C0090FBF4F0CF
:10BBF000C0B2EBE72DE9F84F82460E4614461F46C9
:10BC0000DDF82C804FF0000B002C03DA4FF0010B15
:10BC1000604204B2002517E0424629462046FFF75D
:10BC2000D1FF8146BBF1000F03D0A8EB090000F063
:10BC3000FF09701901B2CDF800903A4650460A9BB0
:10BC400000F078F8681C05B2A542E5DBBDE8F88F86
:10BC50002DE9F84F06468A4614461F46DDF82C802B
:10BC60004FF0000B002C03DA4FF0010B604204B2DE
:10BC7000002517E0424629462046FFF7A3FF8146EC
:10BC8000BBF1000F03D0A8EB090000F0FF09711908
:10BC900008B2CDF800903A4651460A9B00F04AF8A7
:10BCA000681C05B2A542E5DBBDE8F88F080100205D
:10BCB000A40100200C01002007B581B0BDF80800E8
:10BCC000C00AC2F1FF014843BDF80410C90A01FBD4
:10BCD0000200010ABDF8000061F3CF200090BDF81A
:10BCE0000800C0F34510C2F1FF014843BDF804103D
:10BCF000C1F3451101FB0200010ABDF8000061F328
:10BD00004A100090BDF8080000F01F00C2F1FF01CA
:10BD10004843BDF8041001F01F0101FB0200010AB5
:10BD2000BDF8000061F304000090BDF80010084663
:10BD300004B000BD2DE9FF4F83B004460D46174601
:10BD4000DDF84080B8F1100F02DA07B0BDE8F08FDF
:10BD5000B8F1FB0F01DD4FF0FF08B7F90000A0427A
:10BD60000BDCB7F90400A04207DBB7F90200A842D8
:10BD700003DCB7F90600A84200DAE6E7FEF7ADFDFE
:10BD80008146484605F03EFA064606F1100000F0EE
:10BD90008EFC8246308A201A04B2708A281A05B2B4
:10BDA000D9F8140078B1CDF80880BDF81800ADF8C6
:10BDB00004000095B16823460FFA8AF24846D9F884
:10BDC00014C0E0471FE000200290D6F808B005FB41
:10BDD0000A400BEB400B0298A0B9B8F1FF0F04D159
:10BDE000BDF81800ABF800000CE0BBF800004246BC
:10BDF000014600900698FFF75FFF0190BDF8040030
:10BE0000ABF8000000BF00BF9FE72DE9FF4F83B0F4
:10BE1000064688461446DDF84090FEF75EFD8246F1
:10BE2000DAF8140000B3B4F9005018E0B4F9027065
:10BE30000FE0CDF80890BDF81800ADF804000097A9
:10BE40002B46424631465046DAF814C0E047781C8B
:10BE500007B2B4F90600B842EBDA681C05B2B4F9CF
:10BE60000400A842E2DA71E0B4F9020000FB08F035
:10BE700006EB4006B9F1FF0F2FD1B4F9005006E0F0
:10BE800006EB4500BDF818100180681C05B2B4F936
:10BE90000400A842F4DAB4F9000006EB400BA088D5
:10BEA0002188401A401C400000B2029006EB480670
:10BEB0006088401C07B20BE0B4F9001006EB4100AB
:10BEC0005946029A11F0A9FD06EB4806781C07B204
:10BED000B4F90600B842EFDA38E04FF0000B00206A
:10BEE0000290029801904A4601990698FFF7E4FEF5
:10BEF0000090B4F9027024E0B4F9005019E0BBF1ED
:10BF0000000F14D136F81500BDF80410884209D08E
:10BF100006EB4500008801904A4601990698FFF714
:10BF2000CBFE009006EB4500BDF800100180681CB8
:10BF300005B2B4F90400A842E1DA06EB4806781C21
:10BF400007B2B4F90600B842D6DA00BF07B0BDE8C0
:10BF5000F08F2DE9FF4F85B0804689461D46102D94
:10BF600002DA09B0BDE8F08FFB2D00DDFF254A465F
:10BF7000414603A805F0F8FC074607B9F1E7FEF7CC
:10BF8000ACFC8346584605F03DF90446BDF80C006C
:10BF9000218A401A00B2ADF80400BDF80E10608A84
:10BFA000081A00B2ADF80600BDF81000218A401A48
:10BFB00000B2ADF80800BDF81210608A081A00B28D
:10BFC000ADF80A00D4F808A004F1100000F06FFBEF
:10BFD0000646BDF8060010FB06F00AEB400A009585
:10BFE000A06801AA3146079BFFF70FFF00BFB8E723
:10BFF0002DE9FF4F9DB00C46FEA000681C90FEA0EE
:10C0000000681B90FDA30FCB17AD0FC52B98102810
:10C0100002DA21B0BDE8F08F2B98FB2801DDFF206C
:10C020002B901F9800B9F4E7002315A9DDE91F0242
:10C0300004F0E2FD1490149800B9EAE71D98008816
:10C040009DF95810084405B21F98017A407A091AE0
:10C050001D98408808449DF85710401A9DF95910C2
:10C06000401A06B29DF85A00012806D0022809D0CD
:10C0700004280CD0082814D10EE00DF1700B80209C
:10C0800013900FE00DF16C0BC02013900AE00DF13E
:10C090005C0BF020139005E04FF0000BFF20139095
:10C0A00000E0B6E700BFDDE91F0104F09DFD824618
:10C0B000BAF1000F00D1ACE79DF856002844B4F95E
:10C0C000001088420EDBB4F90400A8420ADB9DF898
:10C0D00057003044B4F90210884203DBB4F906007B
:10C0E000B04200DA95E7FEF7F8FB1190119805F0E1
:10C0F00089F8804608F1100000F0D9FA1090D8F8BD
:10C1000008709DF85600C0100D909DF8560000F084
:10C11000070018B10D98401CC0B20D909DF8560054
:10C120009DF85A1010FB01F00C90B4F90000A842E1
:10C1300001DC002002E0B4F90000401B00B20B90CB
:10C140009DF856002844B4F90410884202DC9DF89A
:10C15000560003E0B4F90400401B401C00B20A90F2
:10C16000B4F90200B04201DC002002E0B4F90200A0
:10C17000801B00B209909DF857003044B4F90610B6
:10C18000884202DC9DF8570003E0B4F90600801BEA
:10C19000401C00B20890B8F91200311A109801FB47
:10C1A0000050B8F91010401A07EB4007109A0B998D
:10C1B000099800FB021007EB40070C9909984843C7
:10C1C0009DF85A200B9901FB0200079007980AEB93
:10C1D000D00A079800F007090020049009980E90F3
:10C1E000A7E0139840FA09F012900B980F9080E0A6
:10C1F000C9F108009DF85A10421A9AF800001299E5
:10C200000840104106900698D0B32B98FF280AD119
:10C210009DF85A00082801D1069802E006981BF8FC
:10C22000000005900FE09DF85A00082804D12B99D2
:10C2300006984843001205E006981BF800002B9969
:10C2400048430012059011984069D0B105980290BA
:10C25000BDF8A800ADF804000E988119B8F81200D6
:10C26000081A00B200900F982844B8F81020801ADD
:10C2700003B2D8F808101198D0F814C0109AE0470B
:10C280001BE03888BDF8A810884216D00598FB2816
:10C2900003DDBDF8A80038800FE0059810280CDDFC
:10C2A000049850B9388802900146059A2A98FFF7F9
:10C2B00003FD0390BDF80C003880BF1C9DF85A00A8
:10C2C000C0F1080048450ADD9DF85A0048441FFAAD
:10C2D00080F99DF85A1012980841129005E04FF02D
:10C2E0000009139812900AF1010A0F98401C00B23D
:10C2F0000F900A990F988842FFF67AAF9DF8561072
:10C300000A98091A0B9808449DF85A1000FB0190EE
:10C310001FFA80F90AEBE90A09F00709DDE90A01C9
:10C32000411A1098401A07EB40070E98401C00B2C3
:10C330000E9008990E988842FFF653AF00BF68E64A
:10C340002DE9FE430546884616461F46FF2F05D1B8
:10C3500072004146284611F060FB17E0002412E00D
:10C3600005EB44000088019008EB440000883A4641
:10C3700000900199FFF7A0FC029005EB4400BDF886
:10C3800008100180641CB442EAD300BFBDE8FE83FC
:10C390002DE9FF4F8FB090461298102802DA13B0A3
:10C3A000BDE8F08F1298FB2801DDFF2012900DA848
:10C3B000DDE90F1205F0D8FA0C900C9800B9EEE701
:10C3C0001D9808B1032000E0022082460F9800F07B
:10C3D0006EF90B900F98B0F90200BDF93610884243
:10C3E00016DABDF936100F98B0F90200081A0B9949
:10C3F00048430BE000FF00000055AAFF0011223364
:10C40000445566778899AABBCCDDEEFF00FB0A880D
:10C410000F98B0F90000BDF93410884207DABDF971
:10C4200034100F98B0F90000081A00FB0A88FEF7D4
:10C4300054FA8146484604F0E5FE0746BDF834004C
:10C44000398A401A00B2ADF83400BDF83610788A47
:10C45000081A00B2ADF83600BDF83800398A401A23
:10C4600000B2ADF83800BDF83A10788A081A00B268
:10C47000ADF83A0007F1100000F019F90A90BD6814
:10C48000BDF836100A9811FB00F005EB4005BDF928
:10C49000340005EB40050DA800F009F909900020D3
:10C4A00008901C9800284AD11D98002847D112985E
:10C4B000FF2844D11F98002841D1D9F8140040B377
:10C4C000BDF9364020E0002616E006FB0A80008811
:10C4D000079012980290BDF81C00ADF8040000947B
:10C4E000BDF83400304403B2B968D9F814C04846E6
:10C4F0000A9AE047701C06B209988642E5DB0B9861
:10C5000000FB0A88601C04B2BDF93A00A042DADAE6
:10C51000CBE0BDF936400DE041462846129B099A12
:10C52000FFF70EFF0B9800FB0A880A9805EB400501
:10C53000601C04B2BDF93A00A042EDDAB5E000207B
:10C54000079007980690DDE91E020699FFF7B4FBF5
:10C550000590BDF93640A2E0002694E0DDF848B031
:10C5600006FB0A8004901D9888B104990A784978DE
:10C5700002EB012189B203910499887800B980E027
:10C58000FF2803D000FB0BF14FEA112B02E00498C7
:10C59000008803901C9830B1BDF80C00B9F81C104D
:10C5A000884200D16DE01F98D0B3BDF81800BDF8E7
:10C5B0000C10884207D003980690DDE91E02069908
:10C5C000FFF77AFB0590D9F8140088B1CDF808B0D0
:10C5D000BDF81400ADF804000094BDF834003044F8
:10C5E00003B2B968D9F814C048460A9AE04747E050
:10C5F000BBF1FF0F04D1BDF8140025F816003FE091
:10C6000005EB460000885A46014601900598FFF761
:10C6100053FB029005EB4600BDF8081001802FE0A7
:10C62000FFE7D9F8140088B1CDF808B0BDF80C00C8
:10C63000ADF804000094BDF83400304403B2B9688A
:10C64000D9F814C048460A9AE04719E0BBF1FF0F39
:10C6500005D105EB4600BDF80C10018010E00898EC
:10C6600070B905EB460000885A46014601900398D0
:10C67000FFF722FB029005EB4600BDF80810018091
:10C6800000BF701C06B209988642FFF667AF0B9890
:10C6900000FB0A880A9805EB4005601C04B2BDF94E
:10C6A0003A00A042BFF658AF00BF00BF77E6014690
:10C6B00088880A88801A401C00B270470146002012
:10C6C0000C290FD006DC02290AD0052907D00B2936
:10C6D0000CD106E00D2906D00E2907D104E000BFD9
:10C6E00000BF00BF00BF00BF012001E0002000BF6D
:10C6F00000BF704701460020CA1E082A0CD2DFE89E
:10C7000002F0050B0B040607080900BF00BF00BFBD
:10C7100000BF00BF012001E0002000BF00BF704744
:10C720002DE9FF4F8FB0064692461D46DDF870B0EA
:10C7300032460DA8109905F017F90C900C9818B90D
:10C74000012013B0BDE8F08FBBF1FF0F02D1332001
:10C75000405D04E03320405D00FB0BF000120B90C5
:10C760002946504603F08CFD04460CB90020E8E74A
:10C77000217C01F01F00FFF7BDFF8046217C01F006
:10C780001F00FFF79BFF0746E069B8B1FF23FD4A92
:10C790003046109903F018FD00204FF6FF71CDE9E7
:10C7A0000201CDE904100146E069FF23F54ACDE915
:10C7B00000013046109900F053FC6FE0606970B1E1
:10C7C0003220405D0390288EADF80800CDE9008747
:10C7D000626930460B9B1099FFF7DAFD5EE00DA809
:10C7E00000F00FFC0A900DA800F00BFC00EB4000DD
:10C7F0000390FFF7AFF9099007A80D9901600E9912
:10C80000416000BF012105F07BF8BDF8340031889C
:10C81000401A00B20690BDF836007188401A00B286
:10C820000590BDF93600049032E00998009020464A
:10C830000A9BDDE9052104F0A5F98146B9F1010F54
:10C8400004D0204604F0B8F900207AE73220405D99
:10C850000390288EADF80800CDE9008707A80B9B50
:10C86000099A1099FFF794FDBDF81E00401C00B214
:10C87000ADF81E00BDF82200401C00B2ADF8220049
:10C880000598401C00B205900498401C00B204902A
:10C89000BDF93A1004988142C7DA00BF012050E781
:10C8A0002DE9F04387B006460F4615469846DDF859
:10C8B0003890C5B9FF23B34A3946304603F084FCAB
:10C8C00000204FF6FF71CDE90201CDE90410AEA1C1
:10C8D000FF23AC4ACDE900103946304600F0C0FBDA
:10C8E00007B0BDE8F08343462A4639463046CDF8C6
:10C8F0000090FFF715FF0446B4B9FF23A14A39465B
:10C90000304603F061FC00204FF6FF71CDE90201D3
:10C91000CDE904109CA1FF239A4ACDE900103946C5
:10C92000304600F09DFBDBE700BFD9E70146002061
:10C930000F291DD2DFE801F008091C1C0B0E0C109A
:10C940001316191114171A0000BF002012E000BFBF
:10C9500010200FE018200DE000BF01200AE000BF0A
:10C96000022007E000BF042004E000BF082001E02F
:10C97000002000BF00BF70472DE9FE4304460D466E
:10C9800016461F4600200290029801902068C0F3CE
:10C990008A20A84204DC2068C0F38A20451E02E0F9
:10C9A000002D00DA00252068B6EB505F04DB012182
:10C9B0002068C1EB505602E0002E00DA0026A36882
:10C9C000207800F01F00042809D0207800F01F0014
:10C9D000062804D0207800F01F00052813D1217804
:10C9E00001F01F00FFF7A2FF4FEAE0082068C0F344
:10C9F0008A20704300FB08F005FB080903EB0900DF
:10CA00000088019088E0207800F01F00072819D1E5
:10CA1000083305F00700ED102268C2F38A22D21D08
:10CA2000D21002FB06515A5CC0F107084FF0010C0E
:10CA30000CFA08FC02EA0C02C0F1070C42FA0CF2F4
:10CA4000019269E0207800F01F00082819D1103306
:10CA5000AA07500FAD102268C2F38A22D21C92108E
:10CA600002FB06515A5CC0F106084FF0030C0CFAA9
:10CA700008FC02EA0C02C0F1060C42FA0CF2019228
:10CA80004AE0207800F01F00092819D14033EA0756
:10CA9000500F6D102268C2F38A22521C521002FB02
:10CAA00006515A5CC0F104084FF00F0C0CFA08FC58
:10CAB00002EA0C02C0F1040C42FA0CF201922BE0E3
:10CAC000207800F01F000A2809D103F5806321684F
:10CAD000C1F38A2101FB0650195C01911CE020780A
:10CAE00000F01F000B280ED0207800F01F000C284B
:10CAF00009D0207800F01F000D2804D0207800F025
:10CB00001F000E2808D117B1388E019004E00020D4
:10CB100000900098019000BFBDF804100846BDE8E1
:10CB2000FE832DE9FF4303461868C0F38A2088423C
:10CB300004DC1868C0F38A20411E02E0002900DAF4
:10CB400000211868B2EB505F04DB01251868C5EBC3
:10CB5000505202E0002A00DA00229C68187800F0A7
:10CB60001F00052814D11868C0F38A20504300EB39
:10CB7000400001EB41068519A81C205C04B0BDE80B
:10CB8000F0830000602C00204E6F0A646174610025
:10CB9000187800F01F000B281BD101F00705C91001
:10CBA0001868C0F38A20C01DC01000FB0216A05DEB
:10CBB000C5F107084FF0010C0CFA08FC00EA0C0064
:10CBC000C5F1070C40FA0CF70FB10020D6E7FF20A3
:10CBD000D4E7187800F01F000C281CD1F9A00068D9
:10CBE00003908807450F89101868C0F38A20C01C7D
:10CBF000801000FB0216A05DC5F106084FF0030C83
:10CC00000CFA08FC00EA0C00C5F1060C40FA0CF71F
:10CC100003A8C05DB2E7187800F01F000D2826D1E8
:10CC20000FF2A439D9E901C8D9F80000D9F80C905D
:10CC3000CDE901C8CDF80C900090C807450F491008
:10CC40001868C0F38A20401C401000FB0216A05D4B
:10CC5000C5F104084FF00F0C0CFA08FC00EA0C00B8
:10CC6000C5F1040C40FA0CF71DF8070086E71878A8
:10CC700000F01F000E2806D11868C0F38A2000FBC0
:10CC80000215605D7AE700BFFF2077E72DE9FF47D7
:10CC900005460E461746AC68287800F01F000428A9
:10CCA00004D0287800F01F00062815D1297801F05B
:10CCB0001F00FFF73BFE4FEAE0082868C0F38A2018
:10CCC000784300FB08F006FB080904EB0900424624
:10CCD00003A910F0A2FE94E0287800F01F000528B8
:10CCE00016D1297801F01F00FFF720FE4FEAE00877
:10CCF0002868C0F38A20784300FB08F006FB080987
:10CD0000A8F1010204EB090003A910F086FE78E007
:10CD1000287800F01F0007281DD1083406F007010D
:10CD2000F6102A68C2F38A22D21DD21002FB0760D5
:10CD3000225CC1F1070C012303FA0CF39A4322543D
:10CD4000BDF80C2002F00102C1F107039A40235CF8
:10CD50001A43225455E0287800F01F0008281DD1FE
:10CD60001034B207510FB6102A68C2F38A22D21CBF
:10CD7000921002FB0760225CC1F1060C032303FA48
:10CD80000CF39A432254BDF80C2002F00302C1F1C7
:10CD900006039A40235C1A43225432E0287800F0BC
:10CDA0001F0009281DD14034F207510F76102A6860
:10CDB000C2F38A22521C521002FB0760225CC1F1AE
:10CDC000040C0F2303FA0CF39A432254BDF80C20F1
:10CDD00002F00F02C1F104039A40235C1A4322546B
:10CDE0000FE0287800F01F000A280AD104F58064BB
:10CDF0002968C1F38A2101FB0760BDF80C1021549A
:10CE000000BFBDE8FF872DE9F04304460D461746F5
:10CE10001E46A368207800F01F00052813D1217852
:10CE200001F01F00FFF782FD4FEAE0082068C0F321
:10CE30008A20784300FB08F005FB080909EB08008D
:10CE4000401E1E547DE0207800F01F000B2820D1EA
:10CE5000F61105F00701ED102268C2F38A22D21DF7
:10CE6000D21002FB07501A5CC1F107084FF0010C09
:10CE70000CFA08FC22EA0C021A5406F00102C1F175
:10CE8000070C02FA0CF213F800C042EA0C021A5422
:10CE900057E0207800F01F000C2820D1B611AA0717
:10CEA000510FAD102268C2F38A22D21C921002FBED
:10CEB00007501A5CC1F106084FF0030C0CFA08FC8D
:10CEC00022EA0C021A5406F00302C1F1060C02FA1F
:10CED0000CF213F800C042EA0C021A5431E0207838
:10CEE00000F01F000D2820D13611EA07510F6D10F8
:10CEF0002268C2F38A22521C521002FB07501A5CAD
:10CF0000C1F104084FF00F0C0CFA08FC22EA0C02E5
:10CF10001A5406F00F02C1F1040C02FA0CF213F8D5
:10CF200000C042EA0C021A540BE0207800F01F0007
:10CF30000E2806D12168C1F38A2101FB07501E5437
:10CF400000BFBDE8F08317B583B0037803F01F037B
:10CF50000B2B01D1012912DC037803F01F030C2BEA
:10CF600001D103290BDC037803F01F030D2B01D142
:10CF70000F2904DC037803F01F030E2B01D106B048
:10CF800010BD059B0193BDF80430DB0ADB008DF872
:10CF90000230BDF80430C3F345139B008DF8013017
:10CFA000BDF80430DB061B0E8DF80030FF238DF832
:10CFB0000330009B0293826802EB8103029C1C6099
:10CFC00000BFDCE70055AAFF001122334455667705
:10CFD0008899AABBCCDDEEFF0146032001B970475A
:10CFE0000A461378202B04DB13787F2B01DC012009
:10CFF00005E01378802B01DB022000E0002000BF59
:10D00000EDE7014688880A88801A401C00B2704704
:10D0100001460020302905DB392903DCA1F130026B
:10D02000D0B21CE0612902DBA1F12002D1B2A1F152
:10D030004102062A10D2DFE802F0030507090B0DB2
:10D040000A200BE00B2009E00C2007E00D2005E092
:10D050000E2003E00F2001E0002000BF00BF70475A
:10D060002DE9FF4FA7B082461446DDF8E480DDE9E4
:10D070003476606A269006F0020020B9504600F02F
:10D080005AFA259010E047F61841B4F92A008DE8C5
:10D090004300B4F92830394609A8626A05F0C9FC92
:10D0A000BDF92400259000BF00BF2698007A618D4D
:10D0B000084400B2249000202390BAF80000ADF894
:10D0C0008800BAF80200ADF88A0000202190209074
:10D0D000369870B13698B0F9000021903698B0F9C2
:10D0E00002002090BDF88A102098084400B2ADF8E4
:10D0F0008A000025681E1F90B8F1000F24D02098E8
:10D1000010BBBAF9020000281EDABAF90210D8F8EA
:10D110000800401A002805DDBAF90210D8F8080006
:10D12000401A04E0BAF90200D8F80810401A24990D
:10D130004900C1F58061884203DD4FF0FF30C8F837
:10D140000000D8F800001F90B8F1000F0BD01F9816
:10D15000002808DB1F9DBDF88A00B8F804100844B9
:10D1600000B2ADF88A000096B4F928207819DDE9FC
:10D17000253105F0D6FB00EB05092EE04D46009663
:10D18000B4F928207819DDE9253105F0CAFB81447E
:10D19000BDF88A102498084400B2ADF88A00B8F1AE
:10D1A000000F15D0BDF98A0010F5806F10DBD8F89C
:10D1B000000000280CDAC8F80050BDF98A00BAF95E
:10D1C0000210401AC8F80400BAF90200C8F80800B2
:10D1D000785D10B92BB0BDE8F08FBDF98A102498A6
:10D1E00001442898B0F902008142C7DB06F0040030
:10D1F000D0B10096B4F92830A9EB050291B27819A4
:10D20000269A05F048FB2390504600F094F92399A4
:10D21000A0EB010B0BEBDB70BDF8881001EB60009D
:10D2200000B2ADF8880018E006F00800A8B100963A
:10D23000B4F92830A9EB050291B27819269A05F0C5
:10D240002AFB2390504600F076F92399401ABDF846
:10D250008810084400B2ADF888002A98FF2802D14F
:10D260002C20005D04E02C20005D2A994843001228
:10D270001E9000201D901B90B2490AA8FDF77AFF6E
:10D28000608CADF82A000AA8BDF82A10ADF82C1061
:10D290004BE1369830B1BDF888102198084400B2AF
:10D2A000ADF8880000201D901C95E5E01CA93846CB
:10D2B000A54A1268904709901C9978180021A24A43
:10D2C00012689047089006F00100002877D09FA0D0
:10D2D00001780998814213D11D9828B91C9880B211
:10D2E0001B9001201D90C7E01D98012802D100204D
:10D2F0001D9005E01D98022802D100201D90BBE082
:10D300001D9801285BD10998202857D1DDE91B0120
:10D31000081A07284ED11B98384401680591808867
:10D32000ADF8180000208DF81A009DF81500FFF7E1
:10D330006FFE83469DF81400FFF76AFE0BEB0010AA
:10D3400004909DF81700FFF763FE83469DF81600D2
:10D35000FFF75EFE0BEB001003909DF81900FFF73E
:10D3600057FE83469DF81800FFF752FE0BEB0010A6
:10D370000290049BD8B2039BD9B2029BDAB24FEA67
:10D38000D20CBDF804306CF3040301934FEA910C06
:10D39000BDF804306CF34A1301934FEAD00CBDF88A
:10D3A00004306CF3CF230193BDF804C063461A9395
:10D3B00002E004E0208C1A9002201D905CE0206ABC
:10D3C00007901D98022801D11A980790DDE90821DD
:10D3D000269803F020FC00B219904FF6FF713798A1
:10D3E000884230D0389888422DD03846584A1C9907
:10D3F0001268904783463798834523DD38988345E4
:10D4000020DCBDF88800ADF81400BDF88A00ADF846
:10D410001600BDF8881019980144208D0844401E5C
:10D4200000B2ADF81800BDF88A1024980844401ED8
:10D4300000B2ADF81A000AAA05A81E9B289902F0AE
:10D44000C3FE00BF00BF1E980190BDF81C00ADF8E0
:10D45000000022A8099B269A2899FEF7C9FD199871
:10D46000002808DDBDF88810228D19981044084462
:10D4700000B2ADF8880000BF1C984845FFF416AF15
:10D480004D460096B4F928207819DDE9253105F0DC
:10D4900048FA8144BAF80000ADF8880006F00400AC
:10D4A000D0B10096B4F92830A9EB050291B27819F1
:10D4B000269A05F0F0F92390504600F03CF82399A5
:10D4C000A0EB010B0BEBDB70BDF8881001EB6000EB
:10D4D00000B2ADF8880018E006F00800A8B1009688
:10D4E000B4F92830A9EB050291B27819269A05F013
:10D4F000D2F92390504600F01EF82399401ABDF847
:10D500008810084400B2ADF88800BDF88A1024984D
:10D51000084400B2ADF88A00BDF98A102898B0F925
:10D520000600814200DD55E600BF785D00287FF4EB
:10D53000B0AE00BF4EE6014688880A88801A401CBB
:10D5400000B270479C2C0020D00100202300000076
:10D55000DC01002007B581B0BDF80800C00AC2F1A7
:10D56000FF014843BDF80410C90A01FB0200010A8B
:10D57000BDF8000061F3CF200090BDF80800C0F3B3
:10D580004510C2F1FF014843BDF80410C1F3451135
:10D5900001FB0200010ABDF8000061F34A1000908F
:10D5A000BDF8080000F01F00C2F1FF014843BDF8BC
:10D5B000041001F01F0101FB0200010ABDF8000088
:10D5C00061F304000090BDF80010084604B000BDEF
:10D5D00030B50346022B04D1FE48405C5043001294
:10D5E00030BD032B04D1FC48405C50430012F7E7E8
:10D5F000042B04D1F948405C50430012F0E7C1EB22
:10D60000C105581EB5FBF0F0C4B2F548005D5043AB
:10D61000000AE5E72DE9F04104460D461646FDF700
:10D620005CF9804603F0CEFD0746B4EB650F04DBE2
:10D63000C5F34F040CB1601E84B2B4EB660F04DB7B
:10D64000C6F34F040CB1601E84B2002C01DDE01B58
:10D6500084B22046BDE8F0810FB5A3B02598C088FC
:10D6600080B22290FDF739F9079003F0ABFD2190CD
:10D670002598B0F90C002090259840891F90259896
:10D68000807B1E902698FF2802D12598C07B04E05D
:10D690002598C07B2699484300121D902098401E73
:10D6A00000B22090219818B12098401E00B220901E
:10D6B000239802F0D6FD1C90239802F0D9FD1B9010
:10D6C000DDE91B212298FFF7A5FF2290239801880E
:10D6D000229801442198084400B2ADF868002398CC
:10D6E0004188229801442198084400B2ADF86A00AC
:10D6F00023980188229801442198084400B2ADF88B
:10D7000064002398C1882298091A2198081A00B247
:10D71000ADF86600239881882298091A2198081A82
:10D7200000B2ADF860002398418822980144219806
:10D73000084400B2ADF86200239881882298091A43
:10D740002198081A00B2ADF85C002398C18822988D
:10D75000091A2198081A00B2ADF85E00229802B2A8
:10D7600015A916A804F0F8F920992298401A00B2D9
:10D7700012901298002801DA0020129013A914A820
:10D78000129A04F0E9F900200D900C90229800B252
:10D790000B9000200A90099020992298401A00B21C
:10D7A0000890FDE3BDF95200BDF95010884209DA36
:10D7B000BDF85800BDF85010401A00B20F900F98F5
:10D7C0000E900AE0BDF85800BDF85A10401A00B299
:10D7D0000F900F98401E00B20E90219800287DD027
:10D7E000BDF958100B98814279D0BDF95A000C90C0
:10D7F000DDE90C01401A00B207900B98ADF8180053
:10D800000D98ADF81A00002005902EE10798012828
:10D8100006DD1D9A05990798FFF7DAFE049008E0E7
:10D820001D9A05990798FEF7CDF91D99081AC0B2FF
:10D8300004901E9800F00100D8B31E9800F0080074
:10D84000B8B304980090BDF85E00BDF81A1001440A
:10D850000598084400B20290BDF85C00BDF81810AD
:10D860000844401C00B2019025984089034603906B
:10D87000249ADDE90101FEF75DFA04980090BDF8F5
:10D880005E00BDF818100844401C00B20290BDF8BC
:10D890005C00BDF81A1001440598084400B20190DC
:10D8A0002598408903460390249ADDE90101FEF79B
:10D8B00041FA1E9800F00100E8B31E9800F0040041
:10D8C000C8B304980090BDF86600BDF8181008446D
:10D8D000401C00B20290BDF8640001E054E1CFE0CA
:10D8E000BDF81A10494201440598081A00B2019087
:10D8F0002598408903460390249ADDE90101FEF74B
:10D9000019FA04980090BDF86600BDF81A10014499
:10D910000598084400B20290BDF86400BDF81810E4
:10D9200049420844401E00B20190259840890346B0
:10D930000390249A00E003E0DDE90101FEF7FAF923
:10D940001E9800F00200E0B31E9800F00400C0B37F
:10D9500004980090BDF86A00BDF81A1049420144CD
:10D960000598081A00B20290BDF86800BDF81810BA
:10D9700049420844401E00B2019025984089034660
:10D980000390249ADDE90101FEF7D4F90498009090
:10D99000BDF86A00BDF8181049420844401E00B2A4
:10D9A0000290BDF86800BDF81A104942014405987C
:10D9B000081A00B201902598408903460390249AE2
:10D9C00000E003E0DDE90101FEF7B4F91E9800F084
:10D9D000020007E082090208840902088709020898
:10D9E0008B090208E8B31E9800F00800C8B3049839
:10D9F0000090BDF86200BDF8181049420844401E6E
:10DA000000B20290BDF86000BDF81A1001440598FC
:10DA1000084400B201902598408903460390249A57
:10DA2000DDE90101FEF786F904980090BDF8620077
:10DA3000BDF81A10494201440598081A00B2029034
:10DA4000BDF86000BDF818100844401C00B20190F9
:10DA50002598408903460390249ADDE90101FEF7E9
:10DA600069F90598401C00B205900799059888420D
:10DA7000FFF6CCAEBDF958000B900C980D9000BF8E
:10DA8000BDF95010089881427ED0BDF95A00099026
:10DA9000DDE90901401A00B207900898ADF81800B6
:10DAA0000A98ADF81A00002005904BE1079801286C
:10DAB00009DD1D9A05990798FFF78AFD1D99081A37
:10DAC000C0B2049005E01D9A05990798FEF77AF810
:10DAD00004901E9800F00100F8B11E9800F00800B4
:10DAE000D8B104980090BDF85E00BDF81A1001444A
:10DAF0000598084400B20290BDF85C00BDF818100B
:10DB00000844401E00B201902598408903460390C6
:10DB1000249ADDE90101FEF70DF91E9800F00100DD
:10DB200000B31E9800F00400E0B104980090BDF826
:10DB30006600BDF818100844401E00B20290BDF8FF
:10DB40006400BDF81A10494201440598081A00B251
:10DB500001902598408903460390249ADDE901014C
:10DB6000FEF7E8F81E9800F0020018B31E9800F0C7
:10DB70000400F8B104980090BDF86A00BDF81A10CE
:10DB800049420144059800E0E7E0081A00B202901B
:10DB9000BDF86800BDF8181049420844401C00B2A6
:10DBA00001902598408903460390249ADDE90101FC
:10DBB000FEF7C0F81E9800F0020000B31E9800F0B7
:10DBC0000800E0B104980090BDF86200BDF818109C
:10DBD00049420844401C00B20290BDF86000BDF804
:10DBE0001A1001440598084400B201902598408914
:10DBF00003460390249ADDE90101FEF79BF8BDF985
:10DC00001800401EBDF91A200599114488427DD0A4
:10DC10001E9800F00100F8B11E9800F00800D8B17D
:10DC200004980090BDF85E00BDF818100844401E2E
:10DC300000B20290BDF85C00BDF81A1001440598CE
:10DC4000084400B201902598408903460390249A25
:10DC5000DDE90101FEF76EF81E9800F0010000B347
:10DC60001E9800F00400E0B104980090BDF8660032
:10DC7000BDF81A1001440598084400B20290BDF89E
:10DC80006400BDF8181049420844401C00B20190DD
:10DC90002598408903460390249ADDE90101FEF7A7
:10DCA00049F81E9800F0020008B31E9800F0040026
:10DCB000E8B104980090BDF86A00BDF81810494218
:10DCC0000844401C00B20290BDF86800BDF81A106C
:10DCD000494201440598081A00B2019025984089EC
:10DCE00003460390249ADDE90101FEF723F81E980C
:10DCF00000F0020050B11E9800F0080030B1049806
:10DD00000090BDF86200BDF81A1000E016E049422C
:10DD100001440598081A00B20290BDF86000BDF8F1
:10DD200018100844401E00B201902598408903460F
:10DD30000390249ADDE90101FDF7FCFF0598401CE2
:10DD400000B20590079905988842FFF6AFAEBDF97D
:10DD50005000089009980A9000BF1E9800F001003A
:10DD6000F0B31E9800F00800D0B3BDF85C00BDF819
:10DD7000581001440E98081A00B2ADF84000BDF8E2
:10DD80005C00BDF85810084400B2ADF84400BDF87E
:10DD90005E00BDF85A10084400B2ADF84200BDF86C
:10DDA0005E00BDF85A10084400B2ADF8460010A855
:10DDB0001D9B1F9A2499FEF7CCF8BDF85C00BDF8B6
:10DDC0005A10084400B2ADF84000BDF85C00BDF840
:10DDD0005A10084400B2ADF84400BDF85E0000E0FF
:10DDE00015E0BDF8581001440F98081A00B2ADF8BC
:10DDF0004200BDF85E00BDF85810084400B2ADF80E
:10DE0000460010A81D9B1F9A2499FEF7A2F81E98A1
:10DE100000F00100F0B31E9800F00400D0B3BDF88C
:10DE20006400BDF85A104942084400B2ADF8400001
:10DE3000BDF86400BDF85A104942084400B2ADF87C
:10DE40004400BDF86600BDF8581001440E98081A49
:10DE500000B2ADF84200BDF86600BDF858100844A5
:10DE600000B2ADF8460010A81D9B1F9A2499FEF73A
:10DE700070F8BDF86400BDF858104942084400B27B
:10DE8000ADF84000BDF86400BDF8581049420144A7
:10DE90000F9800E019E0084400B2ADF84400BDF866
:10DEA0006600BDF85A10084400B2ADF84200BDF853
:10DEB0006600BDF85A10084400B2ADF8460010A83C
:10DEC0001D9B1F9A2499FEF744F81E9800F002004B
:10DED000E8B31E9800F00400C8B3BDF96600BDF9B0
:10DEE0005A100844BDF96A10BDF95A205242114433
:10DEF00088422BDDBDF86800BDF85810494208443F
:10DF000000B2ADF84000BDF86800BDF858104942B5
:10DF100001440E98084400B2ADF84400BDF86A0010
:10DF2000BDF85A104942084400B2ADF84200BDF8AD
:10DF30006A00BDF85A104942084400B2ADF84600E4
:10DF400010A81D9B1F9A2499FEF703F800E02DE00E
:10DF5000BDF86800BDF85A104942084400B2ADF857
:10DF60004000BDF86800BDF85A104942084400B2AC
:10DF7000ADF84400BDF86A00BDF8581049420844A5
:10DF800000B2ADF84200BDF86A00BDF85810494231
:10DF900001440F98084400B2ADF8460010A800E014
:10DFA0007DE01D9B1F9A2499FDF7D3FF1E9800F07A
:10DFB0000200E8B31E9800F00800C8B3BDF8600086
:10DFC000BDF85A10084400B2ADF84000BDF860003A
:10DFD000BDF85A10084400B2ADF84400BDF8620024
:10DFE000BDF858104942084400B2ADF84200BDF8EF
:10DFF0006200BDF85810494201440E98084400B22E
:10E00000ADF8460010A81D9B1F9A2499FDF7A1FFAB
:10E01000BDF95E00BDF95A100844BDF96210BDF9A2
:10E020005A205242114488422BDDBDF8600000E0C6
:10E0300027E0BDF8581001440F98081A00B2ADF857
:10E040004000BDF86000BDF85810084400B2ADF8BB
:10E050004400BDF86200BDF85A104942084400B2BD
:10E06000ADF84200BDF86200BDF85A1049420844BC
:10E0700000B2ADF8460010A81D9B1F9A2499FDF729
:10E0800068FF15A916A803F07AFDBDF95200BDF985
:10E090005010884203DA13A914A803F070FDBDF9EB
:10E0A0005A00BDF9581088427FF77CAB21980028B0
:10E0B0007DD0BDF95A000C90DDE90C01401A00B288
:10E0C00007900B98ADF818000D98ADF81A000020D5
:10E0D00005901AE11D9A05990798FDF773FD1D99A2
:10E0E000081AC0B204901E9800F00100D8B31E9820
:10E0F00000F00800B8B304980090BDF85E00BDF8C9
:10E100001A1001440598084400B20290BDF85C0062
:10E11000BDF818100844401C00B2019025984089B1
:10E1200003460390249ADDE90101FDF703FE0498FC
:10E130000090BDF85E00BDF818100844401C00B205
:10E140000290BDF85C00BDF81A100144059808441F
:10E1500000B201902598408903460390249ADDE996
:10E160000101FDF7E7FD1E9800F00100F0B31E98D5
:10E1700000F00400D0B304980090BDF86600BDF82C
:10E1800018100844401C00B20290BDF86400BDF8AD
:10E190001A10494201440598081A00B201902598C6
:10E1A000408903460390249ADDE9010100E0AEE2D4
:10E1B000FDF7C0FD04980090BDF86600BDF81A1088
:10E1C00001440598084400B20290BDF86400BDF80F
:10E1D000181049420844401E00B201902598408919
:10E1E00003460390249ADDE9010100E001E0FDF718
:10E1F000A1FD1E9800F00200F0B31E9800F004008C
:10E20000D0B304980090BDF86A00BDF81A104942D6
:10E2100001440598081A00B20290BDF86800BDF8E4
:10E22000181049420844401E00B2019025984089C8
:10E2300003460390249ADDE90101FDF77BFD049874
:10E240000090BDF86A00BDF8181049420844401E0D
:10E2500000B20290BDF86800BDF81A1049420144AE
:10E260000598081A00B2019025984089034603904A
:10E27000249ADDE9010100E001E0FDF75BFD1E9855
:10E2800000F00200E8B31E9800F00800C8B304983C
:10E290000090BDF86200BDF8181049420844401EC5
:10E2A00000B20290BDF86000BDF81A100144059854
:10E2B000084400B201902598408903460390249AAF
:10E2C000DDE90101FDF736FD04980090BDF862001C
:10E2D000BDF81A10494201440598081A00B202908C
:10E2E000BDF86000BDF818100844401C00B2019051
:10E2F0002598408903460390249ADDE90101FDF742
:10E3000019FD0598401C00B20590079905988842B0
:10E31000FFF6E0AEBDF91800BDF91A10401A00284A
:10E3200005DDBDF91800BDF91A10401A04E0BDF969
:10E330001A00BDF91810401A079988427ED10B982F
:10E34000ADF818000B98ADF81A001D984010049015
:10E350001E9800F00100E0B11E9800F00800C0B166
:10E3600004980090BDF85E00BDF81810084400B293
:10E370000290BDF85C00BDF81A10084400B201908C
:10E380002598408903460390249ADDE90101FDF7B1
:10E39000D1FC1E9800F00100E8B11E9800F00400C6
:10E3A000C8B104980090BDF86600BDF81A10084482
:10E3B00000B20290BDF86400BDF81810494208444C
:10E3C00000B201902598408903460390249ADDE924
:10E3D0000101FDF7AFFC1E9800F00200F0B11E989D
:10E3E00000F00400D0B104980090BDF86A00BDF8B8
:10E3F00018104942084400B20290BDF86800BDF808
:10E400001A104942084400B20190259840890346F9
:10E410000390249ADDE90101FDF78CFC1E9800F0C1
:10E420000200F8B11E9800F00800D8B104980090DE
:10E43000BDF86200BDF81A10494200E013E008443C
:10E4400000B20290BDF86000BDF81810084400B298
:10E4500001902598408903460390249ADDE9010143
:10E46000FDF768FC00BFBDF9520009900898ADF8AF
:10E4700018000A98ADF81A00DDE90901401A00B247
:10E480000790002005903CE11D9A05990798FDF73B
:10E4900099FB04901E9800F00100F8B11E9800F05E
:10E4A0000800D8B104980090BDF85E00BDF81A10BD
:10E4B00001440598084400B20290BDF85C00BDF824
:10E4C00018100844401E00B2019025984089034668
:10E4D0000390249ADDE90101FDF72CFC1E9800F061
:10E4E000010000B31E9800F00400E0B10498009011
:10E4F000BDF86600BDF818100844401E00B2029036
:10E50000BDF86400BDF81A10494201440598081A84
:10E5100000B201902598408903460390249ADDE9D2
:10E520000101FDF707FC1E9800F0020008B31E98D9
:10E5300000F00400E8B104980090BDF86A00BDF84E
:10E540001A10494201440598081A00B20290BDF819
:10E550006800BDF8181049420844401C00B2019000
:10E560002598408903460390249ADDE90101FDF7CF
:10E57000E1FB1E9800F0020000B31E9800F00800B6
:10E58000E0B104980090BDF86200BDF8181049424F
:10E590000844401C00B20290BDF86000BDF81A109B
:10E5A00001440598084400B201902598408903462B
:10E5B0000390249ADDE90101FDF7BCFBBDF91800C9
:10E5C000401EBDF91A200599114488427ED01E983C
:10E5D00000F00100F8B11E9800F00800D8B10498CE
:10E5E0000090BDF85E00BDF818100844401E00B24F
:10E5F0000290BDF85C00BDF81A100144059808446B
:10E6000000B201902598408903460390249ADDE9E1
:10E610000101FDF78FFB1E9800F0010000B31E986A
:10E6200000F00400E0B104980090BDF86600BDF869
:10E630001A1001440598084400B20290BDF8640025
:10E64000BDF8181049420844401C00B201902598BA
:10E65000408903460390249ADDE90101FDF76AFB36
:10E660001E9800F0020008B31E9800F00400E8B104
:10E6700004980090BDF86A00BDF81810494208449B
:10E68000401C00B20290BDF86800BDF81A10494263
:10E6900001440598081A00B2019025984089034664
:10E6A0000390249ADDE90101FDF744FB1E9800F078
:10E6B000020058B11E9800F0080038B1049800908C
:10E6C000BDF86200BDF81A10494200E015E00144AF
:10E6D0000598081A00B20290BDF86000BDF8181045
:10E6E0000844401E00B201902598408903460390DB
:10E6F000249ADDE90101FDF71DFB0598401C00B2DD
:10E700000590079905988842FFF6BEAE00BF27B076
:10E7100000BD2DE9FF4F87B004469146B9F80600C9
:10E720001FFA80F8FCF7D9F8009002F04BFD07467D
:10E73000204601F096FD0690204601F099FD0590D7
:10E74000B9F90C600A98FF2802D199F80F0004E08B
:10E7500099F80F000A9948430012049099F80E5056
:10E76000B9F80A0003904FF0000BDA46701E06B2AB
:10E770004046DDE90521FEF74DFF8046B04506DA4B
:10E78000A6EB0800C01B0FFA80FBB24603E008EBC3
:10E7900007000FFA80FAB9F8060000287ED105F0CC
:10E7A000020098B12088ADF80400A088ADF80800F8
:10E7B0006088ADF806006088304400B2ADF80A0009
:10E7C00001A8DDE903230899FDF7C3FB05F0080064
:10E7D00028B3A088801B00B2ADF80400A088ADF873
:10E7E0000800B4F9021005F0020008B1701C00E046
:10E7F0000020084400B2ADF80600B4F9061005F098
:10E80000010008B1701C00E00020081A00B2ADF849
:10E810000A0001A8DDE903230899FDF79AFB05F03A
:10E82000040028B32088ADF804002088304400B2EA
:10E83000ADF80800B4F9021005F0020008B1701C30
:10E8400000E00020084400B2ADF80600B4F906105C
:10E8500005F0010008B1701C00E00020081A00B2A9
:10E86000ADF80A0001A8DDE903230899FDF771FB63
:10E8700005F00100A8B12088ADF80400A088ADF82B
:10E880000800E088801B00B2ADF80600E088ADF813
:10E890000A0001A8DDE90323089900E004E0FDF780
:10E8A00058FB0BB0BDE8F08F0AF101000FFA80FAB7
:10E8B00005F0020028B16088504400B2ADF80600AF
:10E8C00004E06088404400B2ADF8060005F00100A5
:10E8D00030B1E088A0EB0A0000B2ADF80A0005E014
:10E8E000E088A0EB080000B2ADF80A0005F00400D3
:10E8F00070B12088ADF80400BDF80400304400B2C7
:10E90000ADF8080001A8DDE903230899FDF721FB14
:10E9100005F0080070B1A088ADF80800BDF8080047
:10E92000801B00B2ADF8040001A8DDE903230899BB
:10E93000FDF70FFB20885044A0EB0B0000B2ADF8B0
:10E940000400A088A0EB0A00584400B2ADF808000B
:10E9500005F0020068B16088ADF8060060883044B8
:10E9600000B2ADF80A0001A8DDE903230899FDF71C
:10E97000F0FA05F0010070B1E088ADF80A00BDF8CA
:10E980000A00801B00B2ADF8060001A8DDE90323F0
:10E990000899FDF7DEFABBF1000F7DD005F002000B
:10E9A000E8B105F00400D0B12088ADF8040020885B
:10E9B0004044384400B2ADF8080060884044401C30
:10E9C000384400B2ADF806006088304400B2ADF8BB
:10E9D0000A0001A8DDE903230899FDF7BAFA05F05A
:10E9E0000200F0B105F00800D8B1A088A0EB080043
:10E9F000C01B00B2ADF80400A088ADF80800608824
:10EA00004044401C384400B2ADF8060060883044F1
:10EA100000B2ADF80A0001A8DDE903230899FDF76B
:10EA200098FA05F00100F0B105F00400D8B1208893
:10EA3000ADF8040020884044384400B2ADF8080026
:10EA4000E088801B00B2ADF80600E088A0EB08006B
:10EA5000401EC01B00B2ADF80A0001A8DDE9032387
:10EA60000899FDF776FA05F00100A8B105F0080055
:10EA700090B1A088A0EB0800C01B00B2ADF8040064
:10EA8000A088ADF80800E088801B00B2ADF8060051
:10EA9000E088A0EB080000E00AE0401EC01B00B2C6
:10EAA000ADF80A0001A8DDE903230899FDF751FA42
:10EAB000B9F80600002863D105F00600A8B1208847
:10EAC000ADF804002088384400B2ADF80800608832
:10EAD000ADF806006088384400B2ADF80A0001A81D
:10EAE000DDE903230899FDF734FA05F00A00A8B11F
:10EAF000A088C01B00B2ADF80400A088ADF80800E3
:10EB00006088ADF806006088384400B2ADF80A00AD
:10EB100001A8DDE903230899FDF71BFA05F00500BC
:10EB2000A8B12088ADF804002088384400B2ADF8C0
:10EB30000800E088C01B00B2ADF80600E088ADF820
:10EB40000A0001A8DDE903230899FDF702FA05F0A0
:10EB50000900A8B1A088C01B00B2ADF80400A088CD
:10EB6000ADF80800E088C01B00B2ADF80600E088F0
:10EB7000ADF80A0001A8DDE903230899FDF7E9F9DA
:10EB800000BF8EE60FB5A9B02B98C08880B2289040
:10EB9000FBF7A3FE0B9002F015FB27902B98408803
:10EBA00026902B98808825902C98FF2802D12B98AE
:10EBB000007A04E02B98007A2C99484300122390A5
:10EBC000299801F055FB2190299801F04AFB2090EB
:10EBD000DDE920122898FEF71DFD2890299801886C
:10EBE000289801442798084400B2ADF87C00299881
:10EBF0004188289801442798084400B2ADF87E0067
:10EC000029980188289801442798084400B2ADF853
:10EC100078002998C1882898091A2798081A00B2FC
:10EC2000ADF87A00299881882898091A2798081A37
:10EC300000B2ADF8740029984188289801442798BB
:10EC4000084400B2ADF87600299881882898091AFE
:10EC50002798081A00B2ADF870002998C188289842
:10EC6000091A2798081A00B2ADF87200289802B263
:10EC700012A913A802F070FFBDF87200BDF84E1083
:10EC8000084400B20090BDF87000BDF84C10084474
:10EC900000B20B90BDF87A00BDF84E10084400B2E7
:10ECA0000A90BDF87800BDF84C104942084400B203
:10ECB0000990014616A8DDE90A2302F014FEBDF80A
:10ECC0007200BDF84C10084400B20090BDF870000E
:10ECD000BDF84E10084400B20B90BDF87A10BDF894
:10ECE0004C00084400B20A90BDF87800BDF84E1000
:10ECF0004942084400B20990014614A8DDE90A23FC
:10ED000002F0F1FDBDF87600BDF84E10494208440E
:10ED100000B20090BDF87400BDF84C10084400B279
:10ED20000B90BDF87E00BDF84E104942084400B279
:10ED30000A90BDF87C00BDF84C104942084400B26E
:10ED40000990014618A8DDE90A2302F0CCFDBDF8C0
:10ED50007600BDF84C104942084400B20090BDF85E
:10ED60007400BDF84E10084400B20B90BDF87E0050
:10ED7000BDF84C104942084400B20A90BDF87C002E
:10ED8000BDF84E104942084400B2099001461AA845
:10ED9000DDE90A2302F0A7FD0020119010902898C9
:10EDA00000B20F908AE2279800287DD0BDF94C1060
:10EDB0000F988142F9D0BDF94E001090DDE91001A5
:10EDC000401A00B207900F98ADF818001198ADF8EE
:10EDD0001A000F992898401AC0EB00212198B1FB26
:10EDE000F0F0C0B22290229ADDE92501FEF7B2FBD5
:10EDF0000E90229ADDE92510FEF7ACFB0D90002065
:10EE00000590F8E00798012806DD239A05990798F0
:10EE1000FEF7DEFB049008E0239A05990798FCF7BB
:10EE2000D1FE2399081AC0B2049004980090BDF84E
:10EE30007200BDF818100844401C00B20390BDF8E1
:10EE40007000BDF81A1001440598084400B2029001
:10EE50000D9B2A9A0399FCF76DFF04980090BDF86A
:10EE60007A00BDF818100844401C00B20390BDF8A9
:10EE70007800BDF81A10494201440598081A00B2FA
:10EE800002900D9B2A9A0399FCF754FF0498009076
:10EE9000BDF87E00BDF8181049420844401E00B27B
:10EEA0000390BDF87C0000E0B0E0BDF81A104942C4
:10EEB00001440598081A00B202900E9B2A9A039901
:10EEC000FCF738FF04980090BDF87600BDF81810E4
:10EED00049420844401E00B20390BDF87400BDF8DA
:10EEE0001A1001440598084400B202900E9B2A9A19
:10EEF0000399FCF71FFF11992898411A05980844B7
:10EF0000C0EB00212198B1FBF0F0C0B22290229A10
:10EF1000DDE92510FEF71EFB0C9004980090BDF86B
:10EF20007210BDF81A0001440598084400B203901D
:10EF3000BDF87000BDF818100844401C00B20290E3
:10EF40000C9B2A9A0399FCF7F5FE04980090BDF8F3
:10EF50007A00BDF81A1001440598084400B20390E5
:10EF6000BDF87810BDF8180040420844401E00B2B9
:10EF700002900C9B2A9A0399FCF7DCFE229ADDE9A9
:10EF80002501FEF7E7FA0C9004980090BDF87E008A
:10EF9000BDF81A10494201440598081A00B20390BE
:10EFA000BDF87C00BDF8181049420844401E00B26C
:10EFB00002900C9B2A9A0399FCF7BCFE04980090DF
:10EFC000BDF87610BDF81A00404201440598081AB1
:10EFD00000B20390BDF87410BDF818000844401C3E
:10EFE00000B202900C9B2A9A0399FCF7A3FE0598A5
:10EFF000401C00B20590079905988842FFF602AFC1
:10F00000BDF94C000F901098119000BF00200B909C
:10F010000A9009900890BDF94E10BDF97A00084495
:10F02000BDF95A10884201D001200990BDF94C1059
:10F03000BDF97A000844BDF95210884201D0012080
:10F040000890BDF94E004042BDF97E100844BDF95C
:10F050006210884201D001200A90BDF94C00404264
:10F06000BDF97E100844BDF96A10884201D0012024
:10F070000B900B9808B3BDF89800BDF89410884227
:10F0800002D12698249012E02998B0F90600BDF923
:10F090006A10401AC0EB00212198B1FBF0F0C0B219
:10F0A0002290229ADDE92510FEF754FA24901AA83E
:10F0B000DDE923322A99FCF74CFF0A9808B3BDF822
:10F0C0009800BDF89410884202D12698249012E04E
:10F0D0002998B0F90610BDF96200081AC0EB0021AA
:10F0E0002198B1FBF0F0C0B22290229ADDE9251000
:10F0F000FEF730FA249018A8DDE923322A99FCF7AC
:10F1000028FF099808B3BDF89800BDF8941088420C
:10F1100002D12698249012E02998B0F90610BDF982
:10F120005A00081AC0EB00212198B1FBF0F0C0B2E0
:10F130002290229ADDE92510FEF70CFA249016A8F9
:10F14000DDE923322A99FCF704FF089808B3BDF8DB
:10F150009800BDF89410884202D12698249012E0BD
:10F160002998B0F90600BDF95210401AC0EB0021F1
:10F170002198B1FBF0F0C0B22290229ADDE925106F
:10F18000FEF7E8F9249014A8DDE923322A99FCF768
:10F19000E0FEBDF87210BDF84E00084400B20090C9
:10F1A000BDF87000BDF84C10084400B20790BDF8DF
:10F1B0007A10BDF84E00084400B20690BDF87810F1
:10F1C000BDF84C004042084400B20590014616A824
:10F1D000DDE9062302F087FBBDF87210BDF84C0094
:10F1E000084400B20090BDF87000BDF84E1008440D
:10F1F00000B20790BDF87A10BDF84C00084400B288
:10F200000690BDF87810BDF84E004042084400B2A8
:10F210000590014614A8DDE9062302F064FBBDF861
:10F220007610BDF84E004042084400B20090BDF890
:10F230007400BDF84C10084400B20790BDF87E0081
:10F24000BDF84E104942084400B20690BDF87C005B
:10F25000BDF84C104942084400B20590014618A878
:10F26000DDE9062302F03FFBBDF87600BDF84C1047
:10F270004942084400B20090BDF87400BDF84E1039
:10F28000084400B20790BDF87E00BDF84C1049421A
:10F29000084400B20690BDF87C00BDF84E1049420B
:10F2A000084400B2059001461AA8DDE9062302F0E1
:10F2B0001AFB12A913A802F062FC00BF13A802F007
:10F2C00053FC00287FF46FADBDF89800BDF8941092
:10F2D000884202D12698249012E02998B0F90600BD
:10F2E000BDF96A10401AC0EB00212198B1FBF0F083
:10F2F000C0B22290229ADDE92510FEF72BF9249066
:10F300001AA8DDE923322A99FCF723FEBDF96A0029
:10F31000BDF96210884221D0BDF89800BDF8941064
:10F32000884202D12698249012E02998B0F906006C
:10F33000BDF96210401AC0EB00212198B1FBF0F03A
:10F34000C0B22290229ADDE92510FEF703F924903D
:10F3500018A8DDE923322A99FCF7FBFDBDF89800D7
:10F36000BDF89410884202D12698249012E0299882
:10F37000B0F90600BDF95A10401AC0EB00212198DF
:10F38000B1FBF0F0C0B22290229ADDE92510FEF721
:10F39000E1F8249016A8DDE923322A99FCF7D9FD7B
:10F3A000BDF95200BDF95A10884221D0BDF898101D
:10F3B000BDF89400814202D12698249012E0299849
:10F3C000B0F90600BDF95210401AC0EB0021219897
:10F3D000B1FBF0F0C0B22290229ADDE92510FEF7D1
:10F3E000B9F8249014A8DDE923322A99FCF7B1FD7D
:10F3F000279800287ED02998018828980844801CE6
:10F4000000B2ADF86800299881882898081A801EF3
:10F4100000B2ADF86C0029984088ADF86A002998D0
:10F420004088ADF86E002B984088089002461AA8D4
:10F43000239B2A99FCF78DFD2998C088ADF86A00B6
:10F440002998C088ADF86E002B98808808900246F5
:10F450001AA8239B2A99FCF77CFDBDF94E00109059
:10F46000DDE91001401A00B20B900F98ADF82800AA
:10F470001198ADF82A000F992898401AC0EB002186
:10F480002198B1FBF0F0C0B22290229ADDE925016B
:10F49000FEF760F80D90229ADDE92510FEF75AF884
:10F4A0000E9000200990EEE0239A09990B98FCF742
:10F4B00089FB2399081AC0B2089008980090BDF8FB
:10F4C0007200BDF828100844401C00B20790BDF837
:10F4D0007000BDF82A1001440998084400B2069053
:10F4E0000E9B2A9A0799FCF725FC08980090BDF816
:10F4F0007A0000E058E1BDF828100844401C00B232
:10F500000790BDF87810BDF82A00404201440998E0
:10F51000081A00B206900E9B2A9A0799FCF70AFC7B
:10F5200008980090BDF87E00BDF8281049420844B4
:10F53000401E00B20790BDF87C10BDF82A00404282
:10F5400001440998081A00B206900D9B2A9A07995F
:10F55000FCF7F0FB08980090BDF87600BDF8281085
:10F5600049420844401E00B20790BDF87410BDF82F
:10F570002A0001440998084400B206900D9B2A9A7B
:10F580000799FCF7D7FB11992898411A0998084464
:10F59000C0EB00212198B1FBF0F0C0B22290229A7A
:10F5A000DDE92510FDF7D6FF0C9008980090BDF816
:10F5B0007200BDF82A1001440998084400B207906F
:10F5C000BDF87010BDF828000844401C00B2069039
:10F5D0000C9B2A9A0799FCF7ADFB08980090BDF8A0
:10F5E0007A00BDF82A1001440998084400B2079037
:10F5F000BDF87800BDF8281049420844401E00B20A
:10F6000006900C9B2A9A0799FCF794FB229ADDE955
:10F610002501FDF79FFF0C9008980090BDF87E1023
:10F62000BDF82A00404201440998081A00B2079028
:10F63000BDF87C00BDF8281049420844401E00B2C5
:10F6400006900C9B2A9A0799FCF774FB0898009087
:10F65000BDF87600BDF82A10494201440998081AFD
:10F6600000B20790BDF87400BDF828100844401C93
:10F6700000B206900C9B2A9A0799FCF75BFB09984D
:10F68000401C00B209900B9909988842FFF60CAF14
:10F69000BDF92800BDF92A10401A002805DDBDF982
:10F6A0002800BDF92A10401A04E0BDF92A00BDF96E
:10F6B0002810401A0B99884275D10F98ADF8280090
:10F6C0000F98ADF82A000F98C0EB00212198B1FBEC
:10F6D000F0F0C0B22290229ADDE92501FDF73AFF51
:10F6E0000E90229ADDE92510FDF734FF0D90239846
:10F6F0004010089008980090BDF87200BDF82810DE
:10F70000084400B20790BDF87010BDF82A00084404
:10F7100000B206900D9B2A9A0799FCF70BFB0898FC
:10F720000090BDF87A00BDF82A10084400B2079096
:10F73000BDF87800BDF828104942084400B2069090
:10F740000D9B2A9A0799FCF7F5FA08980090BDF8E6
:10F750007E00BDF828104942084400B20790BDF869
:10F760007C00BDF82A104942084400B206900E9B66
:10F770002A9A0799FCF7DEFA08980090BDF87600FF
:10F78000BDF82A104942084400B20790BDF8741031
:10F79000BDF82800084400B206900E9B2A9A0799EB
:10F7A000FCF7C8FA00BF00BF2DB000BD2DE9FF4F28
:10F7B00089B0044615469A46E88886B2FBF78DF86C
:10F7C000074601F0FFFC089068880790A88806901B
:10F7D000204600F04DFD8046204600F042FD04909A
:10F7E000BAF1FF0F01D1287A03E0287A00FB0AF072
:10F7F00000120390424630460499FDF70BFF06467F
:10F8000008EBD871B6EB610F02DD0DB0BDE8F08FEB
:10F810002088ADF80400A088ADF80800BDF81C00F1
:10F82000BDF8181088422DD16088304400B2ADF880
:10F830000600E088801B00B2ADF80A00E888D0B16D
:10F84000089860B1BDF80600801C00B2ADF8060053
:10F85000BDF80A00801E00B2ADF80A000BE0BDF84A
:10F860000600401C00B2ADF80600BDF80A00401EBC
:10F8700000B2ADF80A0001A8039B079A0A99FCF7A9
:10F8800068FB43E0608830440FFA80F9E088801B11
:10F890000FFA80FBE88890B1089840B109F10200A6
:10F8A0000FFA80F9ABF102000FFA80FB07E009F1D3
:10F8B00001000FFA80F9ABF101000FFA80FBB9F1FA
:10F8C000000F01DA4FF000094F461CE0ADF806705A
:10F8D000ADF80A70B4F90600BDF90610401AC0EB85
:10F8E0000020B0FBF8F0C0B20590DDE905210798D3
:10F8F000FDF730FE009001A8039B009A0A99FCF7DF
:10F9000028FB781C07B25F45E0DD00BF00BF7CE745
:10F910002DE9FF4F95B082461646FAF7DEFF814685
:10F9200001F050FC1490B6F90650B6F9127050462A
:10F9300000F097FC1390504600F09AFC1290A8B289
:10F94000DDE91221FDF766FE05B2149800EB4000D8
:10F95000284405B21498384407B2281D20F003004B
:10F960001190119840001190F81C00F0FC001090CC
:10F9700010981090DDE910218818FCF7EBF80F9033
:10F98000DDF83C80DDF83C80119808EB000B2A463E
:10F990000DA90EA802F0E0F80FE0BDF83800BDF99F
:10F9A0003A1028F81100BDF83A00BDF9381028F8CF
:10F9B00011000DA90EA802F0E2F80EA802F0D4F88A
:10F9C0000028EAD11898FF2801D1307A03E0307A74
:10F9D0001899484300120C90002409E0381B0C9938
:10F9E00048434008B0FBF7F00BF80400601C04B279
:10F9F000BC42F3DBBAF80000284400B2ADF81C00AA
:10FA0000BAF80600401B401C1499401A00B2ADF829
:10FA10001E00BAF80400401B00B2ADF81800BAF896
:10FA20000600401B401C1499401A00B2ADF81A00A1
:10FA300000246BE0BDF81C00001B00B2ADF82C00E8
:10FA4000BDF81E0038F81410084400B2ADF82E00BE
:10FA5000BDF81800204400B2ADF82800BDF81A0027
:10FA600038F81410084400B2ADF82A000CB9002090
:10FA700005E0601E38F9100038F91410401A00B281
:10FA800003904FF000093DE0039818B91BF80900F6
:10FA9000049009E01BF809100398A9EB00001BF87B
:10FAA000000008444008049004980090328A0292B2
:10FAB000BDF92E10BDF92C001346169AFCF73AF941
:10FAC000BDF82E00401C00B2ADF82E00BDF9280094
:10FAD000BDF91C1088420BDD04980090328A029216
:10FAE000BDF92A10BDF928001346169AFCF722F931
:10FAF000BDF82A00401C00B2ADF82A0009F101004F
:10FB00001FFA80F9B945BFDB601C04B2AC4291DD3D
:10FB1000BDF81C00401C00B2ADF82000BDF81E006E
:10FB2000284400B2ADF82200BDF81800401E00B213
:10FB3000ADF82400BDF82200ADF8260000200590A5
:10FB400019E005981BF80030308A0246049008A896
:10FB50001699FCF7FEF9BDF82200401C00B2ADF882
:10FB60002200BDF82600401C00B2ADF82600059822
:10FB7000401C80B205900598B842E2DB19B0BDE8A0
:10FB8000F08F2DE9F04F8DB004468B46174699460D
:10FB9000FAF7A3FE019001F015FB0546B7F90660E0
:10FBA000B7F912000C90204600F05BFB0B9020464A
:10FBB00000F05EFB0A90B0B2DDE90A21FDF72AFDF4
:10FBC00006B2701906B2A088401C401B00B2ADF806
:10FBD000200060883044284400B2ADF82200BDF80F
:10FBE0002000ADF82400E088801B401B00B2ADF877
:10FBF00026002088401E284400B2ADF81800608816
:10FC00003044284400B2ADF81A00BDF81800ADF831
:10FC10001C00E088801B401B00B2ADF81E0020884D
:10FC20003044284400B2ADF810006088401E2844DB
:10FC300000B2ADF81200A088801B401B00B2ADF8E6
:10FC40001400BDF81200ADF8160020883044284496
:10FC500000B2ADF80800E088401C401B00B2ADF8CF
:10FC60000A00A088801B401B00B2ADF80C00BDF854
:10FC70000A00ADF80E004FF0010855E019F808A091
:10FC8000388A534602465946019008A8FCF761F9A4
:10FC9000BDF82000401C00B2ADF82000BDF82400E3
:10FCA000401C00B2ADF82400388A5346024659463B
:10FCB000019006A8FCF74DF9BDF81800401E00B2EF
:10FCC000ADF81800BDF81C00401E00B2ADF81C00D5
:10FCD000388A534602465946019004A8FCF739F980
:10FCE000BDF81200401E00B2ADF81200BDF81600BB
:10FCF000401E00B2ADF81600388A534602465946F7
:10FD0000019002A8FCF725F9BDF80A00401C00B2DA
:10FD1000ADF80A00BDF80E00401C00B2ADF80E00B0
:10FD200008F101000FFA80F80C988045A6DD0DB0AF
:10FD3000BDE8F08F2DE9FF4F99B080469146FAF764
:10FD4000CCFD039001F03EFA8246B9F90650B9F9AC
:10FD50001270404600F085FA1890404600F088FA8C
:10FD60001790A8B2DDE91721FDF754FC05B205EBA9
:10FD70000A0005B27800401C00B21690E819001D78
:10FD800020F0030015901598400015901698C01C9F
:10FD900020F003001490149880001490E819001DBE
:10FDA00020F00300139013981390DDE914210A4406
:10FDB00013995018FBF7CEFE1290129E129E1598C2
:10FDC00030441190DDE914100844129E3044109024
:10FDD000304615990DF01FFF2A460EA90FA801F015
:10FDE000BBFE0FE0BDF83C00BDF93E1026F8110047
:10FDF000BDF83E00BDF93C1026F811000EA90FA871
:10FE000001F0BDFE0FA801F0AFFE0028EAD11C985A
:10FE1000FF2802D199F8080004E099F808001C991D
:10FE2000484300120D9000240EE01698001B0D9917
:10FE300049004843010216984043B1FBF0F1119884
:10FE400040F82410601C04B216988442EDDBB8F828
:10FE50000400401BA0EB0A0000B2ADF82000B8F887
:10FE60000600401BA0EB0A0000B2ADF82200B8F873
:10FE70000400401BA0EB0A0000B2ADF81C00B8F86B
:10FE800002002844504400B2ADF81E00B8F800004B
:10FE90002844504400B2ADF81800B8F80600401BE2
:10FEA000A0EB0A0000B2ADF81A00B8F80000284430
:10FEB000504400B2ADF81400B8F802002844504491
:10FEC00000B2ADF81600002420E100200490834623
:10FED00044E00022794208B22DE02318002B06DA14
:10FEE00036F81430EB1AA3EB0B0319B20DE023180C
:10FEF000AB4200DD21E0231836F8133036F814C089
:10FF0000A3EB0C03A3EB0B0319B27B42994204DA77
:10FF1000F84201D1012304930FE0B94203DD119BA4
:10FF20001B681A4405E0A7EB010C119B53F82C3019
:10FF30001A44411C08B2B842CFDD00BFC2F3072308
:10FF4000109901F80B30049921B10BF101011FFA4E
:10FF500081FB06E00BF101001FFA80FBE819584510
:10FF6000B7DA00BF36F81400BDF81C100844401C76
:10FF700000B2ADF83000BDF81E00001B00B2ADF8B5
:10FF8000320036F81400BDF820100844401C00B2BE
:10FF9000ADF82C00BDF82200204400B2ADF82E00D0
:10FFA000BDF8140036F81410401A401E00B2ADF827
:10FFB0002800BDF81600001B00B2ADF82A00BDF8FD
:10FFC000180036F81410401A401E00B2ADF8240094
:10FFD000BDF81A00204400B2ADF8260001200390BD
:10FFE00087E0BDF92800BDF91410884214DABDF984
:10FFF0002A00BDF9161088420EDA03991098405C69
:020000040801F1
:100000000090B9F810200292BDF92A10BDF928001D
:1000100013461A9AFBF78EFEBDF92400BDF918109D
:10002000884214DABDF92600BDF91A1088420EDDA7
:1000300003991098405C0090B9F810200292BDF925
:100040002610BDF9240013461A9AFBF773FEBDF97A
:100050003000BDF91C10884214DDBDF93200BDF935
:100060001E1088420EDA03991098405C0090B9F88F
:1000700010200292BDF93210BDF9300013461A9AD1
:10008000FBF758FEBDF92C00BDF92010884214DDA5
:10009000BDF92E00BDF9221088420EDD039910989B
:1000A000405C0090B9F810200292BDF92E10BDF905
:1000B0002C0013461A9AFBF73DFEBDF82C00401C9D
:1000C00000B2ADF82C00BDF82400401E00B2ADF81F
:1000D0002400BDF83000401C00B2ADF83000BDF87F
:1000E0002800401E00B2ADF828000398401C80B2E2
:1000F000039003985845FFF674AF2CB94A46404622
:10010000109B1A99FFF73DFD601C04B2E819A0424C
:10011000BFF6DBAE1DB0BDE8F08F2DE9FC4706460B
:100120000F4615469846B5F90640304600F099F856
:100130008146304600F09CF88246A0B252464946BD
:10014000FDF768FA04B23146684600F085F8BDF85C
:100150000000204400B2ADF80000BDF80400001B10
:1001600000B2ADF804006946384601F0AAFC08B1B7
:10017000BDE8FC873146684600F06EF8BDF8020025
:10018000204400B2ADF80200BDF80600001B00B22A
:10019000ADF806006946384601F093FC00B1E7E788
:1001A000287D012806D143462A4639463046FFF7C6
:1001B000C1FD07E0287D28B943462A463946304626
:1001C000FFF7A6FB00BFD3E72DE9F04105460E4639
:1001D00014461F46284600F04BF8012804DB284649
:1001E00000F03FF8012801DABDE8F081608A28B10B
:1001F0003B46224631462846FFF78FFF31462846C8
:1002000001F042FC00B9EFE7207A10280DDD3B46F3
:10021000224631462846FFF7C9FAE08828B13B4616
:10022000224631462846FEF7ADFCA08990B1A07B5E
:1002300080B1E07B10280DDB3B4622463146284644
:10024000FEF767FAE08828B13B4622463146284649
:10025000FDF702FA00BFC7E70A6802604A68426019
:100260007047014688880A88801A401C00B270478F
:100270000146C8884A88801A401C00B270470000B6
:100280002DE9F047074689467C48008810B90020D0
:10029000BDE8F0877A480668002514E005EB850084
:1002A00006EBC000406A774988420ADD05EB85000D
:1002B00006EBC000406A401E05EB850106EBC1015C
:1002C0004862681C85B26D4800888542E6DB0024E0
:1002D000002518E005EB850006EBC0004068B84239
:1002E0000FD105EB850006EBC004616AA0690844E4
:1002F0006062606AB0F57A7F02DD4FF47A70606206
:1003000005E0681C85B25D4800888542E2DB00BFDD
:10031000002C44D1344601250DE005EB850006EBA9
:10032000C000406A616A884203DA05EB850006EB8B
:10033000C004681C85B2514800888542EDDB6068C6
:1003400010B1204600F038FC01F023F8824600206E
:10035000A0614A463946204600F0D4FB8046B8F1F9
:10036000000F0FD1204600F027FC242120460DF07D
:1003700074FC282120460DF070FC4FF000406062B4
:10038000002085E700206062A06918B9504601F09E
:100390000BF8A061A06908B90120A06100BF204648
:1003A00076E770B5064636480568002423E004EB7E
:1003B000840005EBC0004068B04200D0CEB904EB29
:1003C000840005EBC000406828B104EB840105EB14
:1003D000C10000F0F1FB04EB840105EBC100242116
:1003E0000DF03BFC04EB840105EBC10028210DF06E
:1003F00034FC601C84B2214800888442D7DB70BD85
:1004000070B505461E48006830B10020FFF7C9FFEF
:100410001B48006801F07FFF05EB8501C80001F073
:100420004AFF174908600846006808B900BFFEE7A0
:100430001348006818B900201049088070BD0F48A3
:100440000580002413E004EB84010D4A126802EBDE
:10045000C10024210DF001FC04EB8401084A12685C
:1004600002EBC10028210DF0F8FB601C84B20348A8
:1004700000888442E7DB00BFE0E700002C01002099
:100480009C0100200100008070B506460D462C6AD4
:100490004CB1206810B1206801F03DFF204601F00A
:1004A0003AFF0020286270BDC16070472DE9FF4F00
:1004B00087B004460E469046217C01F01F00FCF7F1
:1004C00035FA8346012000FA0BF0401E80B20690F8
:1004D0000027B9460025207C00F01F00072806D021
:1004E000082819D009282DD00A284CD140E02069CD
:1004F000C0F38A20C710208AC0F3822008B1781C7C
:1005000007B207FB08F000EBE6000544083506F0EB
:100510000700C0F1070936E02069C0F38A20871080
:10052000208AC0F3812008B1781C07B207FB08F0CD
:1005300000EBA6000544103506F003000621A1EBF0
:10054000400920E02069C0F38A204710208AC0F3C8
:10055000802008B1781C07B207FB08F000EB6600AA
:100560000544403506F001000421A1EB80090AE0B2
:100570002069C0F38A2707FB0860054405F58065FC
:100580004FF0000900BF00BF206A059000200490D2
:10059000207B20B9606881682944049104E0002030
:1005A00004900BB0BDE8F08F0020039014980190E8
:1005B0004FF0000A25E0DDE90310415C069800FADF
:1005C00009F0084040FA09F0029005980168029885
:1005D00001EB4001019800EB4A0009880180A9EB7A
:1005E0000B004FFA80F9B9F1000F06DACBF10800E1
:1005F0004FFA80F90498401C04900AF101000FFAA8
:1006000080FA0A988245D6DB0120CAE72DE9FF4F20
:100610008DB004460D469146FAA000680C90FAA0F1
:1006200000680B90F9A30FCB07AE0FC6A068008E31
:100630000690002710E0BDF81800C1B207EB470292
:100640001A988154BDF81800020A07EB4700401CB5
:100650001A990A54781C07B210988742EBDB0020E5
:100660000590217C01F01F00FCF760F98246012112
:1006700001FA0AF0401E80B2049000264FF00008F4
:100680004FF0000B207C00F01F000B2806D00C2838
:100690001AD00D282FD00E284DD143E02069C0F389
:1006A0008A20C610208AC0F3822008B1701C06B2CE
:1006B00006FB09F000EBE500804405F00700C0F1FF
:1006C000070B0CA8059036E02069C0F38A2086103D
:1006D000208AC0F3812008B1701C06B206FB09F025
:1006E00000EBA500804405F003000621A1EB400BC0
:1006F0000BA805901FE02069C0F38A204610208ACD
:10070000C0F3802008B1701C06B206FB09F000EBB4
:100710006500804405F001000421A1EB800B07A8CF
:10072000059008E02069C0F38A2606FB0950804442
:100730004FF0000B00BF00BF00200390207B20B9CA
:10074000606881684144039104E00020039011B087
:10075000BDE8F08F00200290002728E0DDE90210BC
:10076000415C049800FA0BF0084040FA0BF001904D
:10077000207C00F01F000E2801D1019902E00199B0
:100780000598415C07EB4700801C1A9A1154ABEBAB
:100790000A004FFA80FBBBF1000F06DACAF108002D
:1007A0004FFA80FB0398401C0390781C07B2109806
:1007B0008742D3DB0120CAE730B50546039C002001
:1007C00030BD2DE9F84F82460C4616461F46DDE93E
:1007D0000A854FF00009207C00F01F00042809D092
:1007E000207C00F01F00052804D0207C00F01F00B2
:1007F00006280BD1207B012845D143463A46314695
:1008000020460095FFF7D8FF81463CE0207C00F0B1
:100810001F000B280ED0207C00F01F000C2809D0F0
:10082000207C00F01F000D2804D0207C00F01F0069
:100830000E2808D143463A46314620460095FFF738
:10084000E5FE81461FE0207C00F01F0007280ED047
:10085000207C00F01F00082809D0207C00F01F0039
:10086000092804D0207C00F01F000A2808D1434644
:100870003A46314620460095FFF718FE814602E0D1
:100880000020BDE8F88F4846FBE7816070472DE9FE
:10089000FC5F80460C46207B012802D10020BDE889
:1008A000FC9F207C00F01F05042D03D0052D01D0F6
:1008B000062D0AD1207B20B9606880686061012024
:1008C000EDE7002060610120E9E7072D05D0082D44
:1008D00003D0092D01D00A2D5AD12846FCF726F85D
:1008E0008146012000FA09F7206A60B9042001F06E
:1008F000E2FC2062206A18B9206A08B900BFFEE74E
:100900000021206A0160266A780001F0D4FC306082
:10091000207B012801D10020C1E762689168002294
:1009200010462EE001EB800A9AF8022001EB800AC3
:100930009AF8013011F820C04FEADC0BBDF800A096
:100940006BF3040ACDF800A04FEA930BBDF800A0AA
:100950006BF34A1ACDF800A04FEAD20BBDF800A005
:100960006BF3CF2ACDF800A0BDF800B0DA46CDF881
:1009700004A0326802EB4002BDF804301380421C30
:100980001046B842CED300BF00206061012086E748
:100990000B2D05D00C2D03D00D2D01D00E2D03D124
:1009A0000020606101207AE721464046FFF76CFD98
:1009B000002074E7416070472DE9F04107460D467D
:1009C00014462846FCF708FB06463EBB287800F094
:1009D0001F01042901DB0E2902DD0020BDE8F081A2
:1009E0002868820A206862F3942020602868420DFB
:1009F000206862F35F5020602878226860F3040268
:100A0000226021E000FF00000055AAFF0011223300
:100A1000445566778899AABBCCDDEEFFFFE7022E2E
:100A200010D10121206861F3942020602068C0F378
:100A3000140000F500102060206820F01F000B302B
:100A4000206001E00020C9E70120C7E7016070478E
:100A500010B5644801F0E2F904460CB900BFFEE7A6
:100A60000CB9002010BD002020606060A060E06034
:100A70002046F7E710B510215A4801F096F9FFF724
:100A8000E7FF04461CB90CB900BFFEE710BDAFF28A
:100A9000D7012046FFF7DAFFAFF20D212046FFF71E
:100AA00089FFAFF2E1212046FFF7EFFEAFF22761A9
:100AB0002046FFF7F9FC00BFE8E72DE9F0410646C4
:100AC0000D46286820F0E00028600027454801F026
:100AD000CFF9044610E00027206840B12A4631468D
:100AE0002046236898470746012F00D106E021469B
:100AF0003C4801F01EFA0446002CECD100BF3846F9
:100B0000BDE8F0812DE9F04104460F469046C4F857
:100B1000088067603846FCF75FFA20730020206287
:100B20000026304801F0A4F9054620E0286808B105
:100B3000686800B916E004F11002394628462B68AF
:100B400098470646012E00D00CE00020E06160616D
:100B50002560214628466A6890470646012E00D146
:100B600007E000BF29461F4801F0E3F90546002DC4
:100B7000DCD100BF1EB9242120460DF06EF83046AE
:100B8000BDE8F0812DE9FC4704460D4616461F4698
:100B9000DDF828804FF000092068806848B1CDE971
:100BA0000078206833462A462146D0F808C0E0473E
:100BB00081464846BDE8FC8710B50446206830B140
:100BC0002068C06818B120682146C268904710BDEF
:100BD00010B504462146034801F0BBF9204601F058
:100BE0009AFB10BDD02E002070B504460D46294654
:100BF00020466268904770BD2DE9F04104460D46DD
:100C000016461F463B46324629462046D4F800C0C9
:100C1000E047BDE8F0812DE9FC4106460C4615464B
:100C20002B46224669463046FFF7E6FF07461FB1CE
:100C3000BDF80000BDE8FC810020FBE702461088FB
:100C40000B88C01A70472DE9FC4780460E4616B93E
:100C50000020BDE8FC87D8F80C406069B04201D1A3
:100C6000A069F6E70025AEE005EB8501A06850F825
:100C70002100301A019005EB8501A06800EB81008E
:100C800080880199884200D29BE0002705EB85010E
:100C9000A06800EB8100807C00F0030040B905EB08
:100CA0008501A06800EB8100C0880199471884E0A5
:100CB00005EB8501A06800EB8100807C00F003005B
:100CC00001280FD105EB8502A16801EB8201C868FC
:100CD00005EB8502A16801EB8201C988019A825C5B
:100CE0008F186AE005EB8501A06800EB8100807C2D
:100CF00000F00300022827D1AA48009005EB8503E5
:100D0000A06800EB8300028A05EB8503A06800EB76
:100D100083000223816801A802F01EF98146B9F11F
:100D2000000F10D005EB8502A16801EB82018968F4
:100D3000A9EB0100400805EB8502A16801EB8201E7
:100D4000C9880F1800BF38E005EB8501A06800EBEB
:100D50008100807C00F0030003282ED19148009090
:100D600005EB8503A06800EB8300028A05EB850391
:100D7000A06800EB83000223816801A802F0ECF870
:100D80008146B9F1000F17D005EB8503A26802EB8D
:100D900083029268A9EB0200400805EB8503A26874
:100DA00002EB8302D16805EB8503A26802EB8302A4
:100DB000D2880B5CD71800BF00BF6661A7613846B8
:100DC00047E7681C85B2608AC0F30900A8423FF774
:100DD0004BAF66610020A06100BF3AE72DE9F0410A
:100DE00005468846EE6841462846FFF72CFF074631
:100DF00017B90020BDE8F081706800EBC7042CB182
:100E000030682168C1F313010844F3E70020F1E7DB
:100E100030B5024614460B4620881D88A84203D0F0
:100E200020881D88401B30BD60885D88401BFAE724
:100E300030B5024614460B4620781D78A84203D0F0
:100E400020781D78401B30BD60785D78401BFAE744
:100E50002DE9FC5F80460D461646D8F80C704FF021
:100E6000000A788AC0F34030002841D1FC68A068AD
:100E7000C0F30160D8B9D4F8009005EB062080B229
:100E8000019049480090A06820F07F420223494623
:100E900001A802F061F88346BBF1000F06D0ABEB6E
:100EA00009004008616811F900A000BF1FE0A068B8
:100EB000C0F3016001281AD1D4F8009005EB062098
:100EC00001903A480090A06820F07F4204234946F0
:100ED00001A802F041F88346BBF1000F06D0ABEB4E
:100EE00009000009616811F900A000BF00BF13E00C
:100EF000F8684368595D43689A5D00290BDD002A54
:100F000009DD531E4C1E90F80DC004FB0C33046821
:100F1000E35C4FFA83FA00BF5046BDE8FC9F2DE921
:100F2000FF5F80460C46D8F80C6040460299FFF7F8
:100F30008AFE07461FB9002004B0BDE8F09F4FF0BD
:100F40000009F06870B140460399FFF77CFE8346C4
:100F5000BBF1000F05D05A4639464046FFF778FFEF
:100F6000814600BF706800EBC7052868010D308A14
:100F700000FB09F001EB201A0AF108004FEA101AF1
:100F8000A4F800A06879E0702879A070A879207191
:100F9000E87940B26071708AC0F38220A0710120AC
:100FA000CAE700003D0C0108310E0108110E0108CE
:100FB00038B50446202120460CF04FFE0020E060AA
:100FC000F02020804FF4A070608000206060A06856
:100FD00020F00200A060A74800680090BDF8000063
:100FE000A083A06820F00100401CA0600020606188
:100FF00038BD2DE9F04104460F4615461E461C211A
:1010000020460CF02AFE276065602068A060E6603C
:10101000BDE8F08170B50546974800F0FFFE044634
:1010200024B90CB900BFFEE7002070BD202229467C
:1010300020460CF079FD202104F59E700CF00DFE89
:101040004FF4807104F13C000CF0E5FD442104F103
:10105000240000F0AAFE8948006808B987480460A7
:101060008648066804600020C4F85C010021084638
:10107000F8F76CFA206300210846F8F767FA606316
:1010800000210846F8F762FAA0637D49606BF9F722
:101090000AFA7B49A06BF9F706FA206BF8F752F8C9
:1010A00076480660234603221E21764801F087FB1E
:1010B0002062206A08B900BFFEE7206A08B9002054
:1010C000B3E7206A01F09AFB2046AEE76B48006860
:1010D000704700B5014611B9FFF7F8FF014611B995
:1010E0004FF4A07000BD087AC0F3400010B9B1F908
:1010F0000200F7E7B1F90000F4E700B5014611B9C5
:10110000FFF7E4FF014609B9F02000BD087AC0F3FB
:10111000400010B9B1F90000F7E7B1F90200F4E7B7
:101120002DE9F04104460E462022314620460CF0BF
:10113000FBFC04F1240000F09BFE054612E0204673
:10114000FFF7C7FF07462046FFF7D7FF80463A461E
:1011500041462846F9F705F9294604F1240000F034
:10116000E8FE0546002DEAD1BDE8F081434908605C
:1011700070472DE9F04105460026FFF7A7FFA8427A
:1011800000D10126002000F0CCF8044608E0E06819
:10119000A84201D10020E060204600F0C2F80446D9
:1011A000002CF4D12946344800F0D3FE284601F043
:1011B000B2F82EB1304800F05BFE0746FFF7D6FFCD
:1011C000BDE8F08100B5014611B9FFF77FFF014688
:1011D00009B9002000BD087A00F00100FAE7416873
:1011E000896921F0010142689161704710B5044698
:1011F0001CB9214800F03CFE10BD21461E4800F0FD
:1012000098FEF9E70146486870470146B1F85C016D
:10121000C0F309007047B0F85C21C2F309028A42AA
:1012200003DA0022C0F85C2106E0B0F85C21C2F3CA
:101230000902521AC0F85C217047014648680068EC
:1012400020B14868406808B1012070470020FCE7E1
:1012500000B502461088518810FB01F31046FFF7D5
:10126000ECFF28B15068C068984201D1012000BD50
:101270000020FCE77C610008882E00208801002007
:10128000AC2B002031AE000810B504461C212046CE
:101290000CF0E3FC002020700A20207514206075FB
:1012A0004FF4C870E0826420208310BD70B50546FD
:1012B000E86810B9FFF70AFFE860E86808B900209D
:1012C00070BD2D4800F0AAFD044624B90CB900BF3A
:1012D000FEE70020F4E75C2120460CF0BEFC1C2257
:1012E000294620460CF020FC94F84C0020F0020027
:1012F000801C84F84C00002020656065A0652346B2
:1013000003221E211D4801F05AFA20612046D7E72A
:1013100070B504460D461C22294620460CF004FCFC
:1013200070BD10B504461CB9134800F0A1FD10BDF6
:101330002146114800F0FDFDF9E770B504460D4661
:101340000026002028606860A860E86020780128F6
:1013500004D1208C2880608C688004E020780228EA
:1013600001D1606A6860606820B1294620466268E1
:1013700090470646304670BD942E0020438E0008EC
:101380000021104A11701049096801440E4A116089
:10139000704700BF01210B4A11700B4908681146C4
:1013A00009780029F6D0704710B50346FFF7F1FF22
:1013B00004469C4201D3E31A01E05B4223441846F1
:1013C00010BD0000900100208C01002010B58AB0F3
:1013D000044694F82000C0F3400020B994F820009F
:1013E00000F0010070B194F82000C0F34000F0B9A3
:1013F00094F8200000F00100C8B194F82000C0F378
:101400008000A0B12422214601A80CF08DFB2146CA
:10141000FD4800F09EFD204600F07DFF0120FB49C5
:101420000870049810B101A8049988471FE0E08B68
:10143000404200B2608394F8200000F00100B0B197
:1014400094F82010C1F3800119B9A18B494209B267
:1014500061831034217C8908C943227C61F38202B4
:1014600022742068616821606060103C00BFE7481A
:1014700000780AB010BD2DE9F0410746E24800F0BF
:10148000F7FC044608E0206A20F0080020622146AC
:10149000DD4800F04EFD0446002CF4D1DC48006825
:1014A000FFF782FF0646D84800F0E2FC04463CE025
:1014B0000020D649087094F82000C0F3C00038BB63
:1014C000206A20F0080008302062608B304400B2AF
:1014D0006083B4F91A0000281ADBB4F91A00218BD2
:1014E000884202DD208B00B260832046A1688847D5
:1014F0000546606818B129B2D4E900029047B4F9F2
:101500001A00218B884202DB2046FFF75FFF00BFF5
:10151000BE48007820B1BC4800F0AAFC044604E0B4
:101520002146B94800F005FD0446002CC0D1FFF764
:1015300030FFB7490860BDE8F08110B52421B248FA
:1015400000F033FCFFF725FFB149086000230322B8
:101550001E21B04801F033F910BD10B50146088BCB
:10156000B1F91A40A04202D14FF4806205E0B1F90E
:101570001A0080020C8B90FBF4F2D1E90440001BAE
:1015800000FB02F39B120869034418B210BD10B5AA
:101590000446242120460CF060FB4FF4FA702083AF
:1015A0000020206164206061AFF25100A06010BD96
:1015B0002DE9F04107460D464FF00008924800F033
:1015C00057FC044617E021468F4800F0B2FC06465F
:1015D0002068B8420ED16068A84200D055B92146B3
:1015E000894800F0B6FC204600F095FE01208749AE
:1015F000087080463446002CE5D14046BDE8F081B5
:1016000070B50546686818B1D5E90001FFF7D0FF4D
:101610007D4800F003FC04460CB900BFFEE704B9A6
:1016200070BD95F8200020F0040085F820002422E9
:10163000294620460CF078FA606820B1238A19B256
:10164000D4E90002904701207049087000BFE7E725
:1016500070B500256C4800F00BFC044606E0681CE1
:1016600085B22146684800F064FC0446002CF6D19F
:101670002846691C8DB270BD30B504460B46981AD9
:10168000002801DD981A00E0D01A05464FF47A7060
:10169000684390FBF4F1B1F5803F01D34FF6FF7141
:1016A00001B9491C88B230BDF8B50446208BB4F9A5
:1016B0001A10884202D14FF4806505E0B4F91A008F
:1016C0008002218BB0FBF1F54FF4806001231A46B4
:1016D00000210090284600F05AFD0746D4E9041086
:1016E000401A00FB07F6B6122069064430B2F8BD76
:1016F000F8B50446208BB4F91A10884202D14FF491
:10170000806505E0B4F91A008002218BB0FBF1F589
:101710004FF48060431E1A4600210090284600F0D6
:1017200036FD0746D4E90410401A00FB07F6B6124E
:101730002069064430B2F8BDF8B50446208BB4F9F0
:101740001A10884202D14FF4806505E0B4F91A00FE
:101750008002218BB0FBF1F54FF480604FF467738A
:10176000642200210090284600F011FD0746D4E9CC
:101770000410401A00FB07F6B6122069064430B286
:10178000F8BDF8B50446208BB4F91A10884202D18E
:101790004FF4806505E0B4F91A008002218BB0FB9C
:1017A000F1F54FF4806040F214534FF416720021AB
:1017B0000090284600F0EBFC0746D4E90410401ADC
:1017C00000FB07F6B6122069064430B2F8BD2DE9D9
:1017D000F8430546288BB5F91A10884202D14FF418
:1017E000806405E0B5F91A008002298BB0FBF1F4A2
:1017F000D5E90410461AB4F5CC7F0DD240F6C410DA
:101800006043840A4BE00000B82E002098010020BD
:101810009401002077140108B4F5CC7F0DD340F279
:101820006620844209D2A4F5CC7404EB8404C4F588
:101830008064062096FBF0F631E040F26620844298
:101840000BD340F23330844207D2A4F2662404EB77
:101850008404062096FBF0F621E040F23330844207
:101860000ED3B4F5667F0BD8A4F2333404EB8400B6
:101870004400C4F58064F11706EB11710E110EE0FF
:10188000B4F5667F0BD9B4F5806F08D8A4F299340B
:1018900004EB84004400F11706EB11710E11B4F54E
:1018A000806F01D94FF4806400204FF448734FF4E7
:1018B000806211460090204600F069FC804608FBDB
:1018C00006F7BF126869C71B38B2BDE8F883014646
:1018D000B1F91A000A8B904202DB888A00B2704785
:1018E000088A00B2FBE710B5029C01804280838029
:1018F000C48010BD02880A44521E12B28280704712
:1019000042880A44521E12B2C2807047F0B50346A4
:101910000C46154600BF98881988401A401C00B232
:10192000064600BFD8885988401A401C00B20746B6
:101930001C805D8031461846FFF7DCFF39461846AB
:10194000FFF7DEFFF0BD10B50146B1F90420B1F993
:101950000030D21A521CB1F90630B1F902401B1BFB
:101960005B1C02FB03F010BD30B50346B1F900402B
:10197000B2F90050AC4202DDB1F9004001E0B2F929
:1019800000401C80B1F90240B2F90250AC4202DDC5
:10199000B1F9024001E0B2F902405C80B1F90440C3
:1019A000B2F90450AC4202DAB1F9044001E0B2F9F4
:1019B00004409C80B1F90640B2F90650AC4202DA0C
:1019C000B1F9064001E0B2F90640DC800120B3F92C
:1019D0000040B3F90450AC4205DCB3F90240B3F95E
:1019E0000650AC4200DD002030BD10B5B1F900302A
:1019F000B2F90040A34202DAB1F9003001E0B2F9D5
:101A000000300380B1F90230B2F90240A34202DA99
:101A1000B1F9023001E0B2F902304380B1F904308B
:101A2000B2F90440A34202DDB1F9043001E0B2F999
:101A300004308380B1F90630B2F90640A34202DDDA
:101A4000B1F9063001E0B2F90630C38010BD10B51F
:101A500002460020B1F90030B2F90040A34212DB87
:101A6000B1F90030B2F90440A3420CDCB1F9023004
:101A7000B2F90240A34206DBB1F90230B2F90640E6
:101A8000A34200DC012010BD0246B2F90000B1F90A
:101A90000430984213DCB2F90400B1F900309842E6
:101AA0000DDBB2F90200B1F90630984207DCB2F959
:101AB0000600B1F90230984201DB01207047002096
:101AC000FCE710B502460020B2F90030B1F9004041
:101AD000A34212DBB2F90230B1F90240A3420CDB9F
:101AE000B2F90430B1F90440A34206DCB2F9063081
:101AF000B1F90640A34200DC012010BD70B50546D7
:101B0000EC68D4E900108847204600F004FC70BD62
:101B10002DE9F04106460F46082000F0CCFB0446B4
:101B200014B90020BDE8F0812346052200210948B0
:101B300000F045FE054625B9204600F0ECFB0020EC
:101B4000F0E726606760EC60284600F060FE012048
:101B5000E8E70000FD1A0108028000234380C2F17B
:101B600001031BB20B8070470146B1F90200B1F9C5
:101B70000020904201DC012070470020FCE74288F1
:101B8000521C12B24280B1F90020002A07DC0B88F7
:101B900042885200521C1A4412B20A800CE0028899
:101BA000521E12B2028042880388D21A5200521C7E
:101BB0000B881A4412B20A80704718B50346D4083D
:101BC000BDF8000064F3040000908C08BDF800002C
:101BD00064F34A100090DC08BDF8000064F3CF20E5
:101BE0000090BDF80040204618BD2DE9F04F85B0AB
:101BF000824689461446CAEB0A204FF4B471B0FB02
